:020000040800F2
:100000000050002045100008911000086D7D000888
:1000100091100008911000089110000800000000E5
:100020000000000000000000000000009110000827
:10003000911000080000000091100008B1A0000815
:10004000911000089110000891100008911000080C
:1000500091100008911000089110000891100008FC
:1000600091100008911000089110000891100008EC
:1000700091100008911000084D3F000891100008F1
:1000800091100008753F00089110000891100008B9
:1000900091100008911000089110000891100008BC
:1000A000911000085D4F0008714F0008FD4E0008D8
:1000B000114F0008214F0008354F0008911000082B
:1000C000911000089110000891100008911000088C
:1000D0009110000875400008954000089110000834
:1000E000911000089110000891100008911000086C
:1000F0009110000891100008494F00089110000865
:100100000000000000000000000000009110000846
:10011000911000089110000891100008911000083B
:10012000911000089110000891100008911000082B
:10013000911000089110000800000000000000006D
:1001400091100008911000089110000800000000B4
:10015000000000000000000000000000000000009F
:10016000000000000000000091100008911000083D
:1001700091100008000000000000000000000000D6
:080180000000000091100008CE
:1001880010B5054C237833B9044810B10448AFF3CF
:1001980000800121217010BDC4050020000000006E
:1001A80074E2010808B5064B1BB106480649AFF3CF
:1001B80000800648016811B1054A02B1904708BDA0
:1001C8000000000074E20108C8050020C4050020F2
:1001D8000000000081F0004102E000BF83F000430E
:1001E80030B54FEA41044FEA430594EA050F08BFCA
:1001F80090EA020F1FBF54EA000C55EA020C7FEA8E
:10020800645C7FEA655C00F0E2804FEA5454D4EB0A
:100218005555B8BF6D420CDD2C4480EA020281EAD4
:10022800030382EA000083EA010180EA020281EA0C
:100238000303362D88BF30BD11F0004F4FEA01315E
:100248004FF4801C4CEA113102D0404261EB41016D
:1002580013F0004F4FEA03334CEA133302D05242F3
:1002680063EB430394EA050F00F0A780A4F10104AF
:10027800D5F1200E0DDB02FA0EFC22FA05F28018E9
:1002880041F1000103FA0EF2801843FA05F35941CF
:100298000EE0A5F120050EF1200E012A03FA0EFC4E
:1002A80028BF4CF0020C43FA05F3C01851EBE37178
:1002B80001F0004507D54FF0000EDCF1000C7EEB95
:1002C80000006EEB0101B1F5801F1BD3B1F5001FD3
:1002D8000CD349085FEA30004FEA3C0C04F10104F2
:1002E8004FEA445212F5800F80F09A80BCF1004F1B
:1002F80008BF5FEA500C50F1000041EB045141EA9D
:10030800050130BD5FEA4C0C404141EB010111F49D
:10031800801FA4F10104E9D191F0000F04BF014648
:100328000020B1FA81F308BF2033A3F10B03B3F126
:1003380020020CDA0C3208DD02F1140CC2F10C02B6
:1003480001FA0CF021FA02F10CE002F11402D8BF14
:10035800C2F1200C01FA02F120FA0CFCDCBF41EAE0
:100368000C019040E41AA2BF01EB0451294330BDAF
:100378006FEA04041F3C1CDA0C340EDC04F114048C
:10038800C4F1200220FA04F001FA02F340EA030063
:1003980021FA04F345EA030130BDC4F10C04C4F1A9
:1003A800200220FA02F001FA04F340EA0300294689
:1003B80030BD21FA04F0294630BD94F0000F83F4D3
:1003C800801306BF81F480110134013D4EE77FEAB6
:1003D800645C18BF7FEA655C29D094EA050F08BF02
:1003E80090EA020F05D054EA000C04BF19461046E3
:1003F80030BD91EA030F1EBF0021002030BD5FEA27
:10040800545C05D14000494128BF41F0004130BD4E
:1004180014F580043CBF01F5801130BD01F00045A2
:1004280045F0FE4141F470014FF0000030BD7FEA15
:10043800645C1ABF194610467FEA655C1CBF0B4610
:10044800024650EA013406BF52EA033591EA030F27
:1004580041F4002130BD00BF90F0000F04BF00211F
:10046800704730B54FF4806404F132044FF0000552
:100478004FF0000150E700BF90F0000F04BF0021CB
:10048800704730B54FF4806404F1320410F0004531
:1004980048BF40424FF000013EE700BF42004FEA2C
:1004A800E2014FEA31014FEA02701FBF12F07F43A9
:1004B80093F07F4F81F06051704792F0000F14BFA6
:1004C80093F07F4F704730B54FF4607401F00045EA
:1004D80021F0004120E700BF50EA010208BF704741
:1004E80030B54FF000050AE050EA010208BF704736
:1004F80030B511F0004502D5404261EB41014FF49F
:10050800806404F132045FEA915C3FF4DCAE4FF0A2
:1005180003025FEADC0C18BF03325FEADC0C18BF89
:10052800033202EBDC02C2F1200300FA03FC20FADA
:1005380002F001FA03FE40EA0E0021FA02F1144427
:10054800C1E600BF70B54FF0FF0C4CF4E06C1CEA3C
:1005580011541DBF1CEA135594EA0C0F95EA0C0FB1
:1005680000F0DEF82C4481EA030621EA4C5123EA24
:100578004C5350EA013518BF52EA033541F4801153
:1005880043F4801338D0A0FB02CE4FF00005E1FB06
:1005980002E506F00042E0FB03E54FF00006E1FB50
:1005A80003569CF0000F18BF4EF0010EA4F1FF0493
:1005B800B6F5007F64F5407404D25FEA4E0E6D41D3
:1005C80046EB060642EAC62141EA55514FEAC520E4
:1005D80040EA5E504FEACE2EB4F1FD0C88BFBCF560
:1005E800E06F1ED8BEF1004F08BF5FEA500E50F111
:1005F800000041EB045170BD06F0004646EA0101D7
:1006080040EA020081EA0301B4EB5C04C2BFD4EB08
:100618000C0541EA045170BD41F480114FF0000E01
:10062800013C00F3AB8014F1360FDEBF002001F06F
:10063800004170BDC4F10004203C35DA0C341BDCE9
:1006480004F11404C4F1200500FA05F320FA04F0BB
:1006580001FA05F240EA020001F0004221F00041EF
:1006680010EBD37021FA04F642EB06015EEA430E62
:1006780008BF20EAD37070BDC4F10C04C4F1200592
:1006880000FA04F320FA05F001FA04F240EA020045
:1006980001F0004110EBD37041F100015EEA430E16
:1006A80008BF20EAD37070BDC4F1200500FA05F236
:1006B8004EEA020E20FA04F301FA05F243EA0203B5
:1006C80021FA04F001F0004121FA04F220EA0200C4
:1006D80000EBD3705EEA430E08BF20EAD37070BD0A
:1006E80094F0000F0FD101F00046400041EB0101EA
:1006F80011F4801F08BF013CF7D041EA060195F0CC
:10070800000F18BF704703F00046520043EB030385
:1007180013F4801F08BF013DF7D043EA0603704772
:1007280094EA0C0F0CEA135518BF95EA0C0F0CD07D
:1007380050EA410618BF52EA4306D1D181EA0301C3
:1007480001F000414FF0000070BD50EA410606BFBD
:100758001046194652EA430619D094EA0C0F02D102
:1007680050EA013613D195EA0C0F05D152EA033647
:100778001CBF104619460AD181EA030101F0004165
:1007880041F0FE4141F470014FF0000070BD41F0AE
:10079800FE4141F4780170BD70B54FF0FF0C4CF488
:1007A800E06C1CEA11541DBF1CEA135594EA0C0FA7
:1007B80095EA0C0F00F0A7F8A4EB050481EA030EF4
:1007C80052EA03354FEA013100F088804FEA0333DB
:1007D8004FF0805545EA131343EA12634FEA0222A9
:1007E80045EA111545EA10654FEA00260EF000416A
:1007F8009D4208BF964244F1FD0404F5407402D2BC
:100808005B084FEA3202B61A65EB03055B084FEA4C
:1008180032024FF480104FF4002CB6EB020E75EB49
:10082800030E22BFB61A754640EA0C005B084FEA71
:100838003202B6EB020E75EB030E22BFB61A7546EE
:1008480040EA5C005B084FEA3202B6EB020E75EB39
:10085800030E22BFB61A754640EA9C005B084FEAB1
:100868003202B6EB020E75EB030E22BFB61A7546BE
:1008780040EADC0055EA060E18D04FEA051545EAAD
:1008880016754FEA06164FEAC30343EA52734FEA56
:10089800C2025FEA1C1CC0D111F4801F0BD141EACF
:1008A80000014FF000004FF0004CB6E711F4801F34
:1008B80004BF01430020B4F1FD0C88BFBCF5E06F14
:1008C8003FF6AFAEB5EB030C04BFB6EB020C5FEA24
:1008D800500C50F1000041EB045170BD0EF0004E79
:1008E8004EEA113114EB5C04C2BFD4EB0C0541EAAB
:1008F800045170BD41F480114FF0000E013C90E6A8
:1009080045EA060E8DE60CEA135594EA0C0F08BF6B
:1009180095EA0C0F3FF43BAF94EA0C0F0AD150EA6A
:1009280001347FF434AF95EA0C0F7FF425AF1046FD
:1009380019462CE795EA0C0F06D152EA03353FF425
:10094800FDAE1046194622E750EA410618BF52EAA2
:1009580043067FF4C5AE50EA41047FF40DAF52EA76
:1009680043057FF4EBAE12E74FEA4102B2F1E043F0
:1009780024BFB3F5001CDCF1FE5C0DD901F0004C7E
:100988004FEAC0024CEA5070B2F1004F40EB8300CE
:1009980008BF20F00100704711F0804F21D113F1FA
:1009A8003872BCBF01F00040704741F480114FEA33
:1009B8005252C2F11802C2F1200C10FA0CF320FABC
:1009C80002F018BF40F001004FEAC1234FEAD323D9
:1009D80003FA0CFC40EA0C0023FA02F34FEA430343
:1009E800CCE77FEA625307D150EA01331EBF4FF0CC
:1009F800FE4040F44000704701F0004040F0FE40E7
:100A080040F40000704700BF80F0004002E000BFE3
:100A180081F0004142001FBF5FEA410392EA030FE1
:100A28007FEA226C7FEA236C6AD04FEA1262D2EB2B
:100A38001363C1BFD218414048404140B8BF5B4230
:100A4800192B88BF704710F0004F40F4000020F0C9
:100A58007F4018BF404211F0004F41F4000121F0DF
:100A68007F4118BF494292EA030F3FD0A2F1010229
:100A780041FA03FC10EB0C00C3F1200301FA03F167
:100A880000F0004302D5494260EB4000B0F5000F8A
:100A980013D3B0F1807F06D340084FEA310102F149
:100AA8000102FE2A51D2B1F1004F40EBC25008BFFB
:100AB80020F0010040EA03007047490040EB0000C5
:100AC80010F4000FA2F10102EDD1B0FA80FCACF1F4
:100AD800080CB2EB0C0200FA0CF0AABF00EBC250F3
:100AE80052421843BCBFD0401843704792F0000FE1
:100AF80081F4000106BF80F400000132013BB5E734
:100B08004FEA41037FEA226C18BF7FEA236C21D0A9
:100B180092EA030F04D092F0000F08BF084670470E
:100B280090EA010F1CBF0020704712F07F4F04D1DC
:100B3800400028BF40F00040704712F100723CBFEF
:100B480000F50000704700F0004343F0FE4040F419
:100B5800000070477FEA226216BF08467FEA2363D7
:100B68000146420206BF5FEA412390EA010F40F4C2
:100B7800800070474FF0000304E000BF10F000430E
:100B880048BF40425FEA000C08BF704743F09643F5
:100B980001464FF000001CE050EA010208BF704710
:100BA8004FF000030AE000BF50EA010208BF704797
:100BB80011F0004302D5404261EB41015FEA010CAC
:100BC80002BF84460146002043F0B64308BFA3F1A4
:100BD8008053A3F50003BCFA8CF2083AA3EBC25386
:100BE80010DB01FA02FC634400FA02FCC2F12002A5
:100BF800BCF1004F20FA02F243EB020008BF20F0DC
:100C08000100704702F1200201FA02FCC2F1200241
:100C180050EA4C0021FA02F243EB020008BF20EA36
:100C2800DC7070474FF0FF0C1CEAD0521EBF1CEA64
:100C3800D15392EA0C0F93EA0C0F6FD01A4480EA52
:100C4800010C400218BF5FEA41211ED04FF000633B
:100C580043EA501043EA5111A0FB01310CF0004067
:100C6800B1F5000F3EBF490041EAD3715B0040EA8D
:100C7800010062F17F02FD2A1DD8B3F1004F40EB5D
:100C8800C25008BF20F00100704790F0000F0CF030
:100C9800004C08BF49024CEA502040EA51207F3AF4
:100CA800C2BFD2F1FF0340EAC250704740F40000CF
:100CB8004FF00003013A5DDC12F1190FDCBF00F0C0
:100CC80000407047C2F10002410021FA02F1C2F16E
:100CD800200200FA02FC5FEA310040F1000053EA0A
:100CE8004C0308BF20EADC70704792F0000F00F058
:100CF800004C02BF400010F4000F013AF9D040EA5E
:100D08000C0093F0000F01F0004C02BF490011F4F1
:100D1800000F013BF9D041EA0C018FE70CEAD153EF
:100D280092EA0C0F18BF93EA0C0F0AD030F0004C6F
:100D380018BF31F0004CD8D180EA010000F0004023
:100D4800704790F0000F17BF90F0004F084691F0E1
:100D5800000F91F0004F14D092EA0C0F01D142021B
:100D68000FD193EA0C0F03D14B0218BF084608D1E4
:100D780080EA010000F0004040F0FE4040F400002E
:100D8800704740F0FE4040F4400070474FF0FF0CC1
:100D98001CEAD0521EBF1CEAD15392EA0C0F93EA08
:100DA8000C0F69D0A2EB030280EA010C49024FEA5A
:100DB800402037D04FF0805343EA111143EA101313
:100DC8000CF000408B4238BF5B0042F17D024FF4CB
:100DD800000C8B4224BF5B1A40EA0C00B3EB510FA6
:100DE80024BFA3EB510340EA5C00B3EB910F24BF8F
:100DF800A3EB910340EA9C00B3EBD10F24BFA3EB14
:100E0800D10340EADC001B0118BF5FEA1C1CE0D1DB
:100E1800FD2A3FF650AF8B4240EBC25008BF20F08E
:100E2800010070470CF0004C4CEA50207F32C2BFE2
:100E3800D2F1FF0340EAC250704740F400004FF07F
:100E48000003013A37E792F0000F00F0004C02BFB0
:100E5800400010F4000F013AF9D040EA0C0093F07A
:100E6800000F01F0004C02BF490011F4000F013BD4
:100E7800F9D041EA0C0195E70CEAD15392EA0C0F3C
:100E880008D142027FF47DAF93EA0C0F7FF470AF74
:100E9800084676E793EA0C0F04D14B023FF44CAFB7
:100EA80008466EE730F0004C18BF31F0004CCAD14C
:100EB80030F000427FF45CAF31F000437FF43CAF88
:100EC8005FE700BF4FF0FF3C06E000BF4FF0010CAA
:100ED80002E000BF4FF0010C4DF804CD4FEA40028C
:100EE8004FEA41037FEA226C18BF7FEA236C11D0D6
:100EF80001B052EA530C18BF90EA010F58BFB2EB89
:100F0800030088BFC81738BF6FEAE17018BF40F008
:100F1800010070477FEA226C02D15FEA402C05D1BC
:100F28007FEA236CE4D15FEA412CE1D05DF8040B41
:100F3800704700BF844608466146FFE70FB5FFF7D4
:100F4800C9FF002848BF10F1000F0FBD4DF808ED8C
:100F5800FFF7F4FF0CBF012000205DF808FB00BF7D
:100F68004DF808EDFFF7EAFF34BF012000205DF8D7
:100F780008FB00BF4DF808EDFFF7E0FF94BF012024
:100F880000205DF808FB00BF4DF808EDFFF7D2FF21
:100F980094BF012000205DF808FB00BF4DF808ED64
:100FA800FFF7C8FF34BF012000205DF808FB00BF31
:100FB8004FEA4002B2F1FE4F0FD34FF09E03B3EB5E
:100FC80012620DD94FEA002343F0004310F0004F9E
:100FD80023FA02F018BF404270474FF000007047F4
:100FE80012F1610F01D1420205D110F0004008BF93
:100FF8006FF0004070474FF00000704742000ED27B
:10100800B2F1FE4F0BD34FF09E03B3EB126209D43B
:101018004FEA002343F0004323FA02F070474FF0F1
:101028000000704712F1610F01D1420202D14FF066
:10103800FF3070474FF00000704700BF002100F0FC
:1010480004B80C4B5B58435004310B480B4B421807
:101058009A42FFF4F6AF0A4A00F003B8002342F8B8
:10106800043B084B9A42FFF4F9AF15F08BF806F0F1
:1010780055FC704798E2010800000020C4050020D4
:10108800C4050020141F0020FFF7FEBF80B584B000
:1010980000AF786039604FF00003FB734FF0000336
:1010A800BB7340F25413C2F200031A684FF4D853CA
:1010B800C0F2B7039A4202D14FF000032CE007F1C7
:1010C8000E034FF053004FF000014FF0010201F002
:1010D8003DFB0346FB73FB7B83F00103DBB2002B74
:1010E80002D1BB7BE52B02D04FF0000314E07B68F4
:1010F8001A7840F2E053C2F200031A703A6841F2DB
:101108002D13C0F6000313603A6841F2DD13C0F6F0
:10111800000353604FF00103184607F11007BD465E
:1011280080BD00BF80B582B000AF40F2E053C2F28C
:1011380000031B78002B2AD04FF01003FB714FF0EF
:1011480053004FF02D014FF0080201F0DFF94FF086
:1011580053004FF031014FF00A0201F0D7F94FF078
:1011680053004FF02C014FF00C0201F0CFF9FB793E
:1011780003F01F03DBB263F07F03DBB2DBB24FF097
:1011880053004FF038011A4601F0C0F917E04FF04C
:1011980053004FF02D014FF0080201F0B7F94FF05E
:1011A80053004FF031014FF00A0201F0AFF94FF050
:1011B80053004FF02C014FF00A0201F0A7F940F25A
:1011C8002203C2F2000340F209121A8007F108074D
:1011D800BD4680BD80B588B000AF786040F2E0536E
:1011E800C2F200031B78002B6AD04FF00003FB61AA
:1011F8004FF00003BB614FF000037B614FF0000329
:10120800FB74FB7C03F10103FB7407F108034FF047
:1012180053004FF032014FF0080201F097FA3B7A81
:101228001A467B7A4FEA03239BB2D3189BB29BB230
:101238001BB2FA69D318FB61BB7A1A46FB7A4FEAEC
:1012480003239BB2D3189BB29BB21BB2BA69D318C3
:10125800BB613B7B1A467B7B4FEA03239BB2D318C7
:101268009BB29BB21BB27A69D3187B61FB7B03F0FC
:101278007F03BB74FB7C1F2B02D8BB7C002BC0D127
:10128800FB7CFA6992FBF3F39AB27B681A807B685D
:1012980003F10203FA7CB96991FBF2F292B21A8067
:1012A8007B6803F10403FA7C796991FBF2F292B24C
:1012B8001A8040F2E153C2F20003FA7C1A702EE061
:1012C80007F108034FF053004FF032014FF00602C8
:1012D80001F03CFA3B7A1A467B7A4FEA03239BB229
:1012E800D3189BB29AB27B681A807B6803F1020319
:1012F800BA7A1146FA7A4FEA022292B28A1892B260
:1013080092B21A807B6803F104033A7B11467A7B18
:101318004FEA022292B28A1892B292B21A8007F168
:101328002007BD4680BD00BF80B584B000AF78609F
:101338000B467B804FF0190009F06CF84FF06800FD
:101348004FF015014FF0000201F0E0F80346FB737F
:10135800FB7B83F00103DBB2002B02D04FF00003CC
:1013680058E07A6841F22943C0F6000313607A68AE
:1013780041F2B543C0F6000353607A6841F249531D
:10138800C0F6000393607B6844F21842C3F29212DD
:10139800DA607B88622B1BD0622B04DC0A2B2FD0EF
:1013A800142B25D01CE0BC2B0AD0B3F5807F17D1B5
:1013B80040F20003C2F200034FF000021A7027E067
:1013C80040F20003C2F200034FF001021A701FE05E
:1013D80040F20003C2F200034FF002021A7017E055
:1013E80040F20003C2F200034FF003021A700FE04C
:1013F80040F20003C2F200034FF004021A7007E043
:1014080040F20003C2F200034FF005021A7000BF59
:101418004FF00103184607F11007BD4680BD00BF15
:1014280080B582B000AF4FF0190008F0F3FF4FF01D
:1014380068004FF015014FF0000201F067F803460D
:10144800FB71FB7983F00103DBB2002B03D04FF073
:10145800030008F0F9FF40F20003C2F200031B7812
:1014680043F01803DBB24FF068004FF016011A463C
:1014780001F04CF84FF068004FF017014FF00002F0
:1014880001F044F84FF068004FF03D014FF00102C1
:1014980001F03CF84FF068004FF03E014FF00102B8
:1014A80001F034F807F10807BD4680BD80B584B067
:1014B80000AF786007F108034FF068004FF01D0196
:1014C8004FF0060201F042F93B7A4FEA03239AB241
:1014D8007B7A13439BB21BB2002B01DA03F103039F
:1014E8004FEAA3039AB27B681A807B6803F1020271
:1014F800BB7A4FEA032399B2FB7A0B439BB21BB228
:10150800002B01DA03F103034FEAA3039BB2138014
:101518007B6803F104023B7B4FEA032399B27B7B90
:101528000B439BB21BB2002B01DA03F103034FEA12
:10153800A3039BB2138007F11007BD4680BD00BF0F
:1015480080B584B000AF786007F10C034FF06800F5
:101558004FF01B014FF0020201F0F8F83B7B4FEA15
:1015680003227B7B134303F54E5303F110034AF226
:10157800EB02CEF60E2282FB0312D2184FEA222289
:101588004FEAE373D31A9BB203F123039BB29AB2D7
:101598007B681A8007F11007BD4680BD80B588B00A
:1015A80000AFF860B9601346FB804FF0230008F0E5
:1015B80031FF07F11D034FF068004FF075014FF040
:1015C800010201F0C3F80346FB77FB7F83F00103B8
:1015D800DBB2002B02D04FF00003E3E07B7F682BE7
:1015E80002D04FF00003DDE007F114034FF068006C
:1015F8004FF006014FF0060201F0A8F87B7E03F0D9
:1016080001034FEA8303DAB2FB7D03F001034FEADB
:101618004303DBB21343DAB27B7DDBB203F0010391
:10162800DBB21343DBB2BB77BB7F002B1AD0BB7F87
:10163800012B07D140F2E253C2F200034FF000023F
:101648001A7037E0BB7F022B07D140F2E253C2F297
:1016580000034FF001021A702CE04FF0050008F06B
:10166800F3FE27E007F11D034FF068004FF00C016F
:101678004FF0010201F06AF87B7F03F00F03BB779C
:10168800BB7F002B04D14FF0050008F0DDFE11E010
:10169800BB7F042B07D140F2E253C2F200034FF0A4
:1016A80000021A7006E040F2E253C2F200034FF063
:1016B80001021A70FA6841F2B973C0F600031360A8
:1016C800FA6841F2F973C0F60003536040F2E2533E
:1016D800C2F200031B78002B02D14FF06F0301E028
:1016E8004FF06E03FA681372BA6841F65D03C0F6EC
:1016F80000031360BA6841F65113C0F60003536043
:10170800BB6844F21942C3F29212DA60FB88142BC8
:101718002ED0142B04DC052B3AD00A2B30D01FE036
:10172800BC2B0DD0B3F5807F02D0622B10D017E010
:1017380040F20103C2F200034FF000021A702FE0DA
:1017480040F20103C2F200034FF001021A7027E0D1
:1017580040F20103C2F200034FF002021A701FE0C8
:1017680040F20103C2F200034FF003021A7017E0BF
:1017780040F20103C2F200034FF004021A700FE0B6
:1017880040F20103C2F200034FF005021A7007E0AD
:1017980040F20103C2F200034FF006021A7000BFC4
:1017A8004FF00103184607F12007BD4680BD00BF72
:1017B80080B400AF40F2E253C2F200031B78002B62
:1017C80002D0012B08D00FE040F22203C2F200033E
:1017D8004FF400621A8007E040F22203C2F20003CD
:1017E8004FF480521A8000BFBD4680BC704700BFCE
:1017F80080B584B000AF786007F108034FF0680047
:101808004FF03B014FF0060200F0A0FF3B7A4FEA91
:1018180003239AB27B7A13439AB27B681A807B6857
:1018280003F10203BA7A4FEA022291B2FA7A0A4322
:1018380092B21A807B6803F104033A7B4FEA0222D2
:1018480091B27A7B0A4392B21A8007F11007BD461B
:1018580080BD00BF80B582B000AF4FF40053BB809D
:101868004FF00203FB714FF00003BB7140F25413B9
:10187800C2F200031A684FF49053C0F27A039A42F6
:1018880009D107F104034FF48060C4F6000019463B
:1018980001F0B4F913E040F25413C2F200031A68DD
:1018A8004FF4D853C0F2B7039A4208D107F10403A2
:1018B8004FF40060C4F60000194601F09FF94FF09C
:1018C80068004FF06B014FF0800200F01FFE4FF0F0
:1018D800050008F09FFD4FF068004FF019014FF028
:1018E800000200F013FE4FF068004FF06B014FF05C
:1018F800030200F00BFE4FF068004FF037014FF085
:10190800020200F003FE40F20103C2F200031B785A
:101918004FF068004FF01A011A4600F0F7FD4FF03B
:1019280068004FF01B014FF0180200F0EFFD4FF078
:1019380068004FF01C014FF0100200F0E7FD07F1BE
:101948000807BD4680BD00BF80B584B000AF786091
:1019580007F108034FF068004FF043014FF006020B
:1019680000F0F4FE3B7A4FEA03239AB27B7A1343E2
:101978009BB21BB2002B01DA03F103034FEAA30366
:101988009AB27B681A807B6803F10202BB7A4FEA3D
:10199800032399B2FB7A0B439BB21BB2002B01DAEB
:1019A80003F103034FEAA3039BB213807B6803F19F
:1019B80004023B7B4FEA032399B27B7B0B439BB228
:1019C8001BB2002B01DA03F103034FEAA3039BB216
:1019D800138007F11007BD4680BD00BF80B584B0F5
:1019E80000AF78600B467B804FF0190008F012FDBD
:1019F80007F10F034FF068004FF00F014FF001029D
:101A080000F0A4FEFB7BD32B02D04FF000033AE09A
:101A18007A6841F69923C0F6000313607A6841F6A4
:101A2800FD23C0F6000353607B684EF6DD12C3F257
:101A3800A712DA607B884E2B13D05D2B19D0362B7A
:101A480007D040F2E353C2F200034FF000021A70CD
:101A580017E040F2E353C2F200034FF040021A705D
:101A68000FE040F2E353C2F200034FF080021A7015
:101A780007E040F2E353C2F200034FF0C0021A70CD
:101A880000BF4FF00103184607F11007BD4680BD9F
:101A980080B582B000AF4FF0640008F0BBFC4FF097
:101AA80068004FF023014FF0F00200F02FFD0346CD
:101AB800FB71FB7983F00103DBB2002B03D04FF0FD
:101AC800030008F0C1FC4FF0050008F0A3FC40F249
:101AD800E353C2F200031B7843F00F03DBB24FF06D
:101AE80068004FF020011A4600F010FD07F10807C2
:101AF800BD4680BD80B584B000AF786007F10803AB
:101B08004FF068004FF0A8014FF0060200F01EFEEB
:101B18003B7A4FEA03239AB27B7A13439BB21BB2F8
:101B2800002B01DA03F103034FEAA3039AB27B689F
:101B38001A807B6803F10202BB7A4FEA032399B249
:101B4800FB7A0B439BB21BB2002B01DA03F10303B0
:101B58004FEAA3039BB213807B6803F104023B7B2B
:101B68004FEA032399B27B7B0B439BB21BB2002B3A
:101B780001DA03F103034FEAA3039BB2138007F1D1
:101B88001007BD4680BD00BF80B483B000AF786049
:101B98007A684FF44053C4F201039A4214D140F2D8
:101BA800E453C2F200031B889BB203F101039AB20B
:101BB80040F2E453C2F200031A8040F2E453C2F246
:101BC80000031B889BB22FE07A684FF46053C4F27D
:101BD80000039A4214D140F2E653C2F200031B8874
:101BE8009BB203F101039AB240F2E653C2F200033A
:101BF8001A8040F2E653C2F200031B889BB213E03E
:101C080040F2E853C2F200031B889BB203F10103C0
:101C18009AB240F2E853C2F200031A8040F2E85345
:101C2800C2F200031B889BB2184607F10C07BD4699
:101C380080BC704780B58AB000AF78604FF48050A0
:101C48004FF0010114F072FF4FF400304FF0010122
:101C580014F042FF4FF090404FF005014FF005029D
:101C680014F03CFA4FF090404FF006014FF0050297
:101C780014F034FA4FF090404FF007014FF005028E
:101C880014F02CFA4FF0E0033B624FF0020387F8A0
:101C980024304FF0030387F825304FF0000387F80E
:101CA80026304FF0000387F8273007F120034FF064
:101CB8009040194614F02AF94FF400104FF0010132
:101CC80014F00AFF4FF008033B624FF0010387F856
:101CD80024304FF0030387F825304FF0000387F8CE
:101CE80026304FF0000387F8273007F120034FF420
:101CF8008050C4F60000194614F008F94FF48050DB
:101D0800C4F600004FF0080114F0CCF94FF440502D
:101D1800C4F2010014F0C4FF4FF00003BB814FF47C
:101D28008273FB814FF4E0633B824FF000037B82B8
:101D38004FF00003BB824FF40073FB824FF008039F
:101D48003B834FF000037B834FF00703BB8307F10E
:101D58000C034FF44050C4F20100194614F0E4FF9C
:101D68004FF44050C4F201004FF4805115F088F848
:101D78004FF44050C4F201004FF0010115F060F833
:101D880007F12807BD4680BD80B584B000AF7860F4
:101D98000B46FB704FF48053FB8111E0FB89002B4D
:101DA80014BF00230123DBB2FA8902F1FF32FA8162
:101DB800002B05D07868FFF7E7FE0346DBB22EE07C
:101DC80078684FF0020115F0C1F80346002BE5D002
:101DD800FB787868194615F06FF84FF48053FB814B
:101DE80011E0FB89002B14BF00230123DBB2FA8921
:101DF80002F1FF32FA81002B05D07868FFF7C4FEA4
:101E08000346DBB20BE078684FF0010115F09EF84D
:101E18000346002BE5D0786815F074F80346184699
:101E280007F11007BD4680BD80B500AF4FF44050A4
:101E3800C4F20100FFF7FEFE4FF48050C4F6000024
:101E48004FF0080114F03CF94FF44050C4F201007F
:101E58004FF02401FFF798FF4FF44050C4F20100FF
:101E68004FF08001FFF790FF4FF48050C4F6000058
:101E78004FF0080114F016F94FF0640008F0B6FAB4
:101E88004FF48050C4F600004FF0080114F018F920
:101E98004FF44050C4F201004FF02001FFF774FFE7
:101EA8004FF44050C4F201004FF0AF01FFF76CFF50
:101EB8004FF48050C4F600004FF0080114F0F2F817
:101EC8004FF0010008F092FA4FF48050C4F6000079
:101ED8004FF0080114F0F4F84FF44050C4F2010038
:101EE8004FF02301FFF750FF4FF44050C4F20100B8
:101EF8004FF05001FFF748FF4FF48050C4F6000040
:101F08004FF0080114F0CEF84FF0640008F082FAA0
:101F180080BD00BF90B585B000AF78604FF48050A9
:101F2800C4F600004FF0080114F0CAF84FF440500E
:101F3800C4F201004FF0E801FFF726FF4FF000035D
:101F4800FB7313E0FC7B4FF44050C4F201004FF0E8
:101F58000001FFF719FF03461A4607F110010B1994
:101F680003F8082CFB7B03F10103FB73FB7B052BB8
:101F7800E8D94FF48050C4F600004FF0080114F07F
:101F880091F83B7A4FEA03239AB27B7A13439BB2C8
:101F98001BB2002B01DA03F107034FEAE3039AB2FD
:101FA8007B681A807B6803F10202BB7A4FEA03233D
:101FB80099B2FB7A0B439BB21BB2002B01DA03F1F7
:101FC80007034FEAE3039BB213807B6803F1040223
:101FD8003B7B4FEA032399B27B7B0B439BB21BB23B
:101FE800002B01DA03F107034FEAE3039BB21380E6
:101FF8007B7A4FEA03239AB23B7A13439AB241F6AB
:10200800F043C2F200031A80FB7A4FEA03239AB224
:10201800BB7A13439AB241F6F043C2F200035A80E6
:102028007B7B4FEA03239AB23B7B13439AB241F678
:10203800F043C2F200039A8007F11407BD4690BD31
:1020480080B483B000AF78600B467B807A6841F635
:102058003163C0F6000313607A6841F61D73C0F659
:10206800000353607B6842F21F22C3F6A012DA60B5
:102078007B6844F21942C3F29212DA604FF001030E
:10208800184607F10C07BD4680BC704780B500AF05
:102098004FF032004FF024014FF0800200F036FA82
:1020A8004FF0640008F0B6F94FF032004FF020010D
:1020B8004FF0970200F02AFA4FF00A0008F0AAF948
:1020C8004FF032004FF023014FF0100200F01EFADB
:1020D8004FF0640008F09EF940F22203C2F20003B8
:1020E8004FF480521A8080BD80B584B000AF78600C
:1020F80007F108034FF032004FF028014FF00602B5
:1021080000F024FB0346FB73FB7B83F00103DBB287
:10211800002B33D17B7A4FEA03239AB23B7A1343DD
:102128009BB21BB24FEAD372D3184FEA63039AB239
:102138007B681A807B6803F10202FB7A4FEA03236B
:1021480099B2BB7A0B439BB21BB24FEAD371CB183F
:102158004FEA63039BB213807B6803F104027B7B25
:102168004FEA032399B23B7B0B439BB21BB24FEA66
:10217800D371CB184FEA63039BB2138007F11007A2
:10218800BD4680BD80B584B000AF786007F10E030E
:102198004FF032004FF027014FF0010200F0D6FA5D
:1021A8000346FB73FB7B83F00103DBB2002B02D0F9
:1021B8004FF000030DE07A6842F29503C0F6000381
:1021C80013607A6842F2F103C0F6000353604FF0DF
:1021D8000103184607F11007BD4680BD80B483B0DF
:1021E80000AF786007F10C07BD4680BC704700BFA0
:1021F80080B483B000AF0346FB71FB7940F2EC5228
:10220800C2F200024FEA4303D3185B781A4640F241
:10221800F453C2F2000333F812309BB2184607F1A8
:102228000C07BD4680BC704780B483B000AF7860AF
:102238007A684FF4A843C4F200039A420ED140F2E0
:102248000063C2F200031B889BB203F101039AB238
:1022580040F20063C2F200031A800DE040F202630C
:10226800C2F200031B889BB203F101039AB240F249
:102278000263C2F200031A804FF00003184607F108
:102288000C07BD4680BC704780B58CB000AF786045
:102298007A684FF4A843C4F200039A4240F0898058
:1022A8004FF480204FF0010114F016FC4FF4001099
:1022B8004FF0010114F064FC4FF480204FF001014D
:1022C80014F00AFC4FF0100014F0BAFB4FF48060D1
:1022D800C4F600004FF006014FF0040213F0FEFEB2
:1022E8004FF48060C4F600004FF007014FF004027D
:1022F80013F0F4FE07F12803184613F0B5FE07F1B2
:102308000C03184615F0F2FF4FF0020387F82C3043
:102318004FF0030387F82D304FF0010387F82E3074
:102328004FF0000387F82F304FF04003BB6207F1EE
:1023380028034FF48060C4F60000194613F0E6FD48
:102348004FF08003BB6207F128034FF48060C4F6A6
:102358000000194613F0DAFD07F10C03184615F0D2
:10236800C5FF4FF00003BB614FF000033B614FF026
:1023780000037B614FF00003FB614FF000033B62F9
:102388004FF000037B6242F27A53C0F2E003FB6035
:1023980007F10C034FF4A840C4F20000194615F0E9
:1023A8003DFF4FF4A840C4F200004FF0010115F0C2
:1023B800C3FF7A684FF4B043C4F200039A4240F076
:1023C80087804FF480204FF0010114F085FB4FF413
:1023D80080004FF0010114F0D3FB4FF484004FF05C
:1023E800010114F079FB4FF02000C1F2000014F055
:1023F80027FB4FF4A050C4F600004FF006014FF041
:10240800040213F06BFE4FF090404FF00A014FF0BA
:10241800040213F063FE07F12803184613F024FEA4
:1024280007F10C03184615F061FF4FF0020387F817
:102438002C304FF0030387F82D304FF0010387F855
:102448002E304FF0000387F82F304FF04003BB6267
:1024580007F128034FF4A050C4F60000194613F002
:1024680055FD4FF48063BB6207F128034FF090409D
:10247800194613F04BFD07F10C03184615F036FF0B
:102488004FF00003BB614FF000033B614FF00003C6
:102498007B614FF00003FB614FF000033B624FF09C
:1024A80000037B6242F27A53C0F2E003FB6007F15B
:1024B8000C034FF4B040C4F20000194615F0AEFE0C
:1024C8004FF4B040C4F200004FF0010115F034FFA2
:1024D80007F13007BD4680BD80B582B000AF786097
:1024E8004FF4A840C4F20000FFF7CEFE07F108073A
:1024F800BD4680BD80B400AF40F20063C2F2000365
:102508001B889BB21846BD4680BC704780B586B014
:1025180002AF13460246FA710A46BA717B714FF44C
:10252800A843C4F20003FB6040F2FC53C2F200036C
:102538004FF420421A601CE040F2FC53C2F2000340
:102548001B68002B14BF00220122D2B203F1FF3115
:1025580040F2FC53C2F200031960002A09D0F8685F
:10256800FFF762FE0346002B0CBF00230123DBB2FA
:10257800E6E0F8684FF4004115F046FF0346002BEB
:10258800DAD1FB799BB24FF400520092F8681946F1
:102598004FF001024FF0807315F0EAFE40F2FC5351
:1025A800C2F200034FF420421A601CE040F2FC53D0
:1025B800C2F200031B68002B14BF00220122D2B212
:1025C80003F1FF3140F2FC53C2F200031960002A04
:1025D80009D0F868FFF728FE0346002B0CBF00233C
:1025E8000123DBB2ACE0F8684FF0020115F00CFFF4
:1025F8000346002BDAD0BB79F868194615F0E8FED7
:1026080040F2FC53C2F200034FF420421A601CE06F
:1026180040F2FC53C2F200031B68002B14BF0022D7
:102628000122D2B203F1FF3140F2FC53C2F200039F
:102638001960002A09D0F868FFF7F6FD0346002B59
:102648000CBF00230123DBB27AE0F8684FF0800169
:1026580015F0DAFE0346002BDAD0FB799BB24FF077
:1026680000020092F86819464FF001024FF000731B
:1026780015F07EFE40F2FC53C2F200034FF42042F4
:102688001A601CE040F2FC53C2F200031B68002BE6
:1026980014BF00220122D2B203F1FF3140F2FC53F1
:1026A800C2F200031960002A09D0F868FFF7BCFDE0
:1026B8000346002B0CBF00230123DBB240E0F8687F
:1026C8004FF0020115F0A0FE0346002BDAD07B790B
:1026D800F868194615F07CFE40F2FC53C2F200037C
:1026E8004FF420421A601CE040F2FC53C2F200038F
:1026F8001B68002B14BF00220122D2B203F1FF3164
:1027080040F2FC53C2F200031960002A09D0F868AD
:10271800FFF78AFD0346002B0CBF00230123DBB221
:102728000EE0F8684FF0200115F06EFE0346002B0E
:10273800DAD0F8684FF0200115F08AFE4FF0010357
:10274800184607F11007BD4680BD00BF80B586B0AA
:1027580002AF3B600346FB710B46BB7113467B71AE
:102768004FF4A843C4F20003FB6040F2FC53C2F2EA
:1027780000034FF420421A601CE040F2FC53C2F2FE
:1027880000031B68002B14BF00220122D2B203F100
:10279800FF3140F2FC53C2F200031960002A09D04D
:1027A800F868FFF741FD0346002B0CBF0023012307
:1027B800DBB2FBE0F8684FF4004115F025FE034654
:1027C800002BDAD1FB799BB24FF400520092F868E3
:1027D80019464FF001024FF0000315F0C9FD40F211
:1027E800FC53C2F200034FF420421A601CE040F28E
:1027F800FC53C2F200031B68002B14BF0022012205
:10280800D2B203F1FF3140F2FC53C2F20003196067
:10281800002A09D0F868FFF707FD0346002B0CBF14
:1028280000230123DBB2C1E0F8684FF0020115F084
:10283800EBFD0346002BDAD07B79012B03D9BB795A
:1028480063F07F03BB71BB79F868194615F0C0FDCA
:1028580040F2FC53C2F200034FF420421A601CE01D
:1028680040F2FC53C2F200031B68002B14BF002285
:102878000122D2B203F1FF3140F2FC53C2F200034D
:102888001960002A09D0F868FFF7CEFC0346002B30
:102898000CBF00230123DBB288E0F8684FF0400149
:1028A80015F0B2FD0346002BDAD0FB799AB27B799A
:1028B8004FF410510091F86811461A464FF0007312
:1028C80015F056FD3BE040F2FC53C2F200034FF412
:1028D80020421A601CE040F2FC53C2F200031B685D
:1028E800002B14BF00220122D2B203F1FF3140F2C3
:1028F800FC53C2F200031960002A09D0F868FFF7F8
:1029080093FC0346002B0CBF00230123DBB24DE0F0
:10291800F8684FF0040115F077FD0346002BDAD074
:10292800F86815F063FD03461A463B681A703B6861
:1029380003F101033B607B7903F1FF337B717B7902
:10294800002BC0D140F2FC53C2F200034FF42042E6
:102958001A601CE040F2FC53C2F200031B68002B13
:1029680014BF00220122D2B203F1FF3140F2FC531E
:10297800C2F200031960002A09D0F868FFF754FC76
:102988000346002B0CBF00230123DBB20EE0F868DE
:102998004FF0200115F038FD0346002BDAD0F86817
:1029A8004FF0200115F054FD4FF00103184607F1D0
:1029B8001007BD4680BD00BF80B586B000AF4FF49C
:1029C80080404FF0010114F0DBF84FF480404FF0E5
:1029D800010114F029F94FF00203BB754FF42043AD
:1029E800BB824FF00303FB7507F114034FF48060BB
:1029F800C4F60000194600F001F94FF48043BB8289
:102A08004FF00003BB7507F114034FF48060C4F660
:102A18000000194600F0F2F84FF48053BB824FF0E3
:102A28000103BB7507F114034FF48060C4F600007E
:102A3800194600F0E3F84FF46050C4F2000014F0B7
:102A48002FF94FF482737B804FF000033B804FF4E3
:102A5800E063BB804FF400737B814FF00003FB8180
:102A68004FF007033B824FF00203FB804FF0010356
:102A78003B814FF01003BB813B464FF46050C4F2DA
:102A88000000194614F050F94FF46050C4F20000E9
:102A98004FF0010114F0D4F900F082F8034618460B
:102AA80007F11807BD4680BD80B483B000AF034668
:102AB800FB71FB79002B07D04FF48063C4F6000349
:102AC8004FF480521A8506E04FF48063C4F6000381
:102AD8004FF480529A6107F10C07BD4680BC7047DD
:102AE80080B586B000AFF860B9607A604FF4605383
:102AF800C4F200039B893FE0BB68002B06D0BB688B
:102B08001B78BA6802F10102BA6001E04FF0FF03D6
:102B1800FB7500BF4FF46050C4F200004FF0020193
:102B280014F014FA0346002BF4D0FB7D9BB24FF44B
:102B38006050C4F20000194614F0D6F900BF4FF4F3
:102B48006050C4F200004FF0010114F0FFF9034691
:102B5800002BF4D04FF46050C4F2000014F0E8F9F0
:102B68000346FB75FB68002B06D0FB68FA7D1A70DC
:102B7800FB6803F10103FB607B68002B0CBF00239B
:102B88000123DBB27A6802F1FF327A60002BB3D1FD
:102B98004FF00103184607F11807BD4680BD00BF76
:102BA80080B582B000AF4FF09F033B714FF0000338
:102BB8007B714FF00003BB714FF00003FB714FF0C6
:102BC8000100FFF771FF3A4607F104031046194662
:102BD8004FF00402FFF784FF4FF00000FFF764FF97
:102BE8007B78EF2B02D14FF0010301E04FF0000397
:102BF800184607F10807BD4680BD00BF80B588B0FC
:102C080000AF786039604FF00003FB6143E0FB6977
:102C18004FF0010202FA03F37B613B681B881A46F6
:102C28007B691340002B32D07B69FB603B689B7843
:102C380003F00303DBB23B744FF00103FB763B6800
:102C4800DB78022B07D0032B09D0012B0BD14FF0D7
:102C58000103FB7607E04FF00203FB7603E04FF039
:102C68000303FB7600BFFB7E7B744FF00003BB744D
:102C78003B689B784FEA9303DBB203F00C03DBB2AB
:102C8800FB7407F10C037868194613F03FF9FB69E8
:102C980003F10103FB61FB690F2BB8D907F120078A
:102CA800BD4680BD80B58AB000AF78604FF00003A4
:102CB8007B624FF000033B624FF00003FB614FF073
:102CC8000003BB617B689B79002B02D04FF00203A5
:102CD8007B627B685B78002B03D07B6A03F101037E
:102CE8007B624CF68433C0F601037A6A53F82230CB
:102CF8003B614FF000037B62E2E07B6A3A69D318DC
:102D08001B7803F00F03FB737B6A3A69D3181B78AF
:102D180023F00F03FB757B6A3A69D3181B78FF2BE6
:102D280000F0D3807B68DB78002B0FD0FB7B082B6F
:102D380000F0BF80FB7B092B00F0BB80FB7B0A2BDC
:102D480000F0B780FB7B0B2B00F0B3807B68DB794E
:102D5800002B05D07B68DB79FA7B9A4200F0AB80C8
:102D6800FB7D03F03003002B09D07B681B7883F0D0
:102D78000103DBB2002B02D04FF00003FB757B6828
:102D88001B79002B1DD07B689B7983F00103DBB294
:102D9800002B16D07B68DB78002B09D0FB7B042B3B
:102DA80002D0FB7B052B0CD14FF08003FB7508E0AC
:102DB800FB7B082B02D0FB7B092B02D14FF0800351
:102DC800FB757B685B79002B0FD07B689B7983F060
:102DD8000103DBB2002B08D0FB7B032B05D9FB7B5F
:102DE800072B02D84FF08003FB75FB7D03F010031F
:102DF800002B04D0FB7B184600F042FC5CE0FB7D16
:102E080003F02003002B0BD03B6ADBB2FA7B1046A1
:102E1800194600F0E5FB3B6A03F101033B624BE016
:102E2800FB7D03F04003002B2AD07B681B89B3F598
:102E3800FA7F10D9FB7B4FEA03124CF6C433C0F675
:102E48000103D018BB69D9B27B681A897B689B8952
:102E580000F0EEF90FE0FB7B4FEA03124CF6C433A7
:102E6800C0F60103D018BB69D9B27B681A897B68A0
:102E78009B8900F00DFABB6903F10103BB611BE0FC
:102E8800FB7D5BB2002B17DAFB7B4FEA03124CF693
:102E9800C433C0F60103D018FB69D9B27B685A89DC
:102EA8007B68DB8900F024FAFB6903F10103FB610D
:102EB80002E000BF00E000BF7B6A03F101037B6210
:102EC8007B6A0D2B7FF719AF00E000BF07F12807D9
:102ED800BD4680BD80B588B000AF786013460A460D
:102EE800FA703B8007F10C03184614F033FB4FF0DF
:102EF8007003FB604FF001033B824FF000037B82BD
:102F08003B887B614FF002033B834FF48073BB83A4
:102F1800FB780C2B4CD801A252F823F0592F00084B
:102F2800B92F0008B92F0008B92F0008712F000821
:102F3800B92F0008B92F0008B92F0008892F0008F9
:102F4800B92F0008B92F0008B92F0008A12F0008D1
:102F580007F10C037868194614F0EAF878684FF01E
:102F6800080114F021FB23E007F10C0378681946E7
:102F780014F072F978684FF0080114F031FB17E08B
:102F880007F10C037868194614F0F2F978684FF0E5
:102F9800080114F043FB0BE007F10C0378681946AD
:102FA80014F06EFA78684FF0080114F053FB00BF74
:102FB80007F12007BD4680BD80B586B000AFF86038
:102FC800B9601346FB71BB689BB2BB82FB79BB75CA
:102FD8004FF00203FB7507F11403F8681946FFF771
:102FE8000DFE07F11807BD4680BD00BF80B586B04D
:102FF80000AFF860F9723A81FB8040F25463C2F284
:10300800000319780A4613464FEA43039B184FEA10
:10301800830341F28412C2F200029B187B6101F122
:103028000103DAB240F25463C2F200031A70FB687B
:1030380019683A89FB7A084611461A4601F050FE8B
:10304800FB685A68FB689B68104619464FF00202F5
:10305800FFF7B2FFFB681968FB681A7BFB88084614
:1030680011461A46FFF736FFFB689B7B002B06D0FC
:10307800FB681B6818464FF0010114F011FCFB684F
:103088001B6818464FF0010114F032F8FB681B7BEF
:103098000C2B39D801A252F823F000BFD930000810
:1030A800113100081131000811310008E73000081B
:1030B800113100081131000811310008F5300008FD
:1030C80011310008113100081131000803310008DE
:1030D800FB681B6803F134027B691A6014E0FB6823
:1030E8001B6803F138027B691A600DE0FB681B68F6
:1030F80003F13C027B691A6006E0FB681B6803F178
:1031080040027B691A6000BF7B693A899A807B69B3
:10311800184607F11807BD4680BD00BF80B483B0CC
:1031280000AF02460B46FA71BB80FA7940F204639D
:10313800C2F2000353F822301968BB88A3F57A72EB
:10314800F87940F20463C2F2000353F820309B88F8
:1031580003FB02F244F6D353C1F2620383FB02037A
:103168004FEAA3104FEAE273C31A0B6007F10C078A
:10317800BD4680BC704700BF80B483B000AF024634
:103188000B46FA71BB80FA7940F20463C2F200037D
:1031980053F822301B68BA881A6007F10C07BD463D
:1031A80080BC704780B582B000AF02460B46FA710A
:1031B800BB80FA7940F20463C2F2000353F822306C
:1031C800002B0FD0FB790B2B0CD8FA7940F2046353
:1031D800C2F2000353F822309B68F979BA8808468E
:1031E8001146984707F10807BD4680BD80B483B0F3
:1031F80000AF02460B46FA71BB80FA7940F234639D
:10320800C2F2000353F82230002B0CD0FB79072BB5
:1032180009D8FA7940F23463C2F2000353F8223035
:103228001B68BA881A6007F10C07BD4680BC704756
:1032380090B587B000AFF860F9723A81FB804FF41F
:103248009053C0F27A037B61FC7A3B897A69B2FBBE
:10325800F3F39AB2FB88F8684FF00801FFF7C6FE4F
:10326800024640F20463C2F2000343F82420FA7ACB
:1032780040F20463C2F2000353F8222043F22513FC
:10328800C0F60003936007F11C07BD4690BD00BF60
:1032980090B587B000AFF860F9723A81FB8044F2CC
:1032A8004023C0F20F037B61FC7A3B897A69B2FB49
:1032B800F3F39AB2FB88F8684FF00101FFF796FE26
:1032C800024640F20463C2F2000343F82420FA7A6B
:1032D80040F20463C2F2000353F8222043F2811340
:1032E800C0F60003936007F11C07BD4690BD00BF00
:1032F80090B585B000AFF860F9723A81FB80FC7A2E
:103308003A8944F24023C0F20F0393FBF2F39AB2D6
:10331800FB88F8684FF00101FFF768FE024640F2AB
:103328003463C2F2000343F8242007F11407BD46B2
:1033380090BD00BF80B582B000AF02460B46FA715F
:10334800BB80FB79032B1CD841F21423C2F2000383
:103358001B689B88BA889A4213D9FB794FF00102FF
:1033680002FA03F3DAB240F21173C2F200031B78D7
:10337800DBB21343DBB2DAB240F21173C2F20003DC
:103388001A7040F21173C2F200031B780F2B0ED192
:1033980040F21173C2F200034FF000021A7041F2BA
:1033A8001823C2F200031B681B685B68984707F183
:1033B8000807BD4680BD00BF80B584B000AF034696
:1033C8003960FB7140F20873C2F200031A6840F2D8
:1033D8000C73C2F200031A6040F20873C2F20003D1
:1033E8003A681A6040F20873C2F200031A6840F2A1
:1033F8000C73C2F200031B68D31AFB60FA6840F62C
:103408008C239A4207DD40F21073C2F200034FF09A
:1034180000021A7036E0FA6840F2EE239A4224DD80
:10342800FA6840F6C9039A421FDC40F21073C2F2F0
:1034380000031B78072B18D840F21073C2F2000360
:103448001B781A46FB6899B240F2F863C2F200038F
:1034580023F8121040F21073C2F200031A78FB68C6
:103468009BB210461946FFF765FF40F21073C2F28F
:1034780000031B7803F10103DAB240F21073C2F2C1
:1034880000031A7007F11007BD4680BD80B584B0EF
:1034980000AF03463960FB71FA7913464FEA83039C
:1034A8009B184FEA830340F25862C2F200029B184D
:1034B800FB60FB681B69BB60FB689B78002B11D124
:1034C800FB683A685A60FB684FF001029A70BB6863
:1034D8001A68BB681B7B104619464FF0020200F0C1
:1034E80059F838E0FB683A689A60FB689A68FB68A4
:1034F8005B68D21AFB68DA60FB68DA6840F2EE2390
:103508009A421AD9FB68DA6840F6C9039A4214D875
:10351800FB685B781A46FB68DB6899B240F2F8638F
:10352800C2F2000323F81210FB685A78FB68DB68C4
:103538009BB210461946FFF7FDFEFB684FF00002EC
:103548009A70BB681A68BB681B7B104619464FF017
:10355800000200F01FF807F11007BD4680BD00BF4C
:1035680080B586B000AFF860B9601346FB71BB68E0
:103578009BB2BB82FB79BB754FF00203FB7507F169
:103588001403F8681946FFF739FB07F11807BD4619
:1035980080BD00BF80B586B000AF786013460A468C
:1035A800FA703B8007F10C03184614F0C5F8FB7855
:1035B8009BB2BB813B88FB814FF001033B824FF0FC
:1035C80000037B824FF00003BB8207F10C0378688D
:1035D800194614F05DF807F11807BD4680BD00BF15
:1035E80080B584B000AF02460B46FA71BB71BA7958
:1035F80013464FEA83039B184FEA830340F258624D
:10360800C2F200029B18FB60FB794FEA03124CF6EA
:10361800C433C0F60103D318BB60FB68BA795A708B
:10362800FB684FF001021A70FB68BA681A61BB6840
:103638005968BB689A68BB68DB7B084611461A461E
:10364800FFF78EFFBB681A68BB681B7B10461946DC
:103658004FF00002FFF79EFFB8684FF6FF714FF07A
:10366800010201F071FBBB79B868194643F2954233
:10367800C0F6000201F0FCFA07F11007BD4680BD54
:1036880080B584B000AF0346FB7140F25863C2F2C4
:103698000003FB60FB794FEA03124CF6C433C0F613
:1036A8000103D318BB60FB684FF000021A70FB6877
:1036B800BA681A61BB685968BB689A68BB68DB7BE3
:1036C800084611461A46FFF74BFFBB681A68BB68E5
:1036D8001B7B104619464FF00002FFF75BFFB868E6
:1036E8004FF6FF714FF0010201F02EFBB8684FF062
:1036F800000143F2C132C0F6000201F0B9FA07F145
:103708001007BD4680BD00BF80B483B000AF03463C
:10371800FB71FA7940F2F863C2F2000333F8123011
:10372800184607F10C07BD4680BC704780B483B0CB
:1037380000AF7860396041F21823C2F200037A685A
:103748001A6041F21423C2F200033A681A6007F1C2
:103758000C07BD4680BC704780B596B000AFF860D6
:10376800B9607A60FB704FF000037B65FA684FF42C
:103778006053C4F201039A4206D1FB78786819466F
:1037880000F07CFA78650FE0FA684FF48843C4F2D9
:1037980000039A4206D1FB787868194600F008FBC6
:1037A800786501E07B6D26E17B6D4FF000021A62BF
:1037B8007B6D1A6A7B6DDA617B6D4FF000029A624D
:1037C8007B6D9A6A7B6D5A627B6DBA68DA627B6D33
:1037D800FA781A717B6D7A689A607B683B614FF062
:1037E80000037B61FB7803F00403002B06D04FF441
:1037F8000053BB614FF48063FB6105E04FF00003A9
:10380800BB614FF00003FB614FF000037B624FF098
:1038180000033B62FB7803F00103002B03D03B6AF3
:1038280043F004033B62FB7803F00203002B03D050
:103838003B6A43F008033B627B6D1A6D07F1100386
:103848001046194614F03EFA07F12803184614F0FA
:103858005DFF7B6DDB6CBB624FF48053FB644FF004
:1038680000033B654FF00003BB634FF000033B646C
:103878004FF08003FB634FF000037B64FB7803F099
:103888000103002B4BD07B6D1B6B002B33D07B6D62
:10389800DB689BB2BB864FF000033B634FF020030D
:1038A800BB647B6D5B69FB627B6D1B6B184614F018
:1038B800DDFD7B6D1A6B07F128031046194614F0DD
:1038C800E5FE7B6D1B6B18464FF0010114F054FFA9
:1038D8007B6D1B6D18464FF040014FF0010214F04C
:1038E800D5FA7B6D1B6B184614F070FF03461A4619
:1038F8007B6D1A6413E07B6D1B6D184640F2051151
:10390800C0F2050114F02AFB7B6D1B6D184640F2CE
:103918000511C0F205014FF0010214F0D5FA07F1C4
:103928002803184614F0F2FE7B6D9B6CBB624FF4C3
:103938008053FB644FF000033B654FF00003BB630B
:103948004FF000033B644FF08003FB634FF000032C
:103958007B64FB7803F00203002B44D07B6D5B6B28
:10396800002B35D07B6D1B699BB2BB864FF01003D3
:103978003B634FF00003BB647B6D5B6B184614F030
:1039880075FD7B6D5A6B07F128031046194614F034
:103998007DFE7B6D5B6B18464FF002014FF0010214
:1039A80014F022FF7B6D5B6B18464FF0000114F09A
:1039B800FFFE7B6D5B6B4FF000025A607B6D1B6DE9
:1039C80018464FF080014FF0010214F05FFA0AE048
:1039D8007B6D1B6D184640F20711C0F207014FF0CE
:1039E800010214F071FA7B6D1B6D18464FF001014E
:1039F80014F030FA7B6D184607F15807BD4680BDB4
:103A080080B58AB000AF786039607B687B623B68BC
:103A1800FB604FF000033B614FF000037B614FF008
:103A28000003BB614FF000033B624FF00003FB61F2
:103A38007B6A1B7903F00103002B03D0FB6943F079
:103A48000403FB617B6A1B7903F00203002B03D09C
:103A5800FB6943F00803FB617B6A1A6D07F10C03ED
:103A68001046194614F02EF97B6A3A689A6007F1F5
:103A78002807BD4680BD00BF80B483B000AF786022
:103A88000B46FB7007F10C07BD4680BC704700BFB2
:103A980080B582B000AF78607B685B6B7A689169AB
:103AA8007A68926A8A18DA607B685A6A7B689B6AC5
:103AB8009A420CD97B685B6B7A68516A7A68926A19
:103AC8008A1A5A607B685A6A7B689A620BE07B683C
:103AD8005B6B7A6811697A68926A8A1A5A607B689D
:103AE8004FF000029A627B684FF0000283F844208E
:103AF8007B685B6B18464FF0010114F03DFE07F13F
:103B08000807BD4680BD00BF80B485B000AF7860AF
:103B18007B68FB60FB681B6B002B0AD0FB681B6B88
:103B28005A68FB681B6C9A420CBF00230123DBB266
:103B380008E0FB681A6AFB68DB699A420CBF00233D
:103B48000123DBB2184607F11407BD4680BC704755
:103B580080B485B000AF78607B68FB60FB685B6B06
:103B6800002B03D0FB6893F8443008E0FB689A6A9E
:103B7800FB685B6A9A4214BF00230123DBB2184634
:103B880007F11407BD4680BC704700BF80B485B0FC
:103B980000AF78607B68BB60BB681B6B002B18D0DC
:103BA800BB685A69BB68D968BB681B6CCB1AD31849
:103BB8001B78FB73BB681B6C03F1FF32BB681A648C
:103BC800BB681B6C002B18D1BB68DA68BB681A6429
:103BD80013E0BB685A69BB681B6AD3181B78FB7370
:103BE800BB681B6A03F10103BA68D268B3FBF2F140
:103BF80002FB01F29A1ABB681A62FB7B184607F1AE
:103C08001407BD4680BC704780B584B000AF7860AB
:103C18000B46FB707B68FB60FB689A69FB685B6A14
:103C2800D318FA781A70FB685B6A03F10103FA6823
:103C38001269B3FBF2F102FB01F29A1AFB685A62AD
:103C4800FB685B6B002B0AD0FB685B6B1B6803F09F
:103C58000103002B0ED1F868FFF71AFF0AE0FB6892
:103C68001B6D184640F20711C0F207014FF0010220
:103C780014F02AF907F11007BD4680BD80B586B05B
:103C880000AF78600B46FB7040F21473C2F2000379
:103C98007B617A694CF69433C0F6010313607B6943
:103CA8007A689A607A6940F67C03C2F2000353612D
:103CB8007A6940F67C13C2F2000393617B694FF482
:103CC8008072DA607B694FF480721A617A694FF00A
:103CD8005803C4F2020313637A694FF04403C4F231
:103CE800020353637A694FF46053C4F20103136506
:103CF8007B691B6D03F124031A467B69DA647B69CF
:103D08001B6D03F128031A467B699A644FF002037E
:103D18003B734FF003037B734FF00003BB734FF00B
:103D28000103FB73FB7803F00203002B11D04FF45F
:103D38000073BB604FF090404FF009014FF007024D
:103D480012F0CCF907F108034FF09040194612F031
:103D5800DDF8FB7803F00103002B11D04FF48063EA
:103D6800BB604FF090404FF00A014FF0070212F08D
:103D7800B5F907F108034FF09040194612F0C6F85C
:103D88004FF00E033B744FF001037B744FF00103B7
:103D9800BB744FF00103FB7407F11003184613F0CE
:103DA8001DFF7B69184607F11807BD4680BD00BF97
:103DB80080B586B000AF78600B46FB7040F2687340
:103DC800C2F200037B617A694CF69433C0F60103B2
:103DD80013607B697A689A607B694FF08002DA60C9
:103DE8007B694FF040021A617A6940F2BC73C2F2F3
:103DF800000353617A6940F63C03C2F20003936101
:103E08007A694FF08003C4F2020353637A694FF46E
:103E18008843C4F2000313657B691B6D03F1240317
:103E28001A467B69DA647B691B6D03F128031A461D
:103E38007B699A644FF002033B734FF003037B7373
:103E48004FF00003BB734FF00103FB73FB7803F0E3
:103E58000203002B15D04FF02003BB604FF44060E5
:103E6800C4F600004FF005014FF0070212F036F9D2
:103E780007F108034FF44060C4F60000194612F039
:103E880045F8FB7803F00103002B15D04FF04003F1
:103E9800BB604FF44060C4F600004FF006014FF0DD
:103EA800070212F01BF907F108034FF44060C4F64B
:103EB8000000194612F02AF84FF011033B744FF036
:103EC80001037B744FF00003BB744FF00103FB74D4
:103ED80007F11003184613F081FE4FF026033B74D8
:103EE8004FF001037B744FF00103BB744FF00103E3
:103EF800FB7407F11003184613F070FE7B6918462F
:103F080007F11807BD4680BD80B582B000AF786064
:103F18007B685B6B18464FF0000114F02DFC7B6842
:103F28005A6A7B689B6A9A4203D07868FFF7B0FDAB
:103F380004E07B684FF0010283F8442007F108078A
:103F4800BD4680BD80B582B000AF40F21473C2F2A6
:103F580000037B604FF4005014F064FC7868FFF7AE
:103F6800D3FF07F10807BD4680BD00BF80B582B00A
:103F780000AF40F26873C2F200037B604FF000703C
:103F880014F050FC4FF08000C4F202004FF0000122
:103F980014F0F2FB7868FFF7B7FF07F10807BD4692
:103FA80080BD00BF80B584B000AF78607B681B6DB2
:103FB800DB69FB60FB6803F02003002B24D07B68DF
:103FC800DB6A002B08D07B68DB6A7A68126D928CFA
:103FD80092B21046984717E07B685A697B68DB699C
:103FE800D3187A68126D928C92B2D2B21A707B682A
:103FF800DB6903F101037A68D268B3FBF2F102FBD3
:1040080001F29A1A7B68DA61FB6803F08003002BDF
:1040180028D07B689A6A7B685B6A9A4217D07B686B
:104028001B6D7A6891697A68926A8A181278D2B296
:104038001A857B689B6A03F101037A681269B3FBEE
:10404800F2F102FB01F29A1A7B689A620AE07B6835
:104058001B6D184640F20711C0F207014FF000022D
:1040680013F032FF07F11007BD4680BD80B582B05E
:1040780000AF40F21473C2F200037B607868FFF768
:1040880091FF07F10807BD4680BD00BF80B582B02B
:1040980000AF40F26873C2F200037B607868FFF7F4
:1040A80081FF07F10807BD4680BD00BF80B483B01B
:1040B80000AF78600B46FB707B6893F84232002BA8
:1040C80006D0FB78002B14BF00230123DBB2FB7062
:1040D800FB78002B09D07B68D3F834315B687A68A9
:1040E800D2F8342192689A6109E07B68D3F83431B8
:1040F8005B687A68D2F83421926892B21A8507F11F
:104108000C07BD4680BC704780B584B000AF7860AE
:1041180013460A467A807B707B88BB817B78BB73A9
:104128004FF00203FB7307F10C0378681946FEF79A
:1041380065FD07F11007BD4680BD00BF80B582B0A0
:1041480000AF78607B685A687B689B689BB21046B2
:1041580019464FF00402FFF7D7FF07F10807BD46DD
:1041680080BD00BF80B483B000AF78607A684FF636
:10417800FF739A4294BF00230123DBB2184607F16C
:104188000C07BD4680BC704780B588B000AFF860AA
:104198000B467A60FB7240F25813C2F200031B68A8
:1041A800FB61FA697B68B2FBF3F3BB61B869FFF79F
:1041B800D9FF0346002B06D0FB69012B03D9FB6905
:1041C8004FEA5303FB61B869FFF7CCFF0346002BA6
:1041D800E7D140F25813C2F200031A684DF6836320
:1041E800C4F21B33A3FB02134FEA9343FB75BB696D
:1041F8009AB2FB7DF86811461A4600F0A5FDFB7AD5
:10420800F868194644F28D72C0F6000200F030FDDD
:1042180007F12007BD4680BD80B586B000AF786045
:1042280013460A46FA703B8007F10C03184613F050
:1042380083FAFB789BB2BB813B88FB814FF001037B
:104248003B824FF000037B824FF00003BB8207F1F3
:104258000C037868194613F01BFA07F11807BD46D6
:1042680080BD00BF80B582B000AF786013460A46B3
:10427800FA70BB707B6819687B681A7BBB78002B67
:1042880002D04FF0000301E04FF002030846114648
:104298001A46FFF7C1FFFB787868194644F2C572E1
:1042A800C0F6000200F0E4FC07F10807BD4680BD37
:1042B80080B582B000AF78607B685A687B689B687D
:1042C8009BB2104619464FF00102FFF71DFF07F198
:1042D8000807BD4680BD00BF80B483B000AF7860DA
:1042E8007B684FF48072DA607B6803F134027B6884
:1042F8005A617B684FF000021A627B684FF0000237
:10430800DA617B6803F59C727B689A617B684FF47D
:1043180080721A617B684FF000029A627B684FF0E6
:1043280000025A6207F10C07BD4680BC704700BF07
:1043380080B584B000AFF8607A600A46FA72BB7242
:10434800FA684CF6AC33C0F601031360FB684FF013
:1043580003021A71F868FFF7BFFFFB684FF000020D
:1043680083F83C22FB684FF0010283F83822FB688F
:104378004FF0000283F83922FB68BA7A83F84222A8
:10438800FB684FF00002A3F84422FB684FF00002DC
:10439800A3F84622FB68D3F834311846FFF788FFA4
:1043A800FB681B6B1846FFF7C9FEF8684FF0010160
:1043B800FFF77CFE4FF0320006F02CF8FB68D3F8CC
:1043C8003421FB7A104619467A68FFF7DDFEFB6850
:1043D800196BFA7ABB7A084611461A46FFF742FF6C
:1043E80007F11007BD4680BD80B584B000AF786086
:1043F8000B46FB704FF00003FB73FB7B4FF412720C
:1044080002FB03F241F21C23C2F20003D318BB6083
:10441800BB680F4A1A63BB680E4AC3F83421FA7B9B
:10442800FB78B86811467A68FFF782FF40F67C236C
:10443800C2F200037A681A6040F67C23C2F20003D5
:104448004FF001021A7107F11007BD4680BD00BF89
:1044580044CC010854CC010880B584B000AF0346B1
:10446800FB714FF00103FB60FB684FF4127202FB13
:1044780003F241F21C23C2F20003D318BB60BB68ED
:104488000A4A1A63BB680A4AC3F83421FB68D9B2DE
:1044980040F67C23C2F200031A68FB79B868FFF77C
:1044A80047FF07F11007BD4680BD00BF64CC010877
:1044B80074CC010880B483B000AF78607B681A6A56
:1044C8007B68DB6803F1FF339A4204D37B684FF0C3
:1044D80000021A6205E07B681B6A03F101027B682F
:1044E8001A6207F10C07BD4680BC704780B584B0DE
:1044F80000AF78607B6893F83C32002B30D1786845
:1045080000F0C4FA0346002B54D17B689A697B6893
:104518009B6AD2181278FA7303F101027B689A62D7
:104528007B689A6A7B681B699A4203D37B684FF061
:1045380000029A62FB7B4FEA43039BB243F4007389
:104548009BB29AB27B68A3F83E227B684FF00A02BE
:1045580083F83D227B684FF0010283F83C222AE071
:104568007B6893F83D32002B1ED07B68B3F83E324F
:10457800DBB203F00103BB737B68B3F83E324FEA4A
:1045880053039AB27B68A3F83E22BB7B786819462E
:10459800FFF78CFD7B6893F83D3203F1FF33DAB205
:1045A8007B6883F83D2206E07B684FF0000283F8C1
:1045B8003C2200E000BF07F11007BD4680BD00BFE8
:1045C80080B485B000AF78607B6893F83B32002BED
:1045D8001ED17B6893F83A32FB7313E07B68B3F81B
:1045E80040329AB2FB7B4FF0010101FA03F39BB210
:1045F80013439BB29AB27B68A3F84022FB7B03F17A
:104608000103FB737B6893F83932FA7B9A42E5D34E
:1046180007F11407BD4680BC704700BF80B582B063
:1046280000AF78607B684FF0000283F839227B681E
:104638004FF0010283F838227B6893F83B32012B54
:1046480019D17B684FF0000283F83B227B681B6B13
:1046580019687B681B6B1A7B7B6893F84232002BC6
:1046680002D04FF0000301E04FF002030846114664
:104678001A46FFF7D1FD07F10807BD4680BD00BF08
:1046880080B584B000AF78607B681B7903F00103C4
:10469800002B37D07B68B3F8403203F40073002B4B
:1046A80014BF00230123DBB2FB737B68B3F84032ED
:1046B80003F00103002B0CBF00230123DBB2BB7303
:1046C800FB7B002B02D0BB7B002B09D17B68B3F8A6
:1046D800463203F101039AB27B68A3F8462212E03E
:1046E8007B68B3F840324FEA53039BB27B737B6815
:1046F8005A697B681B6AD3187A7B1A707868FFF747
:10470800D9FE00E000BF07F11007BD4680BD00BF1D
:1047180080B582B000AF78607B6893F83832002BA0
:104728002BD17B6893F8393203F10103DAB27B6845
:1047380083F839227B6893F83932092B03D17868DA
:10474800FFF73EFF1AE07B6893F839320A2B15D140
:104758007B6893F83B32002B08D17B68B3F8403272
:1047680043F001039AB27B68A3F840227868FFF708
:1047780087FF7868FFF752FF00E000BF07F10807DE
:10478800BD4680BD80B584B000AF03463960FB717B
:10479800FB794FF4127202FB03F241F21C23C2F2BE
:1047A8000003D318FB60F868FFF7A0FEF868FFF76E
:1047B800AFFF07F11007BD4680BD00BF80B584B0CC
:1047C80000AF03463960FB71FB794FF4127202FBAC
:1047D80003F241F21C23C2F20003D318FB60FB680A
:1047E8001B7903F00103002B00F09380FB6893F81A
:1047F8003832002B44D0FB681B6B1B6818464FF0FF
:10480800000112F067FCFB6893F83C32002B08D0DB
:10481800FB68B3F8443203F101039AB2FB68A3F8CA
:104828004422FB681B6B1968FB681B6B1A7BFB68CF
:1048380093F84232002B02D04FF0020301E04FF010
:104848000003084611461A46FFF7E6FCFB684FF0DE
:10485800010283F83B22FB684FF0000283F83922FB
:10486800FB684FF0000283F83A22FB684FF0000221
:10487800A3F84022FB684FF0000283F8382249E091
:10488800FB6893F83B32012B05D1FB6893F839227A
:10489800FB6883F83A22F868FFF792FEFB6893F802
:1048A8003B32002B1AD1FB684FF0010283F83B2200
:1048B800FB681B6B1968FB681B6B1A7BFB6893F81A
:1048C8004232002B02D04FF0020301E04FF0000308
:1048D800084611461A46FFF79FFC1BE0FB684FF09D
:1048E800000283F83B22FB681B6B1968FB681B6B93
:1048F8001A7BFB6893F84232002B02D04FF000037A
:1049080001E04FF00203084611461A46FFF784FCFF
:1049180000E000BF07F11007BD4680BD80B485B038
:1049280000AF78607B681B7903F00103002B02D18C
:104938004FF0000322E07B68BB60BB681A6ABB6863
:10494800DB699A4202D14FF0000317E0BB681A6A8C
:10495800BB68DB699A4206D9BB681A6ABB68DB691F
:10496800D31AFB6008E0BB681A6ABB68DB68D21818
:10497800BB68DB69D31AFB60FB68DBB2184607F13A
:104988001407BD4680BC704780B483B000AF786020
:104998007B68DA697B68DB6803F1FF339A4206D2E9
:1049A8007B68DB6903F101027B68DA6103E07B68FD
:1049B8004FF00002DA6107F10C07BD4680BC704772
:1049C80080B584B000AF78607B681B7903F0010381
:1049D800002B02D14FF0000313E07868FFF79EFF29
:1049E8000346002B02D14FF000030AE07B685A69A6
:1049F8007B68DB69D3181B78FB737868FFF7C4FF03
:104A0800FB7B184607F11007BD4680BD80B483B014
:104A180000AF78600B46FB707B681B7903F00203DC
:104A2800002B14D07B689A697B685B6AD318FA7884
:104A38001A707B685B6A03F101037A681269B3FB39
:104A4800F2F102FB01F29A1A7B685A6200E000BF99
:104A580007F10C07BD4680BC704700BF80B483B027
:104A680000AF7860396007F10C07BD4680BC70471D
:104A780080B483B000AF78600B46FB707B68FA782F
:104A88001A7107F10C07BD4680BC704780B483B02B
:104A980000AF78607B685A6A7B689B6A9A4214BF49
:104AA80000230123DBB2184607F10C07BD4680BC82
:104AB800704700BF80B485B000AF78604FF0000346
:104AC800FB7303E0FB7B03F10103FB73FA7B40F20A
:104AD8000403C2F2000353F822207B689A42F1D102
:104AE800FB7B184607F11407BD4680BC704700BF22
:104AF80080B485B000AF0346FB804FF00003FB7322
:104B080003E0FB7B03F10103FB73FA7B4CF6A44340
:104B1800C0F6010333F81230FA889A42F1D1FB7BD0
:104B2800184607F11407BD4680BC704790B583B09E
:104B380000AF78600B467B807868FFF7BBFF0346C1
:104B48001C467B881846FFF7D3FF03461A464FEAF0
:104B5800C202D31ADBB2E318DBB2184607F10C071E
:104B6800BD4690BD80B586B000AFF8607B600B464F
:104B7800FB721346BB72FB7A9BB2F8681946FFF7C3
:104B8800D5FF0346FB75FB7D1B2B22D8FA7D41F22E
:104B9800AC63C2F200034FEA02129B1803F1080348
:104BA8007A681A60FA7D41F2AC63C2F200034FEAF8
:104BB80002129B18FA7A1A71FA7D41F2AC63C2F2BA
:104BC80000034FEA02129B1803F10803BA7A1A711C
:104BD80000E000BF07F11807BD4680BD80B582B070
:104BE80000AF78600B46FB70FB780C2B3CD801A219
:104BF80052F823F0314C0008714C0008714C000841
:104C0800714C0008414C0008714C0008714C0008B8
:104C1800714C0008514C0008714C0008714C000898
:104C2800714C0008614C000878684FF002014FF0A1
:104C3800010212F053FE17E078684FF004014FF0BC
:104C4800010212F04BFE0FE078684FF008014FF0B8
:104C5800010212F043FE07E078684FF010014FF0B0
:104C6800010212F03BFE00BF07F10807BD4680BDF8
:104C780080B584B000AFF8600B467A60FB72FB68C1
:104C88001968FB681A7BFB7A084611461A467B6846
:104C9800FFF768FFFB681A68FB681B7B104619461C
:104CA800FFF79CFF07F11007BD4680BD80B584B0B3
:104CB80000AF0346FB71FB793B734FF000037B7336
:104CC8004FF00103BB734FF00103FB7307F10C03B3
:104CD800184612F083FF07F11007BD4680BD00BFDC
:104CE80080B586B000AF786013460A467A807B703C
:104CF80007F10C03184612F0CFF97B8803F1FF3354
:104D08003B6140F25813C2F200031A68797844F202
:104D18004023C0F20F0303FB01F3B2FBF3F39BB292
:104D280003F1FF339BB2BB814FF00003BB824FF00E
:104D38000003FB8107F10C037868194612F026F985
:104D480007F11807BD4680BD80B582B000AF786016
:104D580013460A467A807B707B6819687A887B7864
:104D6800084611461A46FFF7BBFF7B681B681846C2
:104D78004FF0010112F0BCF97B685B7B1846FFF726
:104D880095FF07F10807BD4680BD00BF80B584B018
:104D980000AF78600B467B807B8878681946FFF700
:104DA800C5FE0346FB73FB7B4FEA031241F2AC637B
:104DB800C2F20003D318184607F11007BD4680BD9C
:104DC80080B586B000AF78604FF00003FB734FF0FA
:104DD8000003FB7385E0FA7B4CF6A443C0F601039D
:104DE80033F81230BB73BB7B002B17D178684FF0B8
:104DF800020112F093FD0346012B0FD178684FF0A2
:104E0800020112F0BBFD78684FF00001FFF7BEFF0A
:104E18003861786812F0AEFC78614FE0BB7B042BF8
:104E280017D178684FF0040112F078FD0346012B82
:104E38000FD178684FF0040112F0A0FD78684FF0A8
:104E48000401FFF7A3FF3861786812F09FFC7861CE
:104E580034E0BB7B082B17D178684FF0080112F0BB
:104E68005DFD0346012B0FD178684FF0080112F061
:104E780085FD78684FF00801FFF788FF386178688A
:104E880012F090FC786119E0BB7B0C2B22D178687A
:104E98004FF0100112F042FD0346012B1AD1786839
:104EA8004FF0100112F06AFD78684FF00C01FFF71F
:104EB8006DFF3861786812F081FC78613B699B6806
:104EC800002B09D03B699B683A69127B10467969C7
:104ED800984702E000BF00E000BFFB7B03F101033D
:104EE800FB73FB7B032B7FF676AF07F11807BD46F4
:104EF80080BD00BF80B500AF4FF43050C4F2010050
:104F0800FFF75EFF80BD00BF80B500AF4FF0804067
:104F1800FFF756FF80BD00BF80B500AF4FF480603B
:104F2800C4F20000FFF74CFF80BD00BF80B500AFA2
:104F38004FF40060C4F20000FFF742FF80BD00BFDD
:104F480080B500AF4FF45050C4F20100FFF738FFAE
:104F580080BD00BF80B500AF4FF48840C4F20100A7
:104F6800FFF72EFF80BD00BF80B500AF4FF4904023
:104F7800C4F20100FFF724FF80BD00BF80B500AF79
:104F880041F2AC60C2F200004FF000014FF4E07251
:104F980015F0BAFC80BD00BF80B582B000AF786064
:104FA8000B46FB7041F60473C2F200031A68FB78E3
:104FB8001046194604F028FF07F10807BD4680BDD2
:104FC80080B500AF4FF0000044F6A171C0F60001B3
:104FD80001F066FF80BD00BF90B583B000AF034607
:104FE800FB80FB881846FBF7C9FD0346184643F2C9
:104FF8003331C4F25301FBF715FE034618464FF44C
:105008007041C4F27F51FBF7C1FE03461C4640F6CF
:105018008423C2F200031B681B781846FBF7AEFD19
:10502800034620461946FBF7FDFD03461846FBF7E5
:10503800E5FF03469BB2184607F10C07BD4690BD35
:10504800B0B582B000AF4FF00003BB8040F68823B4
:10505800C2F200031C78234603F007054FF0000056
:10506800FDF7C6F803461A4640F68C23C2F2000341
:1050780023F8152004F10103DAB240F68823C2F2BE
:1050880000031A704FF00003FB710DE0FA7940F647
:105098008C23C2F2000333F81220BB88D318BB80DC
:1050A800FB7903F10103FB71FB79072BEED9BB8870
:1050B8004FEAD3039BB21846FFF78EFF0346DAB2D6
:1050C80041F66C03C2F200031A7007F10807BD46E7
:1050D800B0BD00BF80B400AF41F66C03C2F200035C
:1050E8001B781A4641F66E03C2F200031B889A42E7
:1050F8000FD840F68423C2F200031B689A7841F661
:105108006C03C2F200031B789A4202D84FF00103E5
:1051180001E04FF0000303F00103DBB21846BD467F
:1051280080BC704780B584B000AF786040F68423B7
:10513800C2F200037A681A604FF00003BB604FF0B8
:105148000003FB600FE04FF00000FDF751F8034645
:10515800BA68D318BB604FF00A0005F05BF9FB682A
:1051680003F10103FB60FB681F2BECD9BB684FEA16
:1051780053139BB21846FFF72FFF0346BB604FF04F
:105188000103FB600FE040F68423C2F200031B68B2
:105198005B78FA6802FB03F2BB689A4207D8FB689F
:1051A80003F10103FB60FB68052BECD900E000BFAD
:1051B800FB68DAB240F22003C2F200031A7040F62C
:1051C8008423C2F200031B689B78FA6892B202FB40
:1051D80003F39AB241F66E03C2F200031A8007F194
:1051E8001007BD4680BD00BF80B483B000AF7860B3
:1051F8007B681B88002B0AD17B685B88002B06D153
:105208007B689B88002B02D14FF0010301E04FF02F
:10521800000303F00103DBB2184607F10C07BD4693
:1052280080BC704780B590B000AF78607868FFF7B1
:10523800DBFF0346002B40F0C68040F22103C2F298
:1052480000034FF000021A707B681B881BB21846D7
:1052580001F076FCF8637B685B881BB2184601F0A6
:105268006FFCB8637B689B881BB2184601F068FC2A
:105278007863F86B13F0F2FA3863F86B13F062FB9B
:10528800F862B86B13F0EAFAB862B86B13F05AFB1D
:105298007862786B13F0E2FA3862786B13F052FB9D
:1052A800F861386A396BFBF7BDFC0346BB61386AA5
:1052B800B96AFBF7B7FC03467B61F869396BFBF702
:1052C800B1FC03463B61F86A396AFBF7ABFC03465D
:1052D800FB60F86AF969FBF7A5FC0346BB6040F67A
:1052E8009C23C2F200037A691A60BB6A83F0004308
:1052F8001846F969FBF796FC03461A4640F69C23C4
:10530800C2F200035A6040F69C23C2F200037A6A94
:105318009A60F868796AFBF785FC0346184639698C
:10532800FBF778FB03461A4640F69C23C2F20003BB
:10533800DA60B868796AFBF775FC0346B8691946FC
:10534800FBF766FB03461A4640F69C23C2F20003AD
:105358001A61FB6A83F000431846B96AFBF762FCDE
:1053680003461A4640F69C23C2F200035A61B86904
:10537800796AFBF757FC0346B8681946FBF748FB00
:1053880003461A4640F69C23C2F200039A61386924
:10539800796AFBF747FC03461846F968FBF73AFBBE
:1053A80003461A4640F69C23C2F20003DA61B86A43
:1053B800396BFBF737FC03461A4640F69C23C2F2CA
:1053C80000031A6200E000BF07F14007BD4680BD38
:1053D800F0B585B000AF78607B681B88FB817B687F
:1053E8005B88BB817B689B887B8140F69C23C2F2EB
:1053F80000031C68B7F90E301846FBF7BFFB0346DD
:1054080020461946FBF70EFC03461C4640F69C2333
:10541800C2F20003DD68B7F90C301846FBF7AEFBA3
:10542800034628461946FBF7FDFB03462046194666
:10543800FBF7F0FA03461C4640F69C23C2F2000331
:105448009D69B7F90A301846FBF798FB03462846CA
:105458001946FBF7E7FB034620461946FBF7DAFA3D
:105468000346184613F02EFA03469AB27B681A8050
:105478007B6803F1020440F69C23C2F200035D68D6
:10548800B7F90E301846FBF779FB0346284619464C
:10549800FBF7C8FB03461D4640F69C23C2F20003F7
:1054A8001E69B7F90C301846FBF768FB034630460F
:1054B8001946FBF7B7FB034628461946FBF7AAFA35
:1054C80003461D4640F69C23C2F20003DE69B7F985
:1054D8000A301846FBF752FB034630461946FBF7DD
:1054E800A1FB034628461946FBF794FA03461846DB
:1054F80013F0E8F903469BB223807B6803F10404A8
:1055080040F69C23C2F200039D68B7F90E30184696
:10551800FBF734FB034628461946FBF783FB034693
:105528001D4640F69C23C2F200035E69B7F90C30B1
:105538001846FBF723FB034630461946FBF772FB78
:10554800034628461946FBF765FA03461D4640F60A
:105558009C23C2F200031E6AB7F90A301846FBF70B
:105568000DFB034630461946FBF75CFB034628460D
:105578001946FBF74FFA0346184613F0A3F90346FA
:105588009BB2238007F11407BD46F0BD80B584B0F7
:1055980000AFF860B9601346FB7140F6C020C2F254
:1055A8000000F9684FF0060215F000F9FB7903F1E5
:1055B800FF33072B00F2208101A252F823F000BF2D
:1055C800E95500082356000863560008A956000844
:1055D800E95600082F5700086F570008B55700080C
:1055E80040F6C023C2F200031B889AB2BB681A8037
:1055F800BB6803F1020240F6C023C2F200035B88D5
:105608009BB21380BB6803F1040240F6C023C2F2C8
:1056180000039B889BB21380EFE040F6C023C2F2E0
:1056280000035B889AB2BB681A80BB6803F1020268
:1056380040F6C023C2F200031B88C3F100039BB2EB
:105648009BB21380BB6803F1040240F6C023C2F288
:1056580000039B889BB21380CFE040F6C023C2F2C0
:1056680000031B88C3F100039BB29AB2BB681A807F
:10567800BB6803F1020240F6C023C2F200035B8854
:10568800C3F100039BB29BB21380BB6803F1040211
:1056980040F6C023C2F200039B889BB21380ACE0A3
:1056A80040F6C023C2F200035B88C3F100039BB23B
:1056B8009AB2BB681A80BB6803F1020240F6C023A5
:1056C800C2F200031B889BB21380BB6803F104027B
:1056D80040F6C023C2F200039B889BB213808CE083
:1056E80040F6C023C2F200031B88C3F100039BB23B
:1056F8009AB2BB681A80BB6803F1020240F6C02365
:10570800C2F200035B889BB21380BB6803F10402FA
:1057180040F6C023C2F200039B88C3F100039BB28A
:105728009BB2138069E040F6C023C2F200035B8895
:105738009AB2BB681A80BB6803F1020240F6C02324
:10574800C2F200031B889BB21380BB6803F10402FA
:1057580040F6C023C2F200039B88C3F100039BB24A
:105768009BB2138049E040F6C023C2F200031B88B5
:105778009AB2BB681A80BB6803F1020240F6C023E4
:10578800C2F200035B88C3F100039BB29BB2138093
:10579800BB6803F1040240F6C023C2F200039B88F1
:1057A800C3F100039BB29BB2138026E040F6C023EE
:1057B800C2F200035B88C3F100039BB29AB2BB68D4
:1057C8001A80BB6803F1020240F6C023C2F200034C
:1057D8001B88C3F100039BB29BB21380BB6803F123
:1057E800040240F6C023C2F200039B88C3F1000301
:1057F8009BB29BB2138000E000BF40F22103C2F2CB
:1058080000031B7883F00103DBB2002B02D0B868D9
:10581800FFF7DEFD07F11007BD4680BD80B483B0F9
:1058280000AF786041F21823C2F200037A681A6068
:1058380007F10C07BD4680BC704700BF80B582B039
:1058480000AF0346FB7141F68063C2F200035B7B45
:10585800002B07D040F6D223C2F200034FF001021A
:105868001A7006E040F6D223C2F200034FF000029D
:105878001A704FF4007001F031F80346002B59D02C
:1058880041F21823C2F200031B681B689A6841F6AC
:105898006C63C2F200035B78002B0CBF002301236A
:1058A800DBB2184690470346002B18D040F6D323A6
:1058B800C2F200034FF001021A7041F21823C2F23B
:1058C80000031B681B681B6998470346002B06D01A
:1058D80040F6D323C2F200034FF002021A7041F2DD
:1058E8001823C2F200031B681B68DB68984703464D
:1058F800002B0DD041F66C63C2F200035B78002BDD
:1059080006D140F6D323C2F200034FF002021A7008
:1059180041F21823C2F200031B681B689B69984771
:105928000346002B06D040F6D323C2F200034FF003
:1059380000021A704FF020000AF03EFD0346002BCB
:1059480023D041F68063C2F200039B7A002B06D174
:1059580041F68063C2F20003DB7A002B0ED041F6D9
:105968006C63C2F20003DB7A002B07D140F6D42324
:10597800C2F200034FF001021A7006E040F6D42389
:10598800C2F200034FF000021A7040F6D323C2F2AD
:1059980000031B78022B0AD14FF04C004FF04E0148
:1059A8004FF04E024FF0440300F08AF873E040F6DF
:1059B800D323C2F200031B78012B0AD14FF0530006
:1059C8004FF04D014FF04C024FF04D0300F078F8C6
:1059D80061E040F6D423C2F200031B78012B0AD100
:1059E8004FF053004FF053014FF04E024FF04D036C
:1059F80000F066F84FE040F6D223C2F200031B78AD
:105A0800012B0AD14FF053004FF053014FF05302CE
:105A18004FF04D0300F054F83DE0FB79002B0AD01D
:105A28004FF053004FF04D014FF04D024FF044033B
:105A380000F046F82FE040F6D523C2F200031B78A9
:105A4800012B11D141F66C63C2F200035B78002B85
:105A58000AD04FF053004FF053014FF04D024FF072
:105A68004E0300F02DF816E040F6D023C2F20003F2
:105A78001B78002B04D04FF0320000F0CFF80AE07A
:105A880040F6C823C2F200034FF000021A704FF02C
:105A9800000004F055FA07F10807BD4680BD00BFB5
:105AA80080B483B000AF0346FB7140F6D023C2F246
:105AB8000003FA791A7007F10C07BD4680BC7047DD
:105AC80080B584B000AFF871B9717A713B71FB7918
:105AD8003B72BB797B727B79BB723B79FB7240F678
:105AE800D123C2F200031B7807F11002D31813F870
:105AF800083CA3F144030A2B28D801A252F823F04A
:105B0800455B0008555B0008555B0008555B0008BD
:105B1800555B0008555B0008555B0008555B00089D
:105B28003D5B0008355B00084D5B00084FF06403DF
:105B3800FB810FE04FF0C803FB810BE04FF4FA63E1
:105B4800FB8107E04FF00003FB8103E04FF03203D5
:105B5800FB8100BF40F6D123C2F200031B78022B61
:105B680006D8FB89002B03D0FB89184600F056F8AD
:105B780040F6D123C2F200031B78022B19D904F096
:105B8800D3FA0246FB89D21A40F6CC23C2F20003AC
:105B98001B689A420DD940F6D123C2F200034FF098
:105BA80000021A7040F6D023C2F200034FF0000240
:105BB8001A7040F6C923C2F200031B78012B02D0E9
:105BC800FB89002B25D140F6D123C2F200031B78B4
:105BD800022B0CD840F6D123C2F200031B7803F144
:105BE8000103DAB240F6D123C2F200031A7040F67C
:105BF800C923C2F200034FF000021A7040F6C8230E
:105C0800C2F200034FF000021A704FF0000004F0D7
:105C180097F907F11007BD4680BD00BF80B582B077
:105C280000AF0346FB8040F6C823C2F200031B788E
:105C3800002B3AD004F078FA0246F98840F6CC23D3
:105C4800C2F200031B68CB189A424ED340F6C82311
:105C5800C2F200034FF000021A704FF0000004F087
:105C68006FF904F061FA024640F6CC23C2F2000351
:105C78001A6040F6D023C2F200031B78002B0CD028
:105C880040F6D023C2F200031B7803F1FF33DAB2E7
:105C980040F6D023C2F200031A7040F6C923C2F2BC
:105CA80000034FF001021A701FE004F03DFA0246AB
:105CB80040F6CC23C2F200031B6803F132039A4278
:105CC80014D340F6C823C2F200034FF001021A7041
:105CD8004FF0010004F034F904F026FA024640F6C9
:105CE800CC23C2F200031A6000E000BF07F10807E6
:105CF800BD4680BD80B485B000AF786039604FF094
:105D08000003FB737B68BB6008E0BB681A78FB7B09
:105D18005340FB73BB6803F10103BB607A683B68BF
:105D2800D218BB689A42F0D8FB7B184607F11407D3
:105D3800BD4680BC704700BF80B582B000AF4FF44D
:105D48007843C0F601037B604FF00003FB707B686B
:105D58001A784CF6AC43C0F601031B789A4202D07D
:105D68004FF000031FE07B685B88B3F5697F08D1BB
:105D78007B681B79BE2B04D17B6893F8A133EF2B8A
:105D880002D04FF000030EE078684FF46971FFF716
:105D9800B1FF0346FB70FB78002B02D04FF00003E5
:105DA80001E04FF00103184607F10807BD4680BD22
:105DB80080B584B004AF17480AF07CFB1548164933
:105DC8000AF0B2FB154803F0EFFC15480BF0E8FAAF
:105DD80041F61843C2F200031B78184604F084FF0A
:105DE800104807F0B9FB104808F052FA0F4801F0C4
:105DF8005BFC0F4803F0C8FC0E4B00930E4B01935D
:105E08000E4B02930E480F49034A0F4B05F0ACFFA7
:105E1800BD4680BD371C00204019002064190020B1
:105E28009C190020DA1C0020191C0020D01C00201E
:105E3800681900208919002078190020D81C002032
:105E4800901C002046190020D61C002080B500AF09
:105E5800FFF772FF034683F00103DBB2002B03D088
:105E68004FF00A0004F0F0FA41F67000C2F20000A8
:105E78004FF47841C0F601014FF4697214F096FCB2
:105E880041F67003C2F2000393F8A033022B07D93E
:105E980041F67003C2F200034FF0000283F8A0231A
:105EA80041F67003C2F2000393F8A0334FF0D0021A
:105EB80002FB03F303F5987241F67003C2F2000384
:105EC800D21841F61843C2F2000319464FF0D00326
:105ED800084611461A4614F069FCFFF769FF80BDB1
:105EE80080B500AFFFF7B2FF4FF00F004FF014017D
:105EF8004FF001020FF0C6FF80BD00BF80B582B031
:105F080000AF0346FB71FB794FF0D00202FB03F3AD
:105F180003F5987241F67003C2F20003D21841F6F5
:105F28001843C2F2000311461A464FF0D003084640
:105F380011461A4614F03AFC07F10807BD4680BD21
:105F480080B584B000AF4FF00003FB734FF003033C
:105F5800FB714CF6AC43C0F601031A7841F67003A6
:105F6800C2F200031A7041F67003C2F200034FF444
:105F780069725A8041F67003C2F200034FF0BE0204
:105F88001A7141F67003C2F200034FF0EF0283F872
:105F9800A12341F67003C2F200034FF0000283F818
:105FA800A22341F67000C2F200004FF46971FFF7B6
:105FB800A1FE03461A4641F67003C2F2000383F8B5
:105FC800A22311F0E9FF30E04FF0340012F0B8F8E6
:105FD8004FF47840C0F6010012F010F80346FB7346
:105FE8004FF00003BB6015E0BB6803F1006303F5E5
:105FF800FC33B96841F67002C2F200028A181268CE
:106008001846114612F040F80346FB73BB6803F1CB
:106018000403BB60BA6840F2A3339A4202D8FB7B00
:10602800042BE1D0FB7B042B0DD097F90730002B14
:106038000CBF00230123DBB2FA7902F1FF32FA71B7
:10604800002BC1D100E000BF11F0C6FFFB7B042B81
:1060580007D1FFF771FE034683F00103DBB2002B83
:1060680003D04FF00A0004F0EFF907F11007BD461E
:1060780080BD00BF80B500AFFFF75EFE0346002B72
:1060880002D100F003F800E000BF80BD80B500AF8A
:1060980000F036F9FFF754FF80BD00BF80B483B02D
:1060A80000AF78607B684FF000025A807B684FF041
:1060B80000021A807B684FF000029A8007F10C07F3
:1060C800BD4680BC704700BF80B483B000AF786025
:1060D8007B684FF028021A707B684FF01E029A7294
:1060E8007B684FF017021A757B684FF028025A70C8
:1060F8007B684FF01E02DA727B684FF017025A7500
:106108007B684FF055029A707B684FF02D021A7326
:106118007B684FF000029A757B684FF03202DA70A4
:106128007B684FF000025A737B684FF00002DA7503
:106138007B684FF00B021A717B684FF000029A736C
:106148007B684FF000021A767B684FF014025A7190
:106158007B684FF00802DA737B684FF02D025A769D
:106168007B684FF00E029A717B684FF014021A7424
:106178007B684FF050029A767B684FF05A02DA71CA
:106188007B684FF00A025A747B684FF06402DA7633
:106198007B684FF028021A727B684FF078025A72B7
:1061A8007B684FF02D02DA747B684FF001025A7752
:1061B80007F10C07BD4680BC704700BF80B483B0B0
:1061C80000AF78607B684FF0C8021A807B684FF098
:1061D80014029A707B684FF01E02DA707B684FF0E9
:1061E80001021A717B684FF06402DA807B684FF411
:1061F80096721A817B684FF028025A8107F10C07C2
:10620800BD4680BC704700BF80B483B000AF7860E3
:106218007B684FF015021A707B6849F69A12C3F62C
:1062280019725A607B6842F6F602C3F67C729A606D
:106238007B6840F63D22C3F67772DA6007F10C07F7
:10624800BD4680BC704700BF80B483B000AF7860A3
:106258007B684FF000021A707B684FF000025A709A
:106268007B684FF000029A7007F10C07BD4680BCAE
:10627800704700BF80B483B000AF78607B6840F29D
:106288007E421A807B6840F23A725A807B684FF4EB
:106298007A729A8007F10C07BD4680BC704700BF30
:1062A80080B483B000AF78607B6840F27E521A8079
:1062B8007B6840F2EA525A807B6840F2B4529A8076
:1062C8007B684FF03202DA8007F10C07BD4680BCCC
:1062D800704700BF80B483B000AF78607B684FF030
:1062E80000021A707B684FF000025A707B684FF00A
:1062F80000029A7007F10C07BD4680BC704700BFCA
:1063080080B584B000AF4BF61412C0F6010207F155
:1063180004031068516803C341F67000C2F200001C
:106328004FF000014FF4697214F0EEFA41F618408C
:10633800C2F200004FF000014FF0D00214F0E4FA6E
:106348004CF6AC43C0F601031A7841F67003C2F26A
:1063580000031A7041F67003C2F200034FF0030203
:106368005A7100F0FFFA4FF0020000F0CDFA41F642
:106378007003C2F200034FF0000283F8A02341F635
:106388007003C2F200034FF41672A3F8F02041F62E
:106398007003C2F200034FF0FA02A3F8F22041F6AC
:1063A8007003C2F200034FF02A02A3F8EE20E64879
:1063B800FFF774FEE548FFF747FF41F67003C2F2A6
:1063C80000034FF00002A3F8E62041F67003C2F282
:1063D80000034FF00002A3F8E82041F67003C2F270
:1063E80000034FF00002A3F8EA2041F67003C2F25E
:1063F80000034FF0000283F8ED2041F67003C2F26B
:1064080000034FF4FA72A3F8F62041F67003C2F2C3
:1064180000034FF0010283F8EC2041F67003C2F24A
:1064280000034FF0200283F8F42041F67003C2F213
:1064380000034FF06E0283F8042141F67003C2F2A4
:1064480000034FF02B0283F8052141F67003C2F2D6
:1064580000034FF0210283F8062141F67003C2F2CF
:1064680000034FF0000283F80721B948FFF732FF15
:1064780041F67003C2F200034FF0000283F81021C6
:1064880041F67003C2F2000340F2DC52A3F8122175
:1064980041F67003C2F2000340F24C42A3F8142103
:1064A80041F67003C2F2000340F26C72A3F81621A1
:1064B80041F67003C2F200034FF0000283F818217E
:1064C80041F67003C2F200034FF0000283F819216D
:1064D80041F67003C2F200034FF0010283F81A215B
:1064E8009C48FFF7C7FE9C48FFF7DAFE41F67003A9
:1064F800C2F200034FF4C872A3F8DE2041F670031D
:10650800C2F200034FF03202A3F8E02041F6700314
:10651800C2F200034FF0000283F81C2141F6700319
:10652800C2F200034FF0000283F81D2141F6700308
:10653800C2F200034FF4E132C3F8202141F67003A0
:10654800C2F200034FF41652C3F8242141F6700337
:10655800C2F200034FF0000283F8282141F67003CD
:10656800C2F200034FF0000283F8292141F67003BC
:10657800C2F200034FF0520283F82A2141F6700359
:10658800C2F2000340F6AC529A8141F67003C2F29F
:1065980000034FF000029A7341F67003C2F2000341
:1065A8004FF0000283F81B2141F61843C2F20003A2
:1065B8004FF000021A706948FFF786FD41F618434C
:1065C800C2F200034FF05A02DA7741F61843C2F2DA
:1065D80000034FF0410283F8202041F61843C2F22D
:1065E80000034FF0000283F8232041F61843C2F25B
:1065F80000034FF0000283F8242041F61843C2F24A
:1066080000034FF0000283F8252041F61843C2F238
:10661800000340F2DC52DA8441F61843C2F2000368
:106628004FF0320283F8212041F61843C2F20003EA
:106638004FF0000283F82220494803F07FFF41F61B
:106648001843C2F200034FF000021A8541F61843BE
:10665800C2F200034FF0040283F82E2041F61843DB
:10666800C2F200034FF0280283F82F2041F61843A6
:10667800C2F200034FF0280283F830203948FFF7B0
:10668800C3FD41F61843C2F200034FF0010283F83C
:1066980044204BF60810C0F6010033490AF08CF983
:1066A80041F61843C2F200034FF0000283F870204D
:1066B80041F61843C2F200034FF0000283F871203C
:1066C80041F61843C2F200034FF0280283F8722003
:1066D80041F61843C2F200034FF0010283F8732019
:1066E80041F61843C2F200034FF0000283F8762007
:1066F80041F61843C2F200034FF44872A3F874201D
:1067080041F61843C2F200034FF00A0283F8B8209A
:1067180041F61843C2F200034FF0C80283F8B920CB
:1067280041F61843C2F200034FF49662A3F8BA2068
:1067380041F61843C2F2000340F2D932A3F8BC2054
:106748004FF00003FB6058E0681900205219002040
:106758009C1900204019002046190020191C00200F
:10676800421C00204C1C00207819002041F61843D8
:10677800C2F20003FA6802F10F024FF47F7123F8A6
:10678800321041F61842C2F20002FB6803F10F030F
:106798004FEAC303D3184FF4FA625A8041F61842FD
:1067A800C2F20002FB6803F10F034FEAC303D318D8
:1067B80040F2DC529A8007F10402FB68D31819787A
:1067C80041F61842C2F20002FB6803F10F034FEAD8
:1067D800C303D3180A469A7141F61842C2F200025E
:1067E800FB6803F10F034FEAC303D3184FF0FF020E
:1067F800DA71FB6803F10103FB60FB68072BB5DD69
:1068080041F61843C2F200034FF0010283F8BE209C
:1068180041F61843C2F200034FF0010283F8BF208B
:1068280041F61843C2F200034FF0010283F8C0207A
:106838002148FFF7C3FC4FF00003FB6010E041F66E
:106848007003C2F20003FA6802F101024FEA021271
:106858009B184FF000021A60FB6803F10103FB600C
:10686800FB680B2BEBDD4FF00003FB601CE0FB68C3
:106878004FF0D00202FB03F303F5987241F6700360
:10688800C2F20003D21841F61843C2F200031146BF
:106898001A464FF0D003084611461A4613F086FFF1
:1068A800FB6803F10103FB60FB68022BDFDD07F1E6
:1068B8001007BD4680BD00BFDA1C002080B500AFC0
:1068C80041F67003C2F2000393F8A0331846FFF7AD
:1068D80015FBFFF735FBFFF703FB80BD80B483B0E2
:1068E80000AF786041F67003C2F200039A687B68D3
:1068F8001340002B0CBF00230123DBB2184607F11D
:106908000C07BD4680BC704780B483B000AF786088
:1069180041F67003C2F200039A687B681A4341F695
:106928007003C2F200039A6007F10C07BD4680BCF1
:10693800704700BF80B483B000AF786041F6700341
:10694800C2F200039A687B686FEA03031A4041F6B3
:106958007003C2F200039A6007F10C07BD4680BCC1
:10696800704700BF80B400AF41F67003C2F2000365
:106978004FF000029A60BD4680BC704780B400AFFB
:1069880041F67003C2F200039B681846BD4680BCFE
:10699800704700BF80B500AF4FF04000FFF79EFF83
:1069A8000346002B09D04FF00100FFF797FF03467D
:1069B800002B02D04FF0010301E04FF0000303F079
:1069C8000103DBB2184680BD80B485B000AFF86023
:1069D800B9607A60FA68BB689A4201DABB6806E077
:1069E800FA687B689A4201DD7B6800E0FB6818461C
:1069F80007F11407BD4680BC704700BF80B483B060
:106A080000AF78607B684FF000021A6107F10C074D
:106A1800BD4680BC704700BFB0B582B000AF78609B
:106A280039607B681B6903F101027B681A617B6826
:106A38001B69012B0BD17B683A685A607B685A68DE
:106A48007B681A607B684FF000029A6042E07B68BE
:106A58001C687B681B6838681946F9F7D9FF034634
:106A68001D467B681B691846FAF788F803462846CE
:106A78001946FAF78BF9034620461946F9F7CAFF73
:106A880003461A467B685A607B689C687B681B686B
:106A980038681946F9F7BCFF03461D467B685B68F2
:106AA80038681946F9F7B4FF034628461946FAF735
:106AB800B9F8034620461946F9F7ACFF03461A46CB
:106AC8007B68DA607B685A687B681A607B68DA687A
:106AD8007B689A6007F10807BD46B0BD90B583B0E2
:106AE80000AF78607B681B69012B0FDD7B68DC6871
:106AF8007B681B6903F1FF331846FAF73FF8034632
:106B080020461946FAF742F9034601E04FF0000320
:106B1800184607F10C07BD4690BD00BF80B582B08E
:106B280000AF78607868FFF7D9FF0346184611F080
:106B380097FF0346184607F10807BD4680BD00BF0A
:106B480080B582B000AF0346FB80B7F9063018461F
:106B5800F9F792FC02460B461046194608A3D3E9FA
:106B68000023F9F7EFFC02460B4610461946F9F7E1
:106B7800FBFE0346184607F10807BD4680BD00BF67
:106B8800399D52A246DF913F80B586B000AFF860CC
:106B9800B9607A60FB70FB78002B02D04FF03003AD
:106BA80001E04FF02003FB743B6A7B6103E07B68E4
:106BB80003F1FF337B607B691B78002B0CBF00233C
:106BC8000123DBB27A6902F101027A61002B09D054
:106BD8007B68002BEBDC05E0FA7CBB68F8681146A3
:106BE800984700E000BF7B68002BD4BF0023012337
:106BF800DBB27A6802F1FF327A60002BECD104E054
:106C0800BA7CBB68F868114698473B6A1B78BB7426
:106C1800BB7C002B0CBF00230123DBB23A6A02F1D4
:106C280001023A62002BEBD107F11807BD4680BD7F
:106C380080B58CB002AFF860B9607A603B601AE149
:106C480097F82730252B06D097F82720BB68F868D7
:106C5800114698470FE14FF0000387F826304FF0B0
:106C6800000387F825304FF000037B617B681A78B2
:106C780087F8272003F101037B6097F82730302B32
:106C88000AD17B681A7887F8272003F101037B6013
:106C98004FF0010387F8263097F827302F2B12D9A9
:106CA80097F82730392B0ED897F8271007F10402E8
:106CB80007F11403084611464FF00A0200F064FA7F
:106CC800034687F8273097F827306C2B0AD17B6862
:106CD8001A7887F8272003F101037B604FF001033E
:106CE80087F8253097F82730642B44D0642B0EDCC6
:106CF800582B67D0582B06DC002B00F0CD80252BB5
:106D080000F0B180B6E0632B00F09480B2E0752B00
:106D180005D0782B56D0732B00F09780AAE097F80F
:106D28002530002B0ED03B6803F104023A601A6844
:106D380007F1180310464FF00A014FF0000200F067
:106D4800F3F80DE03B6803F104023A601A6807F1B2
:106D5800180310464FF00A014FF0000200F066F9E0
:106D68007A6997F8263007F118010091F868B96830
:106D7800FFF70AFF7FE097F82530002B0CD03B681F
:106D880003F104023A601B681A4607F1180310461B
:106D9800194600F029F90AE03B6803F104023A6059
:106DA8001A6807F118031046194600F09FF97A6926
:106DB80097F8263007F118010091F868B968FFF7CD
:106DC800E3FE58E097F82530002B14D03B6803F118
:106DD80004023A60196897F82730582B14BF00232B
:106DE8000123DBB21A4607F1180308464FF01001D9
:106DF80000F09AF813E03B6803F104023A6019685E
:106E080097F82730582B14BF00230123DBB21A460A
:106E180007F1180308464FF0100100F007F97A69E6
:106E280097F8263007F118010091F868B968FFF75C
:106E3800ABFE20E03B6803F104023A601B68DAB25B
:106E4800BB68F8681146984715E07A693B6803F112
:106E5800040139601B680093F868B9684FF00003B3
:106E6800FFF792FE07E097F82720BB68F8681146FD
:106E7800984700E000BF7B681A7887F8272097F8C2
:106E88002720002A0CBF00220122D2B203F10103FD
:106E98007B60002A7FF4D4AE07F12807BD4680BD89
:106EA80080B483B000AF7860396040F6D823C2F26E
:106EB80000033A681A6040F6DC23C2F200037A68DD
:106EC8001A6007F10C07BD4680BC70470FB480B547
:106ED80082B000AF07F114037B6040F6DC23C2F2F6
:106EE80000031A6840F6D823C2F200031B68104654
:106EF80019463A697B68FFF79BFE00BF41F60473A9
:106F0800C2F200031B68184602F0C0FF034683F074
:106F18000103DBB2002BF1D107F10807BD46BDE83C
:106F2800804004B0704700BF80B489B000AFF860FB
:106F3800B9607A603B604FF00003FB614FF00103DA
:106F4800BB6104E0BB69BA6802FB03F3BB61FA6882
:106F5800BB69B2FBF3F2BB689A42F3D237E0FA6836
:106F6800BB69B2FBF3F37B61FB68BA69B3FBF2F26E
:106F7800B96901FB02F29B1AFB60BA69BB68B2FBF4
:106F8800F3F3BB61FB69002B05D17B69002B02DCA5
:106F9800BB69002B1BD17B69092B08DD7B68002BA3
:106FA80002D04FF0370301E04FF0570301E04FF0F4
:106FB80030037A69D2B29B18DAB23B681A703B6820
:106FC80003F101033B60FB6903F10103FB61BB694A
:106FD800002BC4D13B684FF000021A7007F1240758
:106FE800BD4680BC704700BF80B582B000AF7860F6
:106FF80039607B68002B0BDA7B68C3F100037B6088
:107008003B684FF02D021A703B6803F101033B60A7
:107018007B6818464FF00A014FF000023B68FFF703
:1070280083FF07F10807BD4680BD00BF80B489B063
:1070380000AFF860B9607A603B604FF00003FB6115
:107048004FF00103BB6104E0BB69BA6802FB03F3BC
:10705800BB61FA68BB69B2FBF3F2BB689A42F3D230
:1070680037E0FA68BB69B2FBF3F37B61FB68BA6986
:10707800B3FBF2F2B96901FB02F29B1AFB60BA6931
:10708800BB68B2FBF3F3BB61FB69002B05D17B69DD
:10709800002B02DCBB69002B1BD17B69092B08DDA7
:1070A8007B68002B02D04FF0370301E04FF0570305
:1070B80001E04FF030037A69D2B29B18DAB23B682C
:1070C8001A703B6803F101033B60FB6903F101039C
:1070D800FB61BB69002BC4D13B684FF000021A70FA
:1070E80007F12407BD4680BC704700BF80B582B059
:1070F80000AF786039607B68002B0BDA7B68C3F1DE
:1071080000037B603B684FF02D021A703B6803F167
:1071180001033B607B6818464FF00A014FF00002FC
:107128003B68FFF783FF07F10807BD4680BD00BF36
:1071380080B483B000AF0346FB71FB792F2B06D9CF
:10714800FB79392B03D8FB79A3F1300315E0FB79E0
:10715800602B06D9FB79662B03D8FB79A3F157037B
:107168000BE0FB79402B06D9FB79462B03D8FB793A
:10717800A3F1370301E04FF0FF33184607F10C077E
:10718800BD4680BC704700BF80B588B000AFB9600D
:107198007A603B600346FB73BB681B68FB614FF07A
:1071A8000003BB6111E07A697B689A4216DCBB690F
:1071B8007A6802FB03F27B69D318BB61FB691B7811
:1071C800FB73FB6903F10103FB61FB7B1846FFF7C7
:1071D800AFFF78617B69002BE5DA00E000BFBB6890
:1071E800FA691A603B68BA691A60FB7B184607F1AE
:1071F8002007BD4680BD00BF80B584B000AFF860F1
:10720800B9607A60FA687B68B2FBF3F3002B09D0A7
:10721800FA687B68B2FBF3F31846B9687A68FFF737
:10722800EBFFB860FB687A68B3FBF2F2796801FBA0
:1072380002F29A1A4BF61C13C0F601039A5CBB685B
:107248001A70BB6803F10103184607F11007BD4621
:1072580080BD00BF80B584B000AFF860B9607A60C7
:107268007B68012B02DD7B68242B02DD4FF00A03CB
:107278007B60FB68002B14DABB684FF02D021A7094
:10728800FB68C3F10001BB6803F101027B68084693
:1072980011461A46FFF7B0FF03464FF000021A7076
:1072A8000AE0FA687B681046B9681A46FFF7A4FF37
:1072B80003464FF000021A70BB68184607F1100722
:1072C800BD4680BD80B58CB000AF7860396007F1ED
:1072D8000C034FF000021A6003F104034FF00002A0
:1072E8001A6003F104034FF000021A6003F104036B
:1072F8004BF64413C0F60103FB6278684FF00001B7
:10730800F9F74CFE0346002B09D0786841F26F214B
:10731800C3F60321F9F77EFB03467B6008E0786833
:1073280041F26F21C3F60321F9F772FB03467B6034
:1073380078684FF00001C4F27A41F9F773FC03460C
:107348001846F9F735FE0346BB62BB6A83EAE37267
:10735800A2EBE37207F11803104619464FF00A0230
:10736800FFF778FFBB6A002B03DB4FF020033B736A
:1073780002E04FF02D033B7307F11803184613F092
:107388005BFC0346012B11D14FF030037B734FF0A8
:107398003003BB734FF03003FB7307F10C0207F1A6
:1073A80018031046194613F045FB32E007F118039D
:1073B800184613F041FC0346022B0ED14FF0300360
:1073C8007B734FF03003BB7307F10C0207F118030E
:1073D8001046194613F02EFB1BE007F11803184658
:1073E80013F02AFC0346032B0BD14FF030037B73B9
:1073F80007F10C0207F118031046194613F01AFB9F
:1074080007E007F10C0207F118031046194613F0BC
:1074180011FB07F10C03184613F00EFC0346DBB210
:10742800A3F1030387F8273097F8273007F10C02F8
:10743800386811461A4613F09DFC97F827303A68C9
:10744800D3184FF000021A703868F96A13F0F2FA8C
:1074580097F8273007F10C02D3183868194613F04B
:10746800E9FA3B68184607F13007BD4680BD00BF02
:1074780090B589B000AF78604FF00003FB6103E07E
:107488007B6803F101037B607B681B78202BF7D0B6
:107498007B681B78092BF3D04FF07E53BB617B6868
:1074A8001B782D2B09D14FF00003CBF68073BB61FD
:1074B8007B6803F101037B6007E07B681B782B2B5B
:1074C80003D17B6803F101037B604FF000037B610C
:1074D8001AE078694FF00001C4F22011F9F7A2FB15
:1074E80003461C467B681B78A3F130031846F9F75E
:1074F80045FB034620461946F9F78CFA03467B619B
:107508007B6803F101037B607B681B782F2B03D911
:107518007B681B78392BDCD97B681B782E2B31D103
:107528004FF00003C4F22013FB607B6803F10103F2
:107538007B601FE07B681B78A3F130031846F9F7DE
:107548001DFB03461846F968F9F720FC03467869DD
:107558001946F9F75FFA03467B61F8684FF00001B6
:10756800C4F22011F9F75EFB0346FB607B6803F168
:1075780001037B607B681B782F2B03D97B681B7802
:10758800392BD7D94FF07E533B617B681B78652B2D
:1075980003D07B681B78452B61D17B6803F101031D
:1075A8007B604FF00003FB617B681B782D2B07D1B4
:1075B8004FF00103FB617B6803F101037B6007E087
:1075C8007B681B782B2B03D17B6803F101037B605D
:1075D8004FF00003BB6011E0BA6813464FEA83031B
:1075E8009B184FEA43031A467B681B78D318A3F10C
:1075F8003003BB607B6803F101037B607B681B7809
:107608002F2B03D97B681B78392BE5D9BB68B3F5D9
:107618009A7F10D94FF49A73BB600CE038694BF627
:107628002041C4F6BE41F9F7FDFA03463B61BB6849
:10763800A3F10803BB60BB68072BEFD80CE03869DF
:107648004FF00001C4F22011F9F7ECFA03463B6150
:10765800BB6803F1FF33BB60BB68002BEFD1FB694C
:10766800002B05D078693969F9F790FB034604E0E7
:1076780078693969F9F7D6FA03461846B969F9F706
:10768800D1FA0346184607F12407BD4690BD00BF4E
:1076980080B400AF40F6E023C2F200034FF00002CE
:1076A8009A80BD4680BC704780B582B000AF7860D4
:1076B80040F6E823C2F200037A681A60FFF7E8FF91
:1076C80007F10807BD4680BD80B483B000AF78607D
:1076D80040F6EC23C2F200037A681A6040F6E02311
:1076E800C2F200034CF6B042C0F601021A6040F63E
:1076F800E023C2F200034FF00002DA8040F6E023F4
:10770800C2F20003184607F10C07BD4680BC70475B
:1077180080B400AF40F6E023C2F200039B881BB29E
:10772800002B14BF00230123DBB21846BD4680BCE2
:10773800704700BF80B400AF40F6E023C2F20003F8
:107748009B8819B240F6E823C2F200031B681B7835
:107758001A4613464FEA83039B189942D4BF002365
:107768000123DBB21846BD4680BC704780B582B0A5
:1077780000AF0346FB71FFF7DDFF0346002B05D082
:10778800FB79002B02D04FF0010301E04FF000031A
:1077980003F00103DBB2184607F10807BD4680BDB8
:1077A80080B400AF40F6E023C2F200039B8819B210
:1077B80040F6E823C2F200031B681B781A4640F61D
:1077C800E823C2F200031B685B78D21813464FEA1D
:1077D80083039B189942D4BF00230123DBB21846C8
:1077E800BD4680BC704700BF80B500AF02F092FE76
:1077F80041F66C63C2F200034FF000021A7080BDBC
:1078080080B400AF40F6E023C2F200039B881BB2AD
:10781800142B0FDD40F6E023C2F200039B889BB2D5
:10782800A3F114039BB29AB240F6E023C2F200031C
:107838009A8006E040F6E023C2F200034FF000020F
:107848009A80BD4680BC704780B582B000AFFFF714
:1078580071FF0346002B4FD041F66C63C2F2000360
:107868005B78002B0CBF00230123DBB21846FFF71F
:107878007DFF0346002B31D04FF00003FB7111E070
:10788800FA7940F6EC23C2F200031B685B8999B2CF
:1078980041F6CC63C2F2000323F81210FB7903F11E
:1078A8000103FB71FB79022BEAD940F6E823C2F207
:1078B80000031B685B889AB241F6CC63C2F20003EE
:1078C800DA8040F6E023C2F20003DB8803F101030B
:1078D8009AB240F6E023C2F20003DA80FFF760FFB5
:1078E8000346002B06D141F66C63C2F200035B78B5
:1078F800002B01D1FFF778FF40F6E023C2F2000326
:107908009B8803F101039AB240F6E023C2F2000318
:107918009A8007F10807BD4680BD00BF80B586B0D4
:1079280000AF4FF00003BB75FEF7A4FBFEF78EFA1D
:1079380041F67003C2F200039B7B002B0CBF0023AF
:107948000123DBB2184602F0FBFBFDF739FB41F6D9
:107958007003C2F2000393F80731002B17D041F6E9
:107968007003C2F2000393F80731012B07D041F6E8
:107978007003C2F2000393F80731092B07D141F6CF
:107988007003C2F2000393F807313B700AE04FF02E
:1079980000033B7041F67003C2F200034FF000028F
:1079A80083F807213B461846FAF718FC4FF0020007
:1079B800FEF794FF0346002B02D09248FDF7B2FB76
:1079C8009148FDF72FFC4FF0020008F00BFD41F63F
:1079D8007003C2F20003B3F8EE1041F67003C2F26E
:1079E800000393F8ED2041F61843C2F200031B8D03
:1079F8001BB2864802F06AF80346BB75BB7D83F06C
:107A08000103DBB2002B03D04FF0030002F01CFD92
:107A18004FF48053C4F600034FF488429A614FF440
:107A28008053C4F600034FF488521A854FF00003C0
:107A3800FB752FE04FF48053C4F600034FF48052D7
:107A4800C4F60002928A92B282F4884292B29A8272
:107A58004FF48053C4F600034FF48052C4F600027A
:107A6800928A92B282F4885292B29A824FF01900A6
:107A780002F0D0FC4FF0010002F062FA4FF019005A
:107A880002F0C8FC4FF0000002F05AFAFB7D03F147
:107A98000103FB75FB7D092BCCD94FF48053C4F649
:107AA80000034FF488521A854FF48053C4F600033C
:107AB8004FF488421A8503F037F941F67003C2F291
:107AC80000035B791846524904F0DAF951480AF084
:107AD80005FD41F67003C2F200035B790E2B06D058
:107AE80041F67003C2F200035B79082B03D14FF013
:107AF8000103BB7202E04FF00003BB724FF48070C9
:107B0800FEF7ECFE0346002B06D14FF00800FEF707
:107B1800E5FE0346002B02D04FF0010301E04FF0D1
:107B2800000303F00103DBB2BB71FEF733FF03462A
:107B3800FB714FF00100FEF7D1FE03467B714FF059
:107B48000800FEF7CBFE0346002B0CBF00230123E1
:107B5800DBB283F00103DBB203F00103DBB23B715C
:107B680005F0CCFC03463B7241F61843C2F2000311
:107B780093F8C03003F00403002B0CBF002301234B
:107B8800DBB27B7241F67003C2F20003B3F8DE3059
:107B9800BB8141F67003C2F20003B3F8E030FB8109
:107BA8004FF47A733B824FF48040FEF797FE03460A
:107BB800002B06D041F67003C2F20003B3F8DA30A6
:107BC8003B82BB89B3F5FA7F02D94FF000033B82B1
:107BD80041F67003C2F20003B3F812317B8241F61A
:107BE8007003C2F2000393F80731012B02D0092B6E
:107BF80004D011E04FF00103FB7211E04FF00703CE
:107C0800FB720DE07419002056190020521900204B
:107C180080180020901900204FF00003FB7200BF6D
:107C28004C48FFF751FD024641F21823C2F2000307
:107C38001A6041F21823C2F200031B681846FDF7C8
:107C4800EDFDFDF79BF941F21823C2F200031B6812
:107C580018464149FBF76AFD07F104031846FBF78C
:107C680021F841F21823C2F200031B68394819466B
:107C780008F0F2FC4FF48070FEF730FE0346002B4C
:107C88001CD04FF00800FEF729FE034683F00103DD
:107C9800DBB2002B12D041F67003C2F2000393F856
:107CA8001D31DAB241F67003C2F2000393F81C31B9
:107CB80010461946294A2A4B05F05EFCFEF76AFE73
:107CC8000346002B18D041F67003C2F20003D3F824
:107CD800242141F67003C2F2000393F828311046BC
:107CE8001946FCF781FB41F67003C2F2000393F8D2
:107CF80029311846FCF7B0FB4FF40060FEF7EEFDA3
:107D08000346002B05D041F60470C2F2000009F0CA
:107D1800BBFB02F0DBF9024640F6F423C2F2000393
:107D28001A6041F67003C2F200035B79052B03D198
:107D38004FF4C87001F074FA4FF47A7001F044FD02
:107D480041F66C63C2F200034FF001025A7300F06F
:107D580033FCFCE778190020D01C0020DA1C002036
:107D6800191C002080B500AF41F67003C2F2000371
:107D7800B3F8D4309BB21BB2184604F073FBFEE78D
:107D880090B58BB000AF41F6CC63C2F20003DB883C
:107D98001AB241F61843C2F20003DB8C9A4203DAA6
:107DA8004FF06403BB6134E041F6CC63C2F20003D8
:107DB800DB881AB240F2CF739A4221DC41F61843AD
:107DC800C2F2000393F825301A4641F6CC63C2F29A
:107DD8000003DB8819B241F61843C2F20003DB8CBA
:107DE800CB1A03FB02F241F61843C2F20003DB8C04
:107DF800C3F5FA6392FBF3F3C3F16403BB6108E0D4
:107E080041F61843C2F2000393F82530C3F1640326
:107E1800BB614FF000033B62A0E141F6CC63C2F2C4
:107E280000033A6A33F812301AB241F67003C2F20C
:107E38000003B3F81231D21A6FF4F9739A4225DBB2
:107E480041F6CC63C2F200033A6A33F812301AB230
:107E580041F67003C2F20003B3F81231D21A40F2AD
:107E6800F3139A4212DC41F6CC63C2F200033A6A79
:107E780033F812301AB241F67003C2F20003B3F8B5
:107E88001231D31A002BB8BF5B4201E04FF4FA73EA
:107E98007B623B6A022B00F08F8041F61843C2F2E6
:107EA800000393F87030002B16D041F61843C2F245
:107EB800000393F870301A467B6A9A4209DA41F651
:107EC8001843C2F2000393F870307A6AD31A7B62BF
:107ED80002E04FF000037B627A6A48F21F53C5F252
:107EE800EB1383FB02034FEA63114FEAE273CB1AE9
:107EF8007B6141F6B863C2F200037A6933F8123045
:107F080099B27B696FF0630202FB03F27B6AD218B5
:107F18007B6903F1010041F6B863C2F2000333F84C
:107F2800103018B241F6B863C2F200037C6933F826
:107F380014301BB2C31A03FB02F248F21F53C5F2F6
:107F4800EB1383FB02034FEA63104FEAE273C31A91
:107F58009BB2CB189BB299B241F69863C2F2000368
:107F68003A6A23F8121041F61843C2F2000393F854
:107F780023307A6A02FB03F244F6D353C1F2620358
:107F880083FB02134FEA63114FEAE273CB1AC3F182
:107F98006403FB61FB699BB2BA6902FB03F248F216
:107FA8001F53C5F2EB1383FB02034FEA63114FEA39
:107FB800E273CB1AFB614FE041F61843C2F20003AB
:107FC80093F87130002B16D041F61843C2F2000323
:107FD80093F871301A467B6A9A4209DA41F61843D7
:107FE800C2F2000393F871307A6AD31A7B6202E016
:107FF8004FF000037B6241F67003C2F2000393F86E
:10800800EC305BB2C3F100039BB27A6A92B202FB16
:1080180003F39BB299B241F69863C2F200033A6A3D
:1080280023F8121041F61843C2F2000393F82430E3
:108038007A6A002AB8BF524202FB03F244F6D353CD
:10804800C1F2620383FB02134FEA63114FEAE27342
:10805800CB1AC3F16403FB6141F61843C2F2000373
:108068003A6A9B185B78FA6902FB03F248F21F53DD
:10807800C5F2EB1383FB02034FEA63114FEAE27385
:10808800CB1ADAB241F63853C2F20003396A5B18E8
:108098001A7041F61843C2F200033A6A9B1803F1BA
:1080A8000803DB78FA6902FB03F248F21F53C5F2B2
:1080B800EB1383FB02134FEA63114FEAE273CB1A07
:1080C800DAB241F63053C2F20003396A5B181A700B
:1080D80041F61843C2F200033A6A9B1803F11003F1
:1080E8005B79FA6902FB03F248F21F53C5F2EB13FE
:1080F80083FB02034FEA63114FEAE273CB1ADAB249
:1081080041F63453C2F20003396A5B181A7041F61B
:10811800CC63C2F200033A6A33F812301AB241F65D
:108128007003C2F20003B3F812319A4212DA41F630
:108138009863C2F200033A6A33F812309BB2C3F173
:1081480000039BB299B241F69863C2F200033A6AFF
:1081580023F812103B6A03F101033B623B6A022BCE
:108168007FF75BAE41F6CC63C2F20003DB881AB23C
:1081780041F67003C2F20003B3F8143110461946F1
:108188004FF4FA62FEF720FC786241F67003C2F2FF
:108198000003B3F814317A6AD31A4FF47A7202FBE7
:1081A80003F241F67003C2F20003B3F81431C3F5C9
:1081B800FA63B2FBF3F37B627A6A48F21F53C5F2A3
:1081C800EB1383FB02134FEA63114FEAE273CB1AF6
:1081D8007B6141F6A063C2F200037A6933F812307A
:1081E80099B27B696FF0630202FB03F27B6AD218D3
:1081F8007B6903F1010041F6A063C2F2000333F882
:10820800103018B241F6A063C2F200037C6933F85B
:1082180014301BB2C31A03FB02F248F21F53C5F213
:10822800EB1383FB02034FEA63104FEAE273C31AAE
:108238009BB2CB189BB29AB241F69863C2F2000384
:10824800DA8041F66C63C2F200035B7A002B78D0C7
:1082580041F63C53C2F200031B889AB241F6FA4336
:10826800C2F200031B889BB2D31A9BB29BB21BB20B
:108278001846FEF765FC3861386910F0EFFAF860C7
:10828800386910F05FFBB86041F69863C2F20003EA
:108298005B881BB21846F8F771FC03461846F96864
:1082A800F8F7C0FC03461C4641F69863C2F2000387
:1082B8001B881BB21846F8F761FC03461846B968D4
:1082C800F8F7B0FC034620461946F8F7A3FB034627
:1082D8001846F8F76DFE0346FB8041F69863C2F234
:1082E80000031B881BB21846F8F748FC03461846DB
:1082F800F968F8F797FC03461C4641F69863C2F202
:1083080000035B881BB21846F8F738FC034618468A
:10831800B968F8F787FC034620461946F8F778FB52
:1083280003461846F8F744FE03469AB241F69863A6
:10833800C2F200031A8041F69863C2F20003FA8879
:108348005A804FF00200FEF7C9FA0346002B2ED0E0
:1083580040F61033C2F200031B7803F10103DAB2CE
:1083680040F61033C2F200031A7040F61033C2F21E
:1083780000031A784AF6AB23CAF6AA23A3FB021312
:108388004FEA93010B464FEA43035B184FEA430356
:10839800D31ADBB2002B0AD1FCF752FEFCF79AFE87
:1083A80003461A4640F61133C2F200031A7040F62B
:1083B8001133C2F200031B78002B0CBF00230123EA
:1083C800DBB21846FDF73AFA00F03AFF034683F0AD
:1083D8000103DBB2002B06D04FF0020007F0ECFFE0
:1083E8000346002B07D101F0FFF9034683F0010390
:1083F800DBB2002B0ED04FF48053C4F600034FF4C9
:108408008052C4F60002928A92B282F4885292B2E2
:108418009A821DE041F66C63C2F200039B78002B40
:1084280006D04FF48053C4F600034FF488521A85DF
:1084380041F66C63C2F200035B78002B06D04FF460
:108448008053C4F600034FF488529A6109F0CCF8BF
:1084580040F6F023C2F200031A6840F61433C2F261
:1084680000031B68D31A002B31DB41F66C63C2F2A0
:1084780000035B7B002B23D141F66C63C2F200033F
:108488004FF000029A704FF48053C4F600034FF483
:108498008052C4F60002928A92B282F4885292B252
:1084A8009A8240F6F023C2F200031B6803F5F42217
:1084B80002F5907240F61433C2F200031A6006E027
:1084C80041F66C63C2F200034FF001029A700AF0A1
:1084D8003DF841F2E803C2F200031B78002B08D1F3
:1084E8004FF40060FEF7FAF90346002B01D009F0BB
:1084F800ADF84FF0200007F05FFF0346002B07D0D0
:1085080040F6F023C2F200031B68184607F022FF6A
:1085180041F61453C2F200039B68002B09D041F6C0
:108528001453C2F200039B6841F6EC40C2F200000B
:10853800984707F12C07BD4690BD00BF80B500AF36
:1085480001F052F90346002B1FD041F66C63C2F2CA
:1085580000039B78002B18D041F66C63C2F200032D
:108568005B78002B20D141F66C63C2F200034FF018
:1085780001025A7041F63C53C2F200031A8841F6D0
:10858800FA43C2F200031A800EE041F66C63C2F2AD
:1085980000035B78002B07D14FF002004FF0FF017A
:1085A8004FF001020DF06EFC80BD00BF80B400AF3B
:1085B800BD4680BC704700BF90B585B000AF4FF096
:1085C8000003FB734FF00003FB804FF000037B7147
:1085D8004FF000033B714FF00800FEF77FF90346A8
:1085E800002B04D0B04808F0BBF803463B7140F6B6
:1085F800F023C2F200031A6840F60033C2F2000307
:108608001B68D31A002B03DA3B79002B00F0E084B7
:108618004FF000033B7140F6F023C2F200031B68E1
:1086280003F59C4202F1200240F60033C2F2000337
:108638001A609D4841F6C861C2F2000108F0BEF810
:108648004FF48040FEF74AF90346002B08D041F664
:108658008063C2F200031B78002B01D101F05AFF9E
:1086680041F67003C2F2000393F81B31002B38D097
:1086780041F67003C2F2000393F81B3103F10302C1
:1086880041F6CC63C2F2000333F812307B80B7F9AD
:108698000230A3F57A7318464FF000014FF47A724E
:1086A800FEF792F903461846F8F768FA03461846A3
:1086B8004FF00001C4F27A41F8F768FB0346184608
:1086C8004FF44041C4F27F41F8F7ACFA034618462C
:1086D800F8F794FC03469AB241F6F843C2F2000355
:1086E8001A804FF40070FEF7F9F80346002B07D004
:1086F80041F21823C2F200031B681B685B699847A4
:108708004FF00003BB602FE0FB7B4FEA9303FB7342
:1087180041F6CC63C2F20003BA6833F812301AB2D9
:1087280041F67003C2F20003B3F814319A4203DD34
:10873800FB7B63F07F03FB7341F6CC63C2F200035B
:10874800BA6833F812301AB241F67003C2F2000365
:10875800B3F816319A4203DAFB7B43F04003FB730C
:10876800BB6803F10103BB60BB68032BCCDD40F69B
:108778000433C2F200031B78FA7B9A4214D140F604
:108788000533C2F200031B78F92B14D840F60533E1
:10879800C2F200031B7803F10103DAB240F6053395
:1087A800C2F200031A7006E040F60533C2F2000375
:1087B8004FF000021A7040F60433C2F20003FA7B4D
:1087C8001A704FF48040FEF789F80346002B2FD02B
:1087D80041F6CC63C2F20003DB881AB241F670039B
:1087E800C2F20003B3F81231194641F67003C2F21F
:1087F8000003B3F8DC30CB1A9A4219DD41F6CC639A
:10880800C2F20003DB881AB241F67003C2F2000319
:10881800B3F81231194641F67003C2F20003B3F8F7
:10882800DC30CB189A4203DA4FF001037B711AE06F
:108838004FF48040FEF752F8034683F00103DBB2A1
:10884800002B10D041F6CC63C2F20003DB881AB2C9
:1088580041F67003C2F20003B3F814319A4202DA07
:108868004FF001037B717B79002B28D001F078FE53
:1088780001F08AFE41F61843C2F20003B3F846300D
:10888800002B1CD041F68063C2F200031B78002B3A
:108898000CD041F66C63C2F200031B78002B05D0A4
:1088A800FFF74CFE0BE000BF7819002041F66C631F
:1088B800C2F200035B78002B01D001F02BFE40F6DA
:1088C8000533C2F200031B78142B40F0A98141F64E
:1088D8006C63C2F200035B78002B2DD041F618437D
:1088E800C2F20003B3F84630002B08D140F6043337
:1088F800C2F200031B785F2B01D101F00BFE41F699
:108908007003C2F2000393F81831002B00F088813D
:1089180041F61843C2F20003B3F84630002B40F08A
:108928007F8140F60433C2F200031B787D2B40F0B0
:10893800778101F0EFFD73E14FF00003BB6040F673
:108948000433C2F200031B78572B1ED14FF47A7000
:1089580000F03AFF4FF48070FDF7C0FF0346002B8C
:1089680001D005F0FDFB4FF0080007F025FD034698
:1089780083F00103DBB2002B50D041F63C53C2F226
:1089880000034FF000021A8048E04FF00400FDF7A2
:10899800A5FF0346002B41D040F60433C2F2000382
:1089A8001B785A2B3AD140F6FB23C2F200031B78FE
:1089B800002B0ED040F6FB23C2F200034FF000025A
:1089C8001A7040F6FC23C2F200034FF001021A703D
:1089D80024E040F6FA23C2F200031B78002B0CBFF8
:1089E80000230123DBB283F00103DBB203F00103B0
:1089F800DAB240F6FA23C2F200031A7040F6FA23FC
:108A0800C2F200031B78002B04D04FF00200FDF7E0
:108A180047F803E04FF00300FDF742F840F604334F
:108A2800C2F200031B785D2B03D14FF00103BB603A
:108A380014E040F60433C2F200031B785B2B03D129
:108A48004FF00203BB6009E040F60433C2F20003B2
:108A58001B785E2B02D14FF00303BB60BB68002B71
:108A680017D0BB68DBB203F1FF33DAB241F670030B
:108A7800C2F2000383F8A023FDF762FAFDF7E6F9D6
:108A8800BB68DBB24FF002004FF028011A460DF028
:108A9800F9F941F61843C2F20003B3F84630002B47
:108AA80009D140F60433C2F200031B786F2B02D1C0
:108AB800FFF744FD33E041F67003C2F2000393F878
:108AC8001831002B11D041F61843C2F20003B3F855
:108AD8004630002B09D140F60433C2F200031B785C
:108AE8007E2B02D1FFF72AFD19E040F60433C2F2CB
:108AF80000031B78972B04D14FF4C87000F090FB4B
:108B08000DE040F60433C2F200031B78A72B06D110
:108B180041F66C63C2F200034FF001029A734FF002
:108B28000003BB6040F60433C2F200031B78BB2B82
:108B380012D141F61843C2F200039B8D9BB203F198
:108B480002039BB29AB241F61843C2F200039A8517
:108B58004FF00103BB604CE040F60433C2F200035F
:108B68001B78B72B12D141F61843C2F200039B8D34
:108B78009BB2A3F102039BB29AB241F61843C2F228
:108B880000039A854FF00103BB6032E040F60433DE
:108B9800C2F200031B78BE2B12D141F61843C2F271
:108BA80000035B8D9BB203F102039BB29AB241F6BC
:108BB8001843C2F200035A854FF00103BB6018E066
:108BC80040F60433C2F200031B78BD2B11D141F6E5
:108BD8001843C2F200035B8D9BB2A3F102039BB260
:108BE8009AB241F61843C2F200035A854FF00103C6
:108BF800BB60BB68002B13D041F67003C2F20003C0
:108C080093F8A0331846FDF779F9FDF799F9FDF7C0
:108C180067F940F60533C2F200034FF000021A70FC
:108C28004FF00400FDF75AFE0346002B76D040F6BD
:108C3800FA23C2F200031B78002B29D041F66C639B
:108C4800C2F200035B78002B22D041F6CC63C2F25B
:108C58000003DB881AB241F67003C2F20003B3F8CE
:108C680014319A4214DD41F68063C2F200031B7886
:108C7800002B0DD140F6FE23C2F200034FF0320262
:108C88001A8040F6FA23C2F200034FF000021A706D
:108C980041F68063C2F200035B7C002B22D040F6D1
:108CA800FD23C2F200031B7883F00103DBB2002B23
:108CB80010D040F6FB23C2F200031B7883F00103B7
:108CC800DBB2002B06D040F6FE23C2F200034FF0C1
:108CD80032021A8040F6FD23C2F200034FF001026F
:108CE8001A701BE040F6FB23C2F200031B78002B2E
:108CF80014D041F66C63C2F200035B78002B0DD1EF
:108D080040F6FB23C2F200034FF000021A7040F64F
:108D1800FC23C2F200034FF001021A704FF0000367
:108D2800BB606EE0BB6803F1040241F6CC63C2F29B
:108D3800000333F812301AB240F213539A42CCBFF0
:108D480000230123DBB21946BA6813464FEA4303EE
:108D58009B1801FA03F398B2BB6803F1040241F6C9
:108D6800CC63C2F2000333F812301AB240F2145343
:108D78009A4210DDBB6803F1040241F6CC63C2F2EB
:108D8800000333F812301AB240F2A3639A4202DCAD
:108D98004FF0010201E04FF00002B9680B464FEABC
:108DA80043035B1803F1010302FA03F39BB2024683
:108DB800134399B2BB6803F1040241F6CC63C2F2D3
:108DC800000333F812301AB240F2A4639A42D4BFB7
:108DD80000230123DBB21846BA6813464FEA43035F
:108DE8009B1803F1020300FA03F39BB20A461343EC
:108DF8009AB2FB8813439BB2FB80BB6803F1010363
:108E0800BB60BB68032B8DDD4FF00003BB601EE029
:108E180041F61842C2F20002BB6803F120034FEA90
:108E28004303D318DA88FB8813409BB2002B0CBF8E
:108E380000230123DBB21A4641F68063C2F2000325
:108E4800B9685B181A70BB6803F10103BB60BB68A3
:108E5800142BDDDD41F68063C2F200035B78002B42
:108E680011D14FF40070FDF739FD0346002B22D0D5
:108E780041F21823C2F200031B681B68DB6898479D
:108E88000346002B17D04FF0020007F095FA03466F
:108E9800002B10D041F66C63C2F20003DB78002B84
:108EA80010D101F05DFB41F66C63C2F200034FF094
:108EB8000102DA7006E041F66C63C2F200034FF07B
:108EC8000002DA7041F68063C2F200039B78002B3F
:108ED80017D041F66C63C2F200034FF00002DA705B
:108EE80041F66C63C2F200031B79002B10D101F02C
:108EF80037FB41F66C63C2F200034FF001021A71AE
:108F080006E041F66C63C2F200034FF000021A71EA
:108F180041F68063C2F200031B78002B06D141F6AC
:108F28006C63C2F200034FF001021A7041F66C63E1
:108F3800C2F20003DB78002B06D141F66C63C2F263
:108F480000031B79002B07D04FF48053C4F60003AD
:108F58004FF488429A6106E04FF48053C4F6000348
:108F68004FF488421A854FF0200007F025FA03468F
:108F7800002B01D007F022F941F68063C2F200030A
:108F88001B7B002B07D041F66C63C2F200034FF045
:108F980001029A7206E041F66C63C2F200034FF0D8
:108FA80000029A7241F67003C2F200035B79082B43
:108FB80006D041F67003C2F200035B790E2B6DD127
:108FC80041F66C63C2F200034FF000025A7265E08A
:108FD80040F60833C2F200031B68042B61D801A2D3
:108FE80052F823F001900008199000083190000809
:108FF800499000087590000840F60833C2F2000353
:109008001B6803F1010240F60833C2F200031A603C
:1090180040F60833C2F200031B6803F1010240F670
:109028000833C2F200031A6040F60833C2F20003A4
:109038001B6803F1010240F60833C2F200031A600C
:1090480040F60833C2F200031B6803F1010240F640
:109058000833C2F200031A604FF48070FDF73EFC3B
:109068000346002B02D004F0E7FB1AE040F6083371
:10907800C2F200034FF000021A604FF40050FDF7EF
:109088002DFC0346002B0BD041F66C63C2F20003A3
:10909800DB7B002B04D0FFF789FA01E000BF00E07A
:1090A80000BF01F013F8024640F6F023C2F20003B5
:1090B8001A6041F67003C2F200039B89002B0DD0A1
:1090C80040F6F023C2F200031A6840F60C33C2F2ED
:1090D80000031B68D31A002BC0F2988041F6700376
:1090E800C2F200039B891A4640F6F023C2F200033D
:1090F8001B68D21840F60C33C2F200031A6001F064
:109108007FFEFEF73DFE00F0E1FF024640F6F02349
:10911800C2F200031A6040F6F023C2F200031B6893
:109128009AB240F6F423C2F200031B689BB2D31A2A
:109138009AB240F6F823C2F200031A8040F6F023F0
:10914800C2F200031A6840F6F423C2F200031A6060
:1091580041F61843C2F2000393F87630002B21D071
:1091680041F66C63C2F20003DB78002B06D141F6AE
:109178006C63C2F200031B79002B13D041F698638D
:10918800C2F20003DB889AB240F60C43C2F2000335
:109198001B889BB2D3189BB29AB241F69863C2F26D
:1091A8000003DA804FF0200007F006F90346002B91
:1091B80016D041F66C63C2F20003DB79002B06D1AE
:1091C80041F66C63C2F200031B7A002B08D041F60B
:1091D8006C63C2F200031B7B002B01D006F070FE0B
:1091E80040F22403C2F200031C6841F67003C2F285
:1091F8000003B3F8F630074807491A46074BA0475B
:1092080003F000FB03F016F803F008F907F1140760
:10921800BD4690BD191C0020371C0020421C0020B0
:1092280080B483B000AF0346FB8040F61A33C2F225
:109238000003FA881A8007F10C07BD4680BC704706
:1092480080B400AF40F61A33C2F200031B88002B2B
:1092580014BF00230123DBB21846BD4680BC70470B
:1092680080B400AF40F61A33C2F200031B88012B0A
:1092780014BF00230123DBB21846BD4680BC7047EB
:1092880080B400AF40F61A33C2F200031B88B3F56E
:10929800C87F14BF00230123DBB21846BD4680BC3B
:1092A800704700BF80B584B000AF78604FF000030E
:1092B800FB733BE0FFF7E4FF0346002B08D0FA7B83
:1092C80040F63433C2F200034FF0000143F8221095
:1092D800FA7BF97B40F63433C2F2000353F82110CD
:1092E800F87B41F65853C2F2000333F810301BB232
:1092F800C91840F63433C2F2000343F82210FA7B4F
:1093080041F65853C2F200034FF0000123F812103F
:1093180041F60853C2F200031B68FA7B4FF00001C4
:1093280023F81210FB7B03F10103FB73FB7B022B79
:10933800C0D9FFF795FF0346002B57D041F60853D5
:10934800C2F20003196840F63433C2F200031B6806
:1093580003F1C80248F21F53C5F2EB1383FB020363
:109368004FEAE3104FEAE273C31A9BB20B8041F64F
:109378000853C2F20003196840F63433C2F20003FE
:109388005B6803F1C80248F21F53C5F2EB1383FB75
:1093980002034FEAE3104FEAE273C31A9BB24B8011
:1093A80041F60853C2F20003196840F63433C2F29A
:1093B80000039B6803F1C80248F21F53C5F2EB1380
:1093C80083FB02034FEAE3104FEAE273C31A9AB22F
:1093D80040F22203C2F200031B88D31A9BB29BB24D
:1093E8008B80786801F0AAF8FDF768FA40F61A331E
:1093F800C2F200031B8803F1FF339AB240F61A3316
:10940800C2F200031A8007F11007BD4680BD00BFF5
:1094180080B584B000AF786040F6FE23C2F2000346
:109428001B88322B2ED141F60853C2F200031B6869
:109438001A8840F61C33C2F200031A8041F608531A
:10944800C2F200031B685A8840F61C33C2F20003BC
:109458005A8041F60853C2F200031B689A8840F606
:109468001C33C2F200039A807B681A8840F62433C2
:10947800C2F200031A807B685A8840F62433C2F28D
:1094880000035A8040F6FE23C2F200031B88002B1B
:1094980000F09A804FF00003FB733DE040F6FE2396
:1094A800C2F200031B88322B08D1FA7B40F628331E
:1094B800C2F200034FF0000143F82210FA7BF97B57
:1094C80040F62833C2F2000353F82110F87B41F626
:1094D8005853C2F2000333F810301BB2C91840F6D3
:1094E8002833C2F2000343F82210FA7B41F658539E
:1094F800C2F200034FF0000123F8121041F608539E
:10950800C2F200031B68FA7B4FF0000123F8121027
:10951800FB7B03F10103FB73FB7B022BBED940F6F7
:10952800FE23C2F200031B88012B40D140F6FD2325
:10953800C2F200034FF000021A7040F6FB23C2F299
:1095480000034FF001021A704FF00200FCF7A8FA6E
:1095580041F60853C2F200031A6840F61C33C2F2FF
:1095680000031B88138041F60853C2F200031A68EF
:1095780040F61C33C2F200035B88538041F608535F
:10958800C2F200031A6840F61C33C2F200039B883B
:10959800938040F62433C2F200031A887B681A804D
:1095A80040F62433C2F200035A887B685A8040F69A
:1095B800FE23C2F200031B8803F1FF339AB240F680
:1095C800FE23C2F200031A8040F6FC23C2F2000315
:1095D8001B78002B58D040F6FC23C2F200034FF052
:1095E80000021A7041F60853C2F20003196840F6E7
:1095F8002833C2F200031A6848F21F53C5F2EB136E
:1096080083FB02034FEA23104FEAE273C31A9BB2AB
:109618000B8041F60853C2F20003196840F628335C
:10962800C2F200035A6848F21F53C5F2EB1383FBDA
:1096380002034FEA23104FEAE273C31A9BB24B802E
:1096480041F60853C2F20003196840F62833C2F203
:1096580000039A6848F21F53C5F2EB1383FB020319
:109668004FEA23104FEAE273C31A9AB240F2220378
:10967800C2F200031B88D31A9BB29BB28B80786816
:1096880000F05CFFFDF71AF907F11007BD4680BD31
:1096980080B483B000AF786041F65853C2F200033B
:1096A8001B889AB27B681B889BB2D31A9BB29AB26A
:1096B80041F65853C2F200031A8041F65853C2F2D9
:1096C80000035B889AB27B685B889BB2D31A9BB213
:1096D8009AB241F65853C2F200035A8041F65853E1
:1096E800C2F200039B889AB27B689B889BB2D31A0C
:1096F8009BB29AB241F65853C2F200039A8007F11E
:109708000C07BD4680BC704780B582B000AF78605A
:1097180041F6FC43C2F200035B6841F65850C2F2BE
:109728000000984740F61933C2F200031B7841F64F
:109738005850C2F2000041F65851C2F200011A46D0
:10974800FBF724FFFFF77CFD034683F00103DBB240
:10975800002B02D07868FFF7A5FD4FF00400FDF755
:10976800BDF80346002B02D07868FFF751FE41F69A
:109778000853C2F200031B681846FFF789FF07F178
:109788000807BD4680BD00BF80B483B000AF7860D5
:1097980041F60853C2F200037A681A6007F10C0711
:1097A800BD4680BC704700BF80B483B000AF78600E
:1097B80040F64833C2F200037A681A6007F10C07D2
:1097C800BD4680BC704700BF80B483B000AF03467D
:1097D800FB8040F64633C2F20003FA881A8007F18C
:1097E8000C07BD4680BC704780B400AF40F64633D6
:1097F800C2F200031B88002B14BF00230123DBB235
:109808001846BD4680BC704780B400AF40F646336A
:10981800C2F200031B88012B14BF00230123DBB213
:109828001846BD4680BC704780B400AF40F646334A
:10983800C2F200031B88B3F57A7F14BF002301230B
:10984800DBB21846BD4680BC704700BF90B585B0F6
:1098580000AF0346FB714FF00003FB73BEE0FFF758
:10986800E3FF0346002B19D097F90F2040F6503339
:10987800C2F200034FF0000143F8221097F90F20BD
:1098880013464FEA83039B184FEA830340F65C3282
:10989800C2F200029B181846FDF7B0F897F90F209E
:1098A80097F90F1040F65033C2F2000353F8211015
:1098B80097F90F0041F64053C2F2000333F8103015
:1098C8001BB2C91840F65033C2F2000343F8221005
:1098D80097F90F2013464FEA83039B184FEA830337
:1098E80040F65C32C2F200029C1897F90F2041F64C
:1098F8004053C2F2000333F812301BB21846F7F790
:109908003DF9034620461946FDF786F897F90F20DA
:1099180041F64053C2F200034FF0000123F8121041
:1099280097F90F2040F61C43C2F200034FF00001E4
:1099380023F81210FFF768FF0346002B4AD097F967
:109948000F2013464FEA83039B184FEA830340F620
:109958005C32C2F200029B181846FDF7DFF8B860C7
:10996800FB79002B10D0FB791846F7F707F9034667
:109978001846B968F7F7F4FA0346002B04D04FF4F9
:109988007A70FFF721FF3BE097F90F1097F90F2046
:1099980040F65033C2F2000353F8223003F5FA724E
:1099A80044F6D353C1F2620383FB02034FEAA310C8
:1099B8004FEAE273C31A9AB240F61C43C2F200039C
:1099C80023F811204FF00A004FF00F014FF0010269
:1099D8000CF058FAFB7B03F10103FB7397F90F3086
:1099E800022B7FF73CAF40F64633C2F200031B88D8
:1099F80003F1FF339AB240F64633C2F200031A80ED
:109A080007F11407BD4690BD80B483B000AF4FF096
:109A18000003FB7120E097F9072097F9071041F63A
:109A28004053C2F2000333F8113099B297F9070096
:109A380040F61C43C2F2000333F810309BB2CB1A35
:109A48009BB299B241F64053C2F2000323F81210B8
:109A5800FB7903F10103FB7197F90730022BDADD7B
:109A680007F10C07BD4680BC704700BF80B500AF4A
:109A780041F61453C2F200035B6841F64050C2F24B
:109A88000000984740F64C33C2F200031B7841F6B9
:109A98004050C2F2000041F64051C2F200011A469D
:109AA800FBF774FDFFF7A0FE034683F00103DBB26A
:109AB800002B08D040F64833C2F200031B681B781D
:109AC8001846FFF7C3FEFFF79FFF80BD90B589B02A
:109AD80000AFF86079817A72FB804FF00003FB7762
:109AE8007B8941F6FC40C2F2000041F61451C2F2F3
:109AF80000011A46F7F752FD0346002B0AD04FF033
:109B08000103FB7740F64C33C2F200034FF0010229
:109B18001A703BE07B8941F61450C2F200001946E6
:109B2800F7F75CFF0346002B07D040F64C33C2F230
:109B380000034FF001021A7028E07B8941F61450A7
:109B4800C2F200001946F7F7EFFB0346002B07D0D7
:109B580040F64C33C2F200034FF001021A7015E0D0
:109B68007B8941F61450C2F200001946F8F768FAEA
:109B78000346002B07D040F64C33C2F200034FF0E7
:109B880000021A7002E04FF0000319E17B7A072BFC
:109B980077D801A151F823F0CB9B0008CB9B000894
:109BA800119C00088B9C00088B9C0008519C0008A5
:109BB8008B9C0008C19B00084FF0020006F028FCAF
:109BC8005FE04FF000033B754FF44873FB8207F1E9
:109BD8001403184641F6FC41C2F20001F7F756FAA1
:109BE8000346002B0DD040F61833C2F200034FF0A5
:109BF80001021A7040F61933C2F200034FF0040252
:109C08001A707B7A012B39D0FB7F002B1CD07B8903
:109C180041F6FC40C2F2000041F61451C2F20001C4
:109C28001A46F7F7BBFC40F61833C2F200034FF0B0
:109C380002021A7040F61933C2F200034FF0010213
:109C48001A707B7A022B1BD041F6FC40C2F200004E
:109C5800F8F798FA0346002B13D040F61833C2F2EF
:109C680000034FF005021A7040F61933C2F20003E0
:109C78004FF000021A707B7A052B02E000BF00E06B
:109C880000BF40F61833C2F200031B78002B0AD13C
:109C98007B7A002B03D04FF000037B7276E74FF0FE
:109CA800020006F0B5FBFB681B78002B06D0FB68AA
:109CB8001A7840F64C33C2F200031A70FB685B78DE
:109CC800002B06D0FB685A7840F61933C2F200031D
:109CD8001A70FB689B78002B06D0FB689A7840F6D0
:109CE8004433C2F200031A704FF0020006F064FB1E
:109CF8000346002B05D041F6FC43C2F200031B6863
:109D0800984741F61453C2F200031B6898474FF076
:109D1800080006F051FB0346002B48D0B7F906208F
:109D280048F21F53C5F2EB1383FB02134FEA63118A
:109D38004FEAE273CB1ABB83B7F9063048F21F52D9
:109D4800C5F2EB1282FB03124FEA62114FEAE3728B
:109D58008A1A4FF0640101FB02F29B1A7B83B7F960
:109D68001C301846F6F70AFF0446B7F91A301846A9
:109D7800F6F704FF0346184648F68901C3F68841FA
:109D8800F6F750FF034620461946F6F743FE03460A
:109D980018464FF00001C4F22011F6F743FF0346BE
:109DA8001A4640F61043C2F200031A6006E040F675
:109DB8001043C2F200034FF000021A604FF0010393
:109DC800184607F12407BD4690BD00BF80B584B092
:109DD80000AF7860396004E0FB7B7868194600F0D2
:109DE80013F83B681B78FB73FB7B002B0CBF00232D
:109DF8000123DBB23A6802F101023A60002BEBD191
:109E080007F11007BD4680BD80B582B000AF78600D
:109E18000B46FB707B681B681B68FA7878681146EC
:109E2800984707F10807BD4680BD00BF80B582B0DE
:109E380000AF78607B681B685B6878689847034662
:109E4800184607F10807BD4680BD00BF80B582B03F
:109E580000AF78607B681B689B6878689847034602
:109E6800184607F10807BD4680BD00BF80B582B01F
:109E780000AF786039607B681B68DB687868396890
:109E8800984707F10807BD4680BD00BF80B582B07E
:109E980000AF78607B681B681B6978689847034641
:109EA800184607F10807BD4680BD00BF80B582B0DF
:109EB80000AF78600B46FB707B681B685B69FA78BB
:109EC80078681146984707F10807BD4680BD00BF6E
:109ED80080B483B000AF0346FB71FB79002B07D039
:109EE8004FF48053C4F600034FF408521A8506E075
:109EF8004FF48053C4F600034FF408529A6107F1F7
:109F08000C07BD4680BC704780B483B000AF0346E1
:109F1800FB71FB79002B07D04FF48053C4F6000384
:109F28004FF408529A6106E04FF48053C4F60003D8
:109F38004FF408521A8507F10C07BD4680BC7047DC
:109F480080B582B000AF0346FB7140F69833C2F289
:109F580000031B68FA791046984707F10807BD46C1
:109F680080BD00BF80B400AF4FF001031846BD4666
:109F780080BC704780B500AFFFF7F4FF0346002BA5
:109F880009D040F69833C2F2000349F61172C0F6C0
:109F980000021A6008E040F69833C2F2000349F65E
:109FA800D962C0F600021A604FF00000FFF7C8FF40
:109FB80080BD00BF80B483B000AF03463960FB7139
:109FC80097F90730002B10DA4FF46D43CEF20003F7
:109FD800FA7902F00F02A2F104013A68D2B24FEA0C
:109FE8000212D2B25B181A760DE04FF46143CEF23A
:109FF800000397F907103A68D2B24FEA0212D2B2B8
:10A008005B1883F8002307F10C07BD4680BC704736
:10A0180080B582B000AF78607B6803F1FF326FF0E3
:10A028007F439A4202D94FF001031DE04EF210031C
:10A03800CEF200037A6802F1FF325A604FF0FF3027
:10A048004FF00F01FFF7B6FF4EF21003CEF20003F8
:10A058004FF000029A604EF21003CEF200034FF068
:10A0680007021A604FF00003184607F10807BD46BB
:10A0780080BD00BF80B594B000AF3B4618460CF0D9
:10A08800A9F93A684DF68363C4F21B33A3FB0213A4
:10A098004FEA934240F69C33C2F200031A6007F17C
:10A0A8005007BD4680BD00BF80B400AF40F6A03366
:10A0B800C2F200031B6803F1010240F6A033C2F2AA
:10A0C80000031A60BD4680BC704700BFB0B400AF43
:10A0D80040F6A033C2F200031C684EF21003CEF221
:10A0E80000039D6840F6A033C2F200031B689C423F
:10A0F800EED14FF47A7303FB04F240F69C33C2F2BC
:10A1080000031B684FF47A7101FB03F3591B40F6F7
:10A118009C33C2F200031B68B1FBF3F3D318184653
:10A12800BD46B0BC704700BF80B400AF40F6A03356
:10A13800C2F200031B681846BD4680BC704700BFCA
:10A14800B0B58CB000AF0346FB714BF64813C0F6B0
:10A15800010307F110041D460FCD0FC495E8030055
:10A1680084E803004FF0030387F82B300CF07AF8EB
:10A178004FF00700C0F242004FF001010CF000FD63
:10A188004FF4CD204FF001010CF0D0FC4FF001004E
:10A19800C1F23E004FF001010CF09EFC0CF06EFD88
:10A1A8004FF00303BB734FF6FF73BB8149F6FF7390
:10A1B800BB8107F10C034FF090401946F8F71EFDDC
:10A1C8004FF6FF73BB8107F10C034FF48060C4F6B0
:10A1D80000001946F8F712FD07F10C034FF4006070
:10A1E800C4F600001946F8F709FD4FF090404FF00B
:10A1F80008014FF006020BF071FF4FF48060C4F6BF
:10A2080000004FF008014FF001020BF067FF4FF418
:10A218008060C4F600004FF009014FF001020BF016
:10A228005DFF4FF40060C4F600004FF006014FF0E8
:10A2380004020BF053FF4FF40060C4F600004FF027
:10A2480007014FF004020BF049FF4FF40060C4F619
:10A2580000004FF008014FF004020BF03FFF4FF4ED
:10A268004060C4F600004FF00C014FF002020BF002
:10A2780035FF4FF44060C4F600004FF00D014FF079
:10A2880002020BF02BFF4FF44060C4F600004FF0C1
:10A298000E014FF002020BF021FF4FF44060C4F6AC
:10A2A80000004FF00F014FF002020BF017FF4FF0C4
:10A2B80090404FF001014FF001020BF00FFF4FF0FB
:10A2C80090404FF002014FF001020BF007FF4FF4EE
:10A2D8008060C4F600004FF000014FF002020BF05E
:10A2E800FDFE4FF48060C4F600004FF001014FF00E
:10A2F80002020BF0F3FE4FF090404FF004014FF0D4
:10A3080002020BF0EBFEFFF735FE4FF48053C4F664
:10A3180000034FF488521A854FF48053C4F60003A3
:10A328004FF488421A854FF00003FB6236E040F292
:10A338005413C2F200031A684FF4D853C0F2B7039B
:10A348009A4213D1FB6A4FEAC30307F13001CB18D5
:10A3580013F81A3C112B09D1FB6A4FEAC30307F122
:10A368003002D3184FF0010203F81A2CFB6A4FEAA7
:10A37800C30307F13001CB1853F8202C07F1100163
:10A38800FB6A4FEAC303CB1803F1040310461946CE
:10A39800F8F734FCFB6A03F10103FB6297F82B2002
:10A3A800FB6A9A42C3D8FFF765FE40F25813C2F21F
:10A3B80000031A6844F6D353C1F26203A3FB0213E5
:10A3C8004FEA93131846FFF723FE4FF4B040C4F248
:10A3D8000000F8F781F8F8F7EFFA4FF0640000F0A2
:10A3E80019F807F13007BD46B0BD00BF80B584B08D
:10A3F80000AF7860FFF76AFEF86000BFFFF766FEFF
:10A408000246FB68D21A7B689A42F7D307F1100715
:10A41800BD4680BD80B582B000AF786003E04FF4E0
:10A428007A70FFF7E3FF7B68002B0CBF0023012342
:10A43800DBB27A6802F1FF327A60002BEFD107F1C4
:10A448000807BD4680BD00BF80B582B000AF034697
:10A45800FB714FF48053C4F600034FF488429A61AD
:10A468004FF48053C4F600034FF488521A854FF412
:10A478008053C4F600034FF48052C4F60002928A57
:10A4880092B282F4884292B29A824FF48053C4F610
:10A4980000034FF48052C4F60002928A92B282F40A
:10A4A800885292B29A82FB7940F2DB1202FB03F3E4
:10A4B800A3F102031846FFF7ADFF4FF00100FFF7C5
:10A4C8003FFD4FF01900FFF7A5FF4FF00000FFF721
:10A4D80037FDCCE780B483B000AF0346FB71FB794E
:10A4E800002B08D044F6F073C2F200034BF6EF627B
:10A4F800CDF6AD621A604FF46D43CEF200034FF013
:10A508000402C0F2FA52DA6007F10C07BD4680BCBB
:10A51800704700BF80B400AF41F66C63C2F200031D
:10A528005B78002B06D041F66C63C2F200034FF053
:10A5380000025A70BD4680BC704700BF80B483B02B
:10A5480000AF78607B684FF000021A807B684FF09C
:10A5580000025A8007F10C07BD4680BC704700BF57
:10A5680080B400AF40F6B033C2F200034FF00002EF
:10A578001A6040F6B033C2F200034FF000025A608E
:10A58800BD4680BC704700BF80B400AF40F6A4331E
:10A59800C2F200034FF000021A6040F6A433C2F280
:10A5A80000034FF000025A6040F6A433C2F20003E1
:10A5B8004FF000029A60BD4680BC704780B592B0EB
:10A5C80000AFF860B9603B601346FB804FF00003B2
:10A5D800BB634FF000037B634FF000033B634FF016
:10A5E8000003FB6241F69863C2F200031B881BB2AA
:10A5F80083EAE372A2EBE37241F69863C2F20003C6
:10A608005B881BB2002BB8BF5B429A42A8BF1346B7
:10A61800BB624FF000037B64F9E141F66C63C2F260
:10A628000003DB78002B07D141F66C63C2F200030C
:10A638001B79002B00F082807B6C002B02D07B6C96
:10A64800012B7BD141F69863C2F200037A6C33F890
:10A6580012301BB24FEA430240F62453C2F2000301
:10A66800796C33F811301BB2D118FB88C3F10002A2
:10A67800FB88084611461A46FCF7A6F9024640F63A
:10A688002443C2F20003796C33F811301BB2D21A9A
:10A698003B68796C33F811301BB2D3187B62FB68C6
:10A6A800DB797A6A02FB03F248F21F53C5F2EB1317
:10A6B80083FB02134FEA63114FEAE273CB1ABB63C1
:10A6C800FB68DB7E1A4613464FEA83739B1A4FEAF0
:10A6D8008303991AFB68DB7E1A4613464FEA830305
:10A6E8009B18B86B1A46FCF76FF9B86340F6B0339D
:10A6F800C2F200037A6C53F822207B6AD3181846FA
:10A708004DF6F001CFF6FF7142F21072FCF75CF9DA
:10A71800014640F6B033C2F200037A6C43F82210C7
:10A7280040F6B033C2F200037A6C53F82230FA686C
:10A73800527C02FB03F34FEA23337B6341F66C63DD
:10A74800C2F20003DB78002B09D041F66C63C2F239
:10A7580000031B79002B02D17B6C022B77D141F6C9
:10A768009863C2F200037A6C33F812301AB21346B7
:10A778004FEA83039B184FEA03131A46F9687B6C68
:10A78800CB181B7892FBF3F33B6240F61443C2F2FA
:10A7980000037A6C33F812301BB23A6AD31A3B6260
:10A7A80041F69863C2F200037A6C33F812301BB298
:10A7B8003B6340F6A433C2F200037A6C53F82220BC
:10A7C8003B6AD31818464CF28011CFF6FF714FF44C
:10A7D8007A52FCF7F9F8014640F6A433C2F20003B6
:10A7E8007A6C43F8221040F61443C2F200037A6CE4
:10A7F80033F812301BB2002BB8BF5B42B3F5207F91
:10A8080008DD40F6A433C2F200037A6C4FF0000171
:10A8180043F8221040F6A433C2F200037A6C53F8CE
:10A82800222044F6D353C1F2620383FB02134FEA9A
:10A83800E3014FEAE273CB1AF9687A6C8A1802F1DD
:10A848000A02127802FB03F34FEAA313FB6241F6F4
:10A858006C63C2F200031B79002B34D07B6C002B95
:10A8680002D07B6C012B2ED1BB6AC3F5FA73BA6B8D
:10A8780002FB03F23B6BB96A01FB03F3D21844F6FF
:10A88800D353C1F2620383FB02134FEA63114FEA09
:10A89800E273CB1A3B64BB6AC3F5FA737A6B02FBAB
:10A8A80003F2FB6AB96A01FB03F3D21844F6D353E7
:10A8B800C1F2620383FB02134FEA63114FEAE273AA
:10A8C800CB1AFB6315E041F66C63C2F20003DB7838
:10A8D800002B0AD07B6C002B02D07B6C012B04D19F
:10A8E800BB6B3B647B6BFB6303E03B6B3B64FB6ACA
:10A8F800FB6340F61443C2F200037A6C33F812305B
:10A908001AB241F63853C2F20003796C5B181B780F
:10A9180003FB02F246F26763C6F2666383FB021327
:10A928004FEA63114FEAE273CB1A3A6CD31A3B64CD
:10A9380040F61443C2F200037A6C33F812301AB2AC
:10A9480040F6DC33C2F20003796C33F811301BB2E5
:10A95800D31AFB6140F61443C2F200037A6C33F851
:10A96800121040F6DC33C2F200037A6C23F812109E
:10A9780040F6E433C2F200037A6C53F8222040F622
:10A98800F033C2F20003796C53F82130D218FB6916
:10A99800D318BB6140F6E433C2F200037A6C53F873
:10A9A800221040F6F033C2F200037A6C43F822100A
:10A9B80040F6E433C2F200037A6CF96943F82210D6
:10A9C80041F63453C2F200037A6C9B181B78BA69BB
:10A9D80002FB03F3002B01DA03F11F034FEA6313B1
:10A9E8007B613B6C9AB2FB6B9BB2D3189AB27B69C2
:10A9F8009BB2D31A9BB299B241F62853C2F2000314
:10AA08007A6C23F812107B6C03F101037B647B6C76
:10AA1800022B7FF702AE07F14807BD4680BD00BF95
:10AA280080B58EB000AFF860B9603B601346FB801C
:10AA38004FF000037B634FF000033B634CE141F6AA
:10AA48006C63C2F20003DB78002B06D141F66C631D
:10AA5800C2F200031B79002B32D03B6B012B02D0D2
:10AA68003B6B002B2CD141F69863C2F200033A6B82
:10AA780033F812301BB24FEA430240F62453C2F2B5
:10AA88000003396B33F811301BB2D118FB88C3F1BE
:10AA98000002FB88084611461A46FBF795FF024656
:10AAA80040F62443C2F20003396B33F811301BB26D
:10AAB800D21A3B68396B33F811301BB2D3187B6359
:10AAC8003B6B022B0FD1BB685B7903F11B0241F68C
:10AAD8009863C2F200039B881BB203FB02F34FEAA0
:10AAE8006313FB6231E041F66C63C2F20003DB786A
:10AAF800002B22D1BB681B7903F11B0241F6986336
:10AB0800C2F20003396B33F811301BB203FB02F3B6
:10AB18004FEA2313FB6241F66C63C2F200031B7910
:10AB2800002B12D0FB685B7C7A6B02FB03F34FEAC5
:10AB38002323FA6AD318FB6207E0FB68DB797A6B98
:10AB480002FB03F34FEA2313FB6240F61443C2F2FD
:10AB580000033A6B33F812301BB2FA6AD31ABB629D
:10AB6800FA683B6BD3181B78BA6A02FB03F34FEA07
:10AB7800E3137B6240F6A433C2F200033A6B53F846
:10AB8800222040F6F823C2F200031B88B96A01FBB1
:10AB980003F34FEAE323F868396B411801F10A011E
:10ABA800097801FB03F3D11840F6A433C2F200037D
:10ABB8003A6B43F8221040F6A433C2F200033A6B12
:10ABC80053F8223018464FF00001CFF6E0714FF4E9
:10ABD8000012FBF7F9FE014640F6A433C2F2000367
:10ABE8003A6B43F8221040F6A433C2F200033A6BE2
:10ABF80053F822304FEA63333B6240F6B833C2F26F
:10AC080000033A6B53F82230BA6AD31AFB6140F654
:10AC1800B833C2F200033A6BB96A43F8221040F61F
:10AC2800F823C2F200031B884FEA13139BB24FF6B6
:10AC3800FF72B2FBF3F39BB2FA6902FB03F34FEA2C
:10AC4800A313FB6140F6C433C2F200033A6B53F816
:10AC5800222040F6D033C2F20003396B53F821307A
:10AC6800D218FB69D318BB6140F6C433C2F20003A3
:10AC78003A6B53F8221040F6D033C2F200033A6B15
:10AC880043F8221040F6C433C2F200033A6BF96964
:10AC980043F82210FA683B6BD31803F114031B78AE
:10ACA800BA6902FB03F34FEA23237B617B6A9AB2FA
:10ACB8003B6A9BB2D3189AB27B699BB2D3189BB2FA
:10ACC80099B241F62853C2F200033A6B23F81210E6
:10ACD8003B6B03F101033B633B6B022B7FF7AFAE8A
:10ACE80007F13807BD4680BD80B483B000AF7860F7
:10ACF8007B68012B09D040F22403C2F200034AF218
:10AD0800C552C0F600021A6009E040F22403C2F2FC
:10AD180000034AF62922C0F600021A6000BF07F1B4
:10AD28000C07BD4680BC704780B500AF40F22203D7
:10AD3800C2F200031B881846F5F720FF03461846A1
:10AD480040F2C931C3F66871F5F76CFF034618463F
:10AD58000DF0B8FD03469AB240F60443C2F2000370
:10AD68001A8040F22203C2F200031B881846F5F746
:10AD780005FF03464EF60A00C4F21C101946F6F702
:10AD880005F8034618464FF48041C4F21C61F5F7F4
:10AD9800FDFF03461A4641F65453C2F200031A60F7
:10ADA80041F61843C2F20003B3F874301846F5F7B9
:10ADB800E5FE03464FF00000C4F261401946F5F77E
:10ADC800E5FF03461846F5F769FB02460B461046B1
:10ADD800194609A3D3E90023F5F7B4FB02460B464D
:10ADE80010461946F5F7C0FD024641F67053C2F207
:10ADF80000031A6080BD00BF3B597E90A9E78140DF
:10AE080080B582B000AFFEF731FE4FF0020005F0CA
:10AE1800D3FA0346002B05D03D48FEF775FC00F039
:10AE280037FC14E041F65853C2F200034FF0000219
:10AE38001A8041F65853C2F200034FF000025A80BC
:10AE480041F65853C2F200034FF000029A8041F6CF
:10AE58007003C2F200035B79012B3CD140F65443E6
:10AE6800C2F200031B881BB24FEA430241F640536B
:10AE7800C2F200039B881BB2D21845F25653C5F2A2
:10AE8800555383FB02014FEAE273CB1A9AB240F69C
:10AE98001443C2F200039A8040F61443C2F200033E
:10AEA8009A8840F65443C2F200031A8041F6405390
:10AEB800C2F200031A8840F61443C2F200031A8053
:10AEC80041F64053C2F200035A8840F61443C2F2D6
:10AED80000035A8018E04FF000037B6011E041F650
:10AEE8004053C2F200037A6833F8121040F6144354
:10AEF800C2F200037A6823F812107B6803F1010399
:10AF08007B607B68022BEAD907F10807BD4680BD44
:10AF1800421C002090B585B000AF786039607B682E
:10AF28001A687B681B6810461946F5F77BFE0346CE
:10AF38001C467B685A687B685B6810461946F5F7BB
:10AF480071FE034620461946F5F764FD03461C4684
:10AF58007B689A687B689B6810461946F5F762FE1D
:10AF6800034620461946F5F755FD034618460DF0E9
:10AF780077FDF860F8684FF00001F5F7E7FF034642
:10AF8800002B1DD17B681B681846F968F5F7FEFE93
:10AF980003461A463B681A607B685B681846F9687E
:10AFA800F5F7F4FE03461A463B685A607B689B68CF
:10AFB8001846F968F5F7EAFE03461A463B689A60B0
:10AFC80007F11407BD4690BD90B59BB000AF7860FF
:10AFD80039607A6807F1300307CA83E807003B68DD
:10AFE8001B6818460DF03AFC78663B681B681846E3
:10AFF8000DF0A8FC38663B685B6818460DF02EFC1F
:10B00800F8653B685B6818460DF09CFCB8653B68C2
:10B018009B6818460DF022FC78653B689B681846CB
:10B028000DF090FC3865786D796EF5F7FBFD0346F9
:10B03800FB64786DF96DF5F7F5FD0346BB64386D73
:10B04800796EF5F7EFFD03467B64386E796DF5F799
:10B05800E9FD03463B64386E396DF5F7E3FD0346B9
:10B06800FB63BB6CFB60FB6D83F000431846396DD6
:10B07800F5F7D8FD03463B61BB6D7B61386CB96D54
:10B08800F5F7D0FD03461846796CF5F7C3FC03467F
:10B09800BB61F86BB96DF5F7C5FD0346F86C194649
:10B0A800F5F7B6FC0346FB613B6E83F00043184698
:10B0B800F96DF5F7B7FD03463B62F86CB96DF5F726
:10B0C800B1FD0346F86B1946F5F7A2FC03467B620F
:10B0D800786CB96DF5F7A6FD03461846396CF5F797
:10B0E80099FC0346BB62F86D796EF5F79BFD034644
:10B0F800FB623A6BFB6810461946F5F793FD034669
:10B108001C467A6BBB6910461946F5F78BFD03465A
:10B1180020461946F5F77EFC03461C46BA6B7B6A47
:10B1280010461946F5F77EFD034620461946F5F701
:10B1380071FC03461A467B681A603A6B3B691046F5
:10B148001946F5F76FFD03461C467A6BFB691046F6
:10B158001946F5F767FD034620461946F5F75AFCE8
:10B1680003461C46BA6BBB6A10461946F5F75AFDEA
:10B17800034620461946F5F74DFC03461A467B68F8
:10B188005A603A6B7B6910461946F5F74BFD034642
:10B198001C467A6B3B6A10461946F5F743FD034691
:10B1A80020461946F5F736FC03461C46BA6BFB6A7F
:10B1B80010461946F5F736FD034620461946F5F7B9
:10B1C80029FC03461A467B689A6007F16C07BD465E
:10B1D80090BD00BF80B483B000AF786039607B68F1
:10B1E80083EAE372A2EBE3723B689A4203DA4FF018
:10B1F80000037B600EE07B68002B04DD7A683B6807
:10B20800D31A7B6006E07B68002B03DA7A683B6818
:10B21800D3187B607B68184607F10C07BD4680BCD5
:10B22800704700BF0000000090B589B000AF78609B
:10B2380040F62843C2F200031B6883F000437B6199
:10B2480040F62843C2F200035B6883F00043BB6109
:10B2580041F63C53C2F200031B881BB21846F5F7AF
:10B268008DFC034683F000431846F5F717F90246AC
:10B278000B4610461946A2A3D3E90023F5F762F955
:10B2880002460B4610461946F5F76EFB0346FB616E
:10B2980041F66853C2F200031B881BB21846F5F743
:10B2A8006DFC0346BB6041F66853C2F200035B883D
:10B2B8001BB21846F5F762FC0346FB6041F668537B
:10B2C800C2F200039B881BB21846F5F757FC0346E9
:10B2D8003B6107F1080207F1140310461946FFF70E
:10B2E80073FE41F61843C2F2000393F84430012B71
:10B2F8004BD141F66C63C2F200035B78002B2DD171
:10B3080040F64C43C2F200031A6840F64C43C2F2BE
:10B3180000031B68002B01DA03F13F034FEAA31374
:10B32800D21A40F64C43C2F200031A6040F64C436E
:10B33800C2F200031B681846F5F720FC02463B6979
:10B3480010461946F5F766FB03461846F5F730FE32
:10B35800024640F64C43C2F200031A603C6940F6CC
:10B368004C43C2F200031B68002B01DA03F13F03D0
:10B378004FEAA3131846F5F701FC03462046194681
:10B38800F5F746FB03463B610FE03C6940F22203B8
:10B39800C2F200031B881846F5F7F0FB0346204667
:10B3A8001946F5F735FB03463B617868F5F7E2FB8C
:10B3B80004467868F5F7DEFB02464CF6CC43C0F647
:10B3C80001031B6810461946F5F724FB034620467F
:10B3D8001946F5F7DBFC03461C463A6940F650432C
:10B3E800C2F200031B6810461946F5F711FB034625
:10B3F80020461946F5F716FC03461A4640F6504310
:10B40800C2F200031B6810461946F5F703FB034612
:10B418001A4640F65043C2F200031A6041F64853F8
:10B42800C2F200031C68BB6818460DF04BFA0246CE
:10B4380041F61843C2F2000393F83030104619461B
:10B44800FFF7C8FE0346E21841F64853C2F200036C
:10B458001A6041F64853C2F200035C68FB6818465C
:10B468000DF030FA024641F61843C2F2000393F891
:10B47800303010461946FFF7ADFE0346E21841F694
:10B488004853C2F200035A6041F64853C2F200031F
:10B498009C6840F65043C2F200031B6818460DF042
:10B4A80011FA024641F61843C2F2000393F82F300E
:10B4B80010461946FFF78EFE0346E21841F6485338
:10B4C800C2F200039A6040F6FC33C2F200031A6825
:10B4D8007B68D21840F6FC33C2F200031A6040F6CB
:10B4E8000043C2F200031B6803F1010240F6004367
:10B4F800C2F200031A6007F12407BD4690BD00BFE1
:10B50800399D52A246DF913FB0B58AB000AF78604E
:10B5180040F62843C2F200031B6818460DF09EF956
:10B52800386240F62843C2F200031B6818460DF043
:10B5380009FAF86140F62843C2F200035B6818462E
:10B548000DF08CF9B86140F62843C2F200035B683D
:10B5580018460DF0F7F978617B681B681846B969D9
:10B56800F5F760FB03461C467B685B681846F9697B
:10B57800F5F758FB034618467969F5F753FB034678
:10B5880020461946F5F746FA03461C467B689B6831
:10B5980018467969F5F746FB03461846396AF5F700
:10B5A80041FB034620461946F5F734FA03463B614A
:10B5B8007B685B681846396AF5F734FB03461C4616
:10B5C8007B689B681846F969F5F72CFB034620460B
:10B5D8001946F5F71DFA0346FB60F86839690DF05E
:10B5E8003DFA034618464FF00001C4F2E141F5F771
:10B5F80019FB03461846F4F751FF02460B4610465E
:10B60800194621A3D3E90023F5F7C6F802460B46ED
:10B6180014461D4640F61043C2F200031B68184644
:10B62800F4F73CFF02460B4620462946F4F7D8FDBE
:10B6380002460B46104619464FF000024FF0000331
:10B64800C4F22403F5F7A8F802460B46104619463B
:10B65800F5F78AF90346BB60B8680DF033F903467D
:10B66800FB84B7F92630002B04DAFB8C03F5B4739E
:10B678009BB2FB84FB8C1BB2184607F12807BD461A
:10B68800B0BD00BFAFF30080182D4454FB21094022
:10B69800B0B58CB000AF4FF00003BB62FEF716FDEB
:10B6A800386240F63043C2F200031B683A6AD31A84
:10B6B800FB61F869F5F75EFA024641F61453C2F2E7
:10B6C8000003DB6810461946F5F7ACFA0346BB6180
:10B6D80040F63043C2F200033A6A1A604FF00003A2
:10B6E800FB62ADE041F64053C2F20003FA6A33F858
:10B6F80012301BB21846F5F741FA03461846B969E5
:10B70800F5F790FA03461A46FB6A4FEA830307F1F6
:10B718003001CB1843F8302C41F61843C2F200032D
:10B7280093F82E30002B64D040F63443C2F2000365
:10B73800FA6A53F8224041F61843C2F2000393F81C
:10B748002E301846F5F71AFA03464FF07E50194680
:10B75800F5F71CFB03464FF07E501946F5F758F9EC
:10B76800034620461946F5F75DFA03461C4641F69E
:10B778005853C2F20003FA6A33F812301BB2184663
:10B78800F5F7FCF9054641F61843C2F2000393F8B1
:10B798002E301846F5F7F2F903464FF07E50194659
:10B7A800F5F7F4FA034628461946F5F73BFA034637
:10B7B80020461946F5F72EF90346194640F6344354
:10B7C800C2F20003FA6A43F8221040F63443C2F288
:10B7D8000003FA6A53F822301846F5F7E9FB0346E6
:10B7E80099B241F66853C2F20003FA6A23F81210BC
:10B7F8000DE041F65853C2F20003FA6A33F812100A
:10B8080041F66853C2F20003FA6A23F8121041F6AF
:10B818006853C2F20003FA6A33F812301AB241F6DA
:10B828006853C2F20003F96A33F811301BB203FB04
:10B8380002F3BA6AD318BB62FB6A03F10103FB6225
:10B84800FB6A022B7FF74EAFBB6A4FF0640202FB24
:10B8580003F240F22203C2F200031B88194640F2A9
:10B868002203C2F200031B8803FB01F392FBF3F3EC
:10B87800BB623B4641F67450C2F200001946FFF71E
:10B88800A3FB4FF0080004F097FD0346002B08D0F7
:10B898003B4640F64040C2F200001946FFF794FBD1
:10B8A80011E03B4640F22800C2F200001946FFF7BB
:10B8B8008BFB40F22800C2F2000040F22801C2F2DD
:10B8C8000001FFF727FB41F67003C2F20003B3F84B
:10B8D800F0301846F5F74EF9034618464FF07E51FA
:10B8E800F5F798F803464FF07E501946F5F74EFAEB
:10B8F80003467B61BB6A9BB2482B43D9BB6A9BB2A8
:10B90800842B3FD84FF00003FB6238E041F67453B4
:10B91800C2F20003FA6A53F8224041F67003C2F2F9
:10B928000003B3F8F0301846F5F724F9034620462B
:10B938001946F5F777F903461C4641F66853C2F2F3
:10B948000003FA6A33F812301BB21846F5F716F9F5
:10B95800034620461946F5F75DF803461846796907
:10B96800F5F760F90346194641F67453C2F200032D
:10B97800FA6A43F82210FB6A03F10103FB62FB6ACF
:10B98800022BC3DD41F67003C2F20003B3F8F230B4
:10B998001846F5F7EFF8034618464FF07E51F5F7CD
:10B9A80039F803464FF07E501946F5F7EFF903468C
:10B9B8003B614FF0080004F0FFFC0346002B3FD02A
:10B9C8004FF00003FB6238E040F64043C2F2000348
:10B9D800FA6A53F8224041F67003C2F20003B3F842
:10B9E800F2301846F5F7C6F8034620461946F5F72B
:10B9F80019F903461C4641F60C53C2F20003FA6AD1
:10BA080033F812301BB21846F5F7B8F8034620464B
:10BA18001946F4F7FFFF034618463969F5F702F9A6
:10BA28000346194640F64043C2F20003FA6A43F857
:10BA38002210FB6A03F10103FB62FB6A022BC3DDE0
:10BA480041F67453C2F200039D6840F60443C2F203
:10BA580000031B881BB21846F5F790F803464FF011
:10BA68000102144628461946F5F798FA0346002BB2
:10BA780002D14FF000031C46E3B21A4641F66C634C
:10BA8800C2F200035A7341F67453C2F200035A68B3
:10BA980041F67453C2F200039B68104619460CF035
:10BAA800DDFF024640F62843C2F200031A6041F661
:10BAB8007453C2F200031B6883F0004441F67453C8
:10BAC800C2F200035A6841F67453C2F200035B687D
:10BAD80010461946F5F7A6F803461D4641F6745375
:10BAE800C2F200039A6841F67453C2F200039B68DD
:10BAF80010461946F5F796F8034628461946F4F70E
:10BB080089FF034618460CF0ABFF0346204619464A
:10BB18000CF0A4FF024640F62843C2F200035A6024
:10BB280040F62843C2F200031B681846F4F7B6FC37
:10BB380002460B461046194687A3D3E90023F4F7BB
:10BB480001FD02460B4610461946F4F70DFF034661
:10BB580018460CF0B7FE03469AB240F62443C2F2E8
:10BB680000031A8040F62843C2F200035B681846B7
:10BB7800F4F794FC02460B461046194676A3D3E91F
:10BB88000023F4F7DFFC02460B4610461946F4F78B
:10BB9800EBFE034618460CF095FE03469AB240F6B3
:10BBA8002443C2F200035A804FF0080004F004FC5A
:10BBB8000346002B0DD040F64040C2F20000FFF7CC
:10BBC800A3FC03461A4641F63C53C2F200031A800E
:10BBD8000CE040F22800C2F20000FFF795FC034693
:10BBE8001A4641F63C53C2F200031A80F869FFF77F
:10BBF8001BFB41F61843C2F2000393F87630002B82
:10BC080000F0A38041F67453C2F200039C6841F629
:10BC18007453C2F200031A6841F67453C2F2000367
:10BC28001B6810461946F4F7FDFF03461D4641F60A
:10BC38007453C2F200035A6841F67453C2F2000307
:10BC48005B6810461946F4F7EDFF03462846194687
:10BC5800F4F7E0FE03461D4641F67453C2F20003B2
:10BC68009A6841F67453C2F200039B68104619465D
:10BC7800F4F7D8FF034628461946F4F7CBFE0346E7
:10BC880018460CF0EDFE034620461946F5F77EF8F7
:10BC98000346FB60F8684CF28F21C3F67541F5F74F
:10BCA80069F90346002B07D040F60C43C2F20003A3
:10BCB8004FF000021A8048E0F8680CF07FFE024658
:10BCC80041F67053C2F200031B6810461946F4F798
:10BCD800A9FF034618460CF0F5FD78627B6AB3F5B8
:10BCE800617F02DD4FF461737B6241F61843C2F253
:10BCF800000393F876301846F4F740FF0446786A54
:10BD0800F4F7BAFB02460B461046194614A3D3E9CA
:10BD18000023F4F741FD02460B4610461946F4F796
:10BD280023FE034618460CF00DFE0346204619462E
:10BD3800F4F778FF034618460CF0C4FD03469AB2A0
:10BD480040F60C43C2F200031A8007F13007BD46E3
:10BD5800B0BD00BFAFF300803B597E90A9E781409A
:10BD6800A2EB0FE5DD16964080B485B000AFF86011
:10BD7800B9607A603B6041F69853C2F20003FA68F2
:10BD88001A6041F69053C2F20003BA681A6041F68D
:10BD98008453C2F200037A681A6041F68853C2F2EB
:10BDA80000033A681A6041F68053C2F20003BA6988
:10BDB8001A6041F69453C2F20003FA691A6041F618
:10BDC8008C53C2F200033A6A1A6007F11407BD46A1
:10BDD80080BC704780B485B000AF786041F6985356
:10BDE800C2F200031A687B684FEAC303D318DB79F1
:10BDF800FB73FB7BFF2B0CD0FB7B4FEA8343002BB1
:10BE080007D0FA7B41F6CC63C2F2000333F8123054
:10BE18000FE07B68072B0ADC41F69853C2F2000357
:10BE28001A687B684FEAC303D3189B8801E040F285
:10BE3800DC531BB2184607F11407BD4680BC704797
:10BE480080B483B000AF7860396041F69853C2F28D
:10BE580000031A687B684FEAC303D3189B795AB268
:10BE68003B681340002B02D04FF0FF3301E04FF046
:10BE78000103184607F10C07BD4680BC704700BF98
:10BE880090B585B000AF03463960FB7140F61C538E
:10BE9800C2F20003FA791A70FB794DF24012C0F62B
:10BEA80001024FEAC303D3185B781A4640F6584399
:10BEB800C2F200031A604FF02000FAF70FFD0346A4
:10BEC800002B06D040F65843C2F200034FF001029F
:10BED8001A60FB79162B38D14FF00003FB6030E075
:10BEE800FB684FEA03133A68D3181B6818464FF0EB
:10BEF8000001F5F72BF80346002B69D1FB684FEAE0
:10BF080003133A68D21840F65C43C2F20003F9689A
:10BF18004FEA01115B181C4613460FCB84E80F004B
:10BF280040F65643C2F200031B7803F10103DAB26C
:10BF380040F65643C2F200031A70FB6803F101038E
:10BF4800FB60FB680B2BCBDD43E0FA794DF2401325
:10BF5800C0F6010313F8322040F65643C2F200033C
:10BF68001A70FB794DF24012C0F601024FEAC30382
:10BF7800D3185B68002B2CD04FF00003FB601DE04A
:10BF8800FB794DF24012C0F601024FEAC303D31801
:10BF98005A68FB684FEA0313D21840F65C43C2F2B2
:10BFA8000003F9684FEA01115B181C4613460FCBD2
:10BFB80084E80F00FB6803F10103FB6040F6564379
:10BFC800C2F200031B781A46FB689A42D8DC00E0EC
:10BFD80000BF4FF48040FAF781FC0346002B6ED077
:10BFE80040F65643C2F200031B78012B67D94FF085
:10BFF8000003FB605AE040F65C43C2F20003FA68B3
:10C008004FEA02129B1803F108031B6818464FF009
:10C018007C51F4F707FE03461A4640F65C43C2F229
:10C028000003F9684FEA01115B1803F108031A606D
:10C0380040F65C43C2F20003FA684FEA02129B180A
:10C0480003F104031B6818464FF07C51F4F7EAFD2E
:10C0580003461A4640F65C43C2F20003F9684FEA09
:10C0680001115B1803F104031A6040F65C43C2F245
:10C078000003FA684FEA02129B1803F10C031B68CD
:10C0880018464FF07C51F4F7CDFD03461A4640F6AA
:10C098005C43C2F20003F9684FEA01115B1803F12F
:10C0A8000C031A60FB6803F10103FB6040F656437A
:10C0B800C2F200031B781A46FB689A429BDCFB79A4
:10C0C800082B02D0FB790E2B07D141F66C63C2F224
:10C0D80000034FF001021A7406E041F66C63C2F2E5
:10C0E80000034FF000021A7400F004F807F1140777
:10C0F800BD4690BD80B582B000AF4FF000037B60B5
:10C1080020E04FF48040FAF7E9FB0346002B07D004
:10C1180041F69053C2F200031B689B889AB206E06E
:10C1280041F68453C2F200031B689B889AB241F619
:10C13800B453C2F20003796823F811207B6803F135
:10C1480001037B607B680B2BDBDD07F10807BD462D
:10C1580080BD00BF90B484B000AF786039607B6860
:10C1680003F101037B604FF00003FB600BE0FB6809
:10C178004FEA03133A68D3184FF000021A60FB68BD
:10C1880003F10103FB60FB680B2BF0DD4DF240125D
:10C19800C0F601027B684FEAC303D3185B68002B23
:10C1A80028D04FF00003FB6019E0FB684FEA031347
:10C1B8003A68D1184DF24012C0F601027B684FEA86
:10C1C800C303D3185A68FB684FEA0313D3180C4605
:10C1D8000FCB84E80F00FB6803F10103FB604DF20D
:10C1E8004013C0F601037A6813F832301A46FB6828
:10C1F8009A42DADC07F11007BD4690BC704700BFD1
:10C2080080B500AF40F23403C2F200031B889BB232
:10C218004FF000001946F6F7E9FF40F23403C2F286
:10C2280000035B889BB24FF001001946F6F7DEFF6A
:10C2380080BD00BF80B500AF40F65843C2F200038E
:10C248001B68002B00F0E58040F61C53C2F2000387
:10C258001B7803F1FF33142B00F2D18001A252F8AE
:10C2680023F000BFEFC2000807C4000807C4000895
:10C27800C1C2000879C3000807C4000807C4000841
:10C288004BC3000807C4000807C4000807C4000817
:10C2980007C4000807C40008ADC3000807C40008A5
:10C2A80007C4000807C4000807C4000807C400083A
:10C2B8007FC30008ADC3000840F23403C2F2000394
:10C2C8001B899BB24FF000001946F6F78FFF40F22A
:10C2D8003403C2F200035B899BB24FF00100194698
:10C2E800F6F784FF98E041F68853C2F200031B6812
:10C2F8005B78002B0BD040F23403C2F200035B8959
:10C308009BB24FF000001946F6F770FF84E041F643
:10C318006C63C2F200035B78002B0BD040F234034D
:10C32800C2F200035B899BB24FF000001946F6F792
:10C338005DFF71E04FF000004FF00001F6F756FF87
:10C348006AE040F23403C2F20003DB889BB24FF08C
:10C3580000001946F6F74AFF40F23403C2F2000320
:10C368001B899BB24FF001001946F6F73FFF53E0D7
:10C37800FFF746FF50E040F23403C2F200031B8986
:10C388009BB24FF000001946F6F730FF40F2340335
:10C39800C2F200035B899BB24FF001001946F6F721
:10C3A80025FF39E040F23403C2F20003DB889BB278
:10C3B8004FF000001946F6F719FF40F23403C2F2B5
:10C3C80000031B899BB24FF001001946F6F70EFFD8
:10C3D80040F23403C2F200035B899BB24FF00200C3
:10C3E8001946F6F703FF40F23403C2F200039B89B3
:10C3F8009BB24FF003001946F6F7F8FE0CE04FF039
:10C408002000FAF76BFA0346002B04D0FFF7F8FE7A
:10C4180001E000BF00E000BF80BD00BF80B582B072
:10C4280000AF4FF00003FB7110E0FA7941F69C531E
:10C43800C2F2000333F812309BB2FA79104619465B
:10C44800F6F7B0FEFB7903F10103FB7140F65643A2
:10C45800C2F200031B78FA799A42E6D307F108077B
:10C46800BD4680BD80B584B000AF0346FB804FF069
:10C478000003FB730BE0FA7B41F69C53C2F2000306
:10C48800F98823F81210FB7B03F10103FB7340F6D4
:10C498005643C2F200031B78FA7B9A42EBD3FFF7AC
:10C4A800BDFF07F11007BD4680BD00BF90B585B040
:10C4B80000AF4FF00003BB804FF00003FB8041F654
:10C4C8006C63C2F200035B78002B0CD141F68453F5
:10C4D800C2F200031B689B889AB240F23403C2F28E
:10C4E8000003DA811EE041F69863C2F20003DB889C
:10C4F80019B241F68453C2F200031B681B881A461E
:10C5080041F68453C2F200031B685B880846114653
:10C518001A46FAF759FA03469AB240F23403C2F2BD
:10C528000003DA8140F23403C2F20003DA8941F6EB
:10C538009C53C2F200031A8041F68053C2F20003F2
:10C548001B681B78002B00F09F804FF00200FFF75C
:10C5580041FC03467B81B7F90A1041F69853C2F2B1
:10C5680000031B6803F110031B881AB241F69853A5
:10C57800C2F200031B6803F110035B881BB2084674
:10C5880011461A46FAF720FA03467B8141F694537E
:10C59800C2F200031B685A897B89D31A9BB27B813C
:10C5A80040F61E53C2F200031B88B7F90A201BB2DB
:10C5B8009A4215DD41F68053C2F200031B681B78CE
:10C5C8001A4640F61E53C2F200031B889BB2D318CA
:10C5D8009BB29AB240F61E53C2F200031A801DE0C5
:10C5E80040F61E53C2F200031B88B7F90A201BB29B
:10C5F8009A4213DA40F61E53C2F200031B889AB21D
:10C6080041F68053C2F200031B681B78D31A9BB211
:10C618009AB240F61E53C2F200031A8041F69853AC
:10C62800C2F200031B6803F110039B795AB240F66B
:10C638001E53C2F200031B881BB203FB02F248F22E
:10C648001F53C5F2EB1383FB02134FEA63114FEA42
:10C65800E273CB1A9AB240F23403C2F200039A8012
:10C6680040F23403C2F200039B889AB241F6945315
:10C67800C2F200031B685B89D3189BB29AB240F2DE
:10C688003403C2F200039A8041F66C63C2F20003DD
:10C698009B7A002B34D041F69863C2F200031B88C2
:10C6A8009AB2BB889BB2D3189BB29AB240F23403B9
:10C6B800C2F20003DA8041F69863C2F200031B88D5
:10C6C8009AB2FB889BB2D3189BB29AB240F2340359
:10C6D800C2F200031A8141F69863C2F200039A88F5
:10C6E80040F23403C2F200035A8141F69863C2F261
:10C6F80000035A8840F23403C2F200039A8133E0FF
:10C7080041F62853C2F200031B889AB2BB889BB239
:10C71800D3189BB29AB240F23403C2F20003DA8013
:10C7280041F62853C2F200031B889AB2FB889BB2D9
:10C73800D3189BB29AB240F23403C2F200031A81B2
:10C7480041F62853C2F200039A8840F23403C2F239
:10C7580000035A8141F62853C2F200035A8840F276
:10C768003403C2F200039A814FF00303FB6042E0F6
:10C7780041F69853C2F200031A68FB684FEAC303F4
:10C78800D3189B795AB240F23403C2F20003F96815
:10C7980033F811301BB203FB02F248F21F53C5F203
:10C7A800EB1383FB02134FEA63114FEAE273CB1AD0
:10C7B80099B240F23403C2F20003FA6823F8121067
:10C7C80040F23403C2F20003FA6833F812309CB224
:10C7D800F868FFF7FFFA03469BB2E3189BB299B2D9
:10C7E80040F23403C2F20003FA6823F81210FB681F
:10C7F80003F10103FB60FB68062BB9DD07F11407A1
:10C80800BD4690BDB0B584B000AF40F65643C2F205
:10C8180000031B78032B2AD941F62853C2F20003E0
:10C828009B8819B241F69863C2F200039B881BB239
:10C8380083EAE372A2EBE3724FF69C73CFF6FF73C1
:10C848009B1A41F69862C2F20002928812B2002A3C
:10C85800B8BF524202F1640208461946FAF7B4F822
:10C8680003469AB241F62853C2F200039A8040F672
:10C878005643C2F200031B78012B40F2A1804FF00F
:10C888000003BB6092E041F69863C2F20003DB88C4
:10C898001BB21846F4F772F9024640F65C43C2F23E
:10C8A8000003B9684FEA01115B181B681046194666
:10C8B800F4F7B8F903461C4641F62853C2F20003C0
:10C8C8005B881BB21846F4F759F9024640F65C43F8
:10C8D800C2F20003B9684FEA01115B1803F10803BB
:10C8E8001B6810461946F4F79DF903462046194679
:10C8F800F4F790F803461C4641F62853C2F20003A9
:10C908001B881BB21846F4F739F9024640F65C4317
:10C91800C2F20003B9684FEA01115B1803F104037E
:10C928001B6810461946F4F77DF903462046194658
:10C93800F4F770F803461C4641F68853C2F2000328
:10C948001B681B785BB2C3F1000241F62853C2F2A0
:10C9580000039B881BB203FB02F31846F4F70EF999
:10C96800024640F65C43C2F20003B9684FEA01117F
:10C978005B1803F10C031B6810461946F4F752F9CB
:10C98800034620461946F4F745F803461846F4F7D7
:10C998000FFB034699B241F69C53C2F20003BA68F2
:10C9A80023F81210BB6803F10103BB6040F656433D
:10C9B800C2F200031B781A46BB689A423FF663AF7F
:10C9C80040F61C53C2F200031B7803F1FF33142B0B
:10C9D80000F2C28201A050F823F000BF03CB000888
:10C9E80061CF000861CF000839CA000843CB0008AE
:10C9F80061CF000861CF0008F3CB000861CF0008C1
:10CA080061CF000861CF000861CF000861CF00083E
:10CA1800EDCB000861CF000861CF000861CF0008A6
:10CA280061CF000861CF00081FCE0008A1CE000822
:10CA38004FF004004FF00201FFF702FA03469AB2E2
:10CA480041F62853C2F200039B889BB203FB02F312
:10CA58009CB24FF004004FF00101FFF7F1F90346D3
:10CA68009AB241F62853C2F200035B889BB203FBDB
:10CA780002F39BB2E3189CB24FF00400FFF7AAF947
:10CA880003469BB2E3189BB29AB240F23403C2F257
:10CA980000031A814FF005004FF00201FFF7D0F9AB
:10CAA80003469AB241F62853C2F200039B889BB210
:10CAB80003FB02F39CB24FF005004FF00101FFF7B2
:10CAC800BFF903469AB241F62853C2F200035B88C5
:10CAD8009BB203FB02F39BB2E3189CB24FF0050034
:10CAE800FFF778F903469BB2E3189BB29AB240F27B
:10CAF8003403C2F200035A812FE24FF005004FF0D1
:10CB08000101FFF79DF903469AB241F62853C2F294
:10CB180000039B889BB203FB02F39CB24FF0050015
:10CB2800FFF758F903469BB2E3189BB29AB240F25A
:10CB38003403C2F200035A810FE241F69853C2F25D
:10CB480000031B689B795AB240F62443C2F20003E3
:10CB58005B881BB203FB02F248F21F53C5F2EB13CA
:10CB680083FB02134FEA23114FEAE273CB1A9CB2FC
:10CB78004FF00000FFF72EF903469BB2E3189BB273
:10CB88009AB240F23403C2F200031A8041F6985375
:10CB9800C2F200031B6803F108039B795AB240F6FE
:10CBA8002443C2F200031B881BB203FB02F248F2C3
:10CBB8001F53C5F2EB1383FB02C34FEA23114FEA5D
:10CBC800E273CB1A9CB24FF00100FFF703F903465A
:10CBD8009BB2E3189BB29AB240F23403C2F200034C
:10CBE8005A80BAE1FFF762FCB7E141F66C63C2F222
:10CBF80000035B78002B0CD141F68453C2F200038A
:10CC08001B689B889AB240F23403C2F20003DA81AF
:10CC18001EE041F69863C2F20003DB8819B241F6C0
:10CC28008453C2F200031B681B881A4641F68453DA
:10CC3800C2F200031B685B88084611461A46F9F7DA
:10CC4800C3FE03469AB240F23403C2F20003DA810B
:10CC580040F23403C2F20003DA8941F69C53C2F26F
:10CC680000031A8041F66C63C2F200039B7A002B22
:10CC780054D04FF003004FF00101FFF7E1F80346ED
:10CC88009AB241F69863C2F200035B889BB203FB39
:10CC980002F39CB24FF003004FF00201FFF7D0F807
:10CCA80003469AB241F69863C2F200031B889BB20E
:10CCB80003FB02F39BB2E3189BB29AB240F234032F
:10CCC800C2F20003DA804FF004004FF00101FFF7D1
:10CCD800B7F803469AB241F69863C2F200035B883C
:10CCE8009BB203FB02F39CB24FF004004FF0020129
:10CCF800FFF7A6F803469AB241F69863C2F200031A
:10CD08001B889BB203FB02F39BB2E3189BB29AB257
:10CD180040F23403C2F200031A8153E04FF00300DB
:10CD28004FF00101FFF78CF803469AB241F62853F9
:10CD3800C2F200035B889BB203FB02F39CB24FF084
:10CD480003004FF00201FFF77BF803469AB241F661
:10CD58002853C2F200031B889BB203FB02F39BB269
:10CD6800E3189BB29AB240F23403C2F20003DA80AD
:10CD78004FF004004FF00101FFF762F803469AB242
:10CD880041F62853C2F200035B889BB203FB02F30F
:10CD98009CB24FF004004FF00201FFF751F8034630
:10CDA8009AB241F62853C2F200031B889BB203FBD8
:10CDB80002F39BB2E3189BB29AB240F23403C2F278
:10CDC80000031A8140F23403C2F20003DB889CB2EC
:10CDD8004FF00300FEF7FEFF03469BB2E3189BB239
:10CDE8009AB240F23403C2F20003DA8040F234030C
:10CDF800C2F200031B899CB24FF00400FEF7EAFF61
:10CE080003469BB2E3189BB29AB240F23403C2F2D3
:10CE180000031A81A1E04FF00403BB6038E0BB684F
:10CE2800C3F1050241F62853C2F2000333F8123069
:10CE38009CB2BB6818464FF00101FFF701F80346A2
:10CE48009BB203FB04F39BB299B240F23403C2F2E3
:10CE58000003BA6823F8121040F23403C2F2000348
:10CE6800BA6833F812309CB2BB681846FEF7B2FFB6
:10CE780003469BB2E3189BB299B240F23403C2F264
:10CE88000003BA6823F81210BB6803F10103BB6002
:10CE9800BB68052BC3D960E04FF00303BB604DE0CE
:10CEA80041F62853C2F200039B889CB2BB6818461F
:10CEB8004FF00201FEF7C4FF03469BB203FB04F3E5
:10CEC8009CB2BB68C3F106034FEA530241F62853EC
:10CED800C2F2000333F812309DB2BB6818464FF017
:10CEE8000101FEF7ADFF03469BB203FB05F39BB2BE
:10CEF800E3189BB299B240F23403C2F20003BA6855
:10CF080023F8121040F23403C2F20003BA6833F86F
:10CF180012309CB2BB681846FEF75CFF03469BB212
:10CF2800E3189BB299B240F23403C2F20003BA6824
:10CF380023F81210BB6803F10103BB60BB68062B22
:10CF4800AED941F69863C2F20003DA8841F69C53E1
:10CF5800C2F200031A8000E000BF4FF02000F9F78A
:10CF6800BDFC0346002B00F012814FF00000FEF7D5
:10CF780031FF03461A4640F23403C2F200031A8016
:10CF88004FF00100FEF726FF03461A4640F234032D
:10CF9800C2F200035A8041F68063C2F200031B7A92
:10CFA800002B00F0F48041F68C53C2F200031B689A
:10CFB8001B7803F00203002B00F0958040F2340345
:10CFC800C2F200031B8899B241F69853C2F20003DB
:10CFD8001B6803F108039B795AB240F62443C2F256
:10CFE80000031B881BB203FB02F248F21F53C5F271
:10CFF800EB1383FB02034FEA23104FEAE273C31AD1
:10D0080098B241F69853C2F200031B689B795BB251
:10D01800C3F1000240F62443C2F200035B881BB24E
:10D0280003FB02F248F21F53C5F2EB1383FB02C362
:10D038004FEA23144FEAE273E31A9BB2C31A9BB276
:10D04800CB189BB29AB240F23403C2F200031A80A2
:10D0580040F23403C2F200035B8899B241F6985358
:10D06800C2F200031B689B795BB2C3F1000240F671
:10D078002443C2F200035B881BB203FB02F248F2AE
:10D088001F53C5F2EB1383FB02034FEA23104FEA49
:10D09800E273C31A98B241F69853C2F200031B68B0
:10D0A80003F108039B795AB240F62443C2F2000305
:10D0B8001B881BB203FB02F248F21F53C5F2EB13A5
:10D0C80083FB02C34FEA23144FEAE273E31A9BB2CD
:10D0D800C3189BB2CB189BB29AB240F23403C2F287
:10D0E80000035A8053E040F23403C2F200031B8865
:10D0F80099B241F69853C2F200031B689B795AB261
:10D1080040F62443C2F200035B881BB203FB02F221
:10D1180048F21F53C5F2EB1383FB02034FEA2310B7
:10D128004FEAE273C31A9BB2CB189BB29AB240F291
:10D138003403C2F200031A8040F23403C2F200033F
:10D148005B8899B241F69853C2F200031B6803F159
:10D1580008039B795AB240F62443C2F200031B88A5
:10D168001BB203FB02F248F21F53C5F2EB1383FB19
:10D1780002C34FEA23104FEAE273C31A9BB2CB18DB
:10D188009BB29AB240F23403C2F200035A804FF0C5
:10D198000003BB602FE040F23403C2F20003BA6818
:10D1A80033F8123019B241F69853C2F200031A68E4
:10D1B800BB684FEAC303D3181B881AB241F69853C9
:10D1C800C2F200031868BB684FEAC303C3185B8840
:10D1D8001BB2084611461A46F9F7F6FB034699B200
:10D1E80040F23403C2F20003BA6823F81210BB6895
:10D1F80003F10103BB60BB68072BCCD941F68C5304
:10D20800C2F200031B681B7803F00403002B45D00F
:10D218004FF000037B6040F61C53C2F200031B78FA
:10D228000E2B06D040F61C53C2F200031B78082BC5
:10D2380003D14FF004037B6011E040F61C53C2F2A7
:10D2480000031B784DF24012C0F601024FEAC303F7
:10D25800D3185B78002B02D04FF002037B604FF0AD
:10D268000003BB6017E0BB68DAB27B68DBB2D31897
:10D27800DAB2BB6803F1040141F6CC63C2F20003E1
:10D2880033F811309BB210461946F5F7AFFFBB686B
:10D2980003F10103BB60BB68032BE4D941F69C533F
:10D2A800C2F200031B88FB814FF00103BB6017E04B
:10D2B80041F69C53C2F20003BA6833F81230B7F94A
:10D2C8000E201BB29A4207DA41F69C53C2F20003C1
:10D2D800BA6833F81230FB81BB6803F10103BB6005
:10D2E80040F65643C2F200031B781A46BB689A42BE
:10D2F800DED84FF00003BB60F2E0B7F90E2041F62C
:10D308008453C2F200031B685B889A421ADD41F617
:10D318009C53C2F20003BA6833F812309AB241F64D
:10D328008453C2F200031B685988FB89CB1A9BB24D
:10D33800D3189BB299B241F69C53C2F20003BA6863
:10D3480023F812104FF48040F9F7C8FA0346002B6F
:10D3580055D041F6CC63C2F20003DB881AB241F61D
:10D368009453C2F200031B685B899A4223DD41F69D
:10D378009C53C2F20003BA6833F8123019B241F66E
:10D388009053C2F200031B685B881A4641F6845327
:10D39800C2F200031B685B88084611461A46F9F773
:10D3A80013FB034699B241F69C53C2F20003BA68D4
:10D3B80023F812107BE041F69C53C2F20003BA68CE
:10D3C80033F8123019B241F68453C2F200031B68D5
:10D3D8009B881A4641F69053C2F200031B681B88CB
:10D3E800084611461A46F9F7EFFA034699B241F68C
:10D3F8009C53C2F20003BA6823F8121057E041F6B2
:10D408009C53C2F20003BA6833F8123019B241F6DD
:10D418008453C2F200031B681B881A4641F68453E2
:10D42800C2F200031B685B88084611461A46F9F7E2
:10D43800CBFA034699B241F69C53C2F20003BA688C
:10D4480023F8121041F6CC63C2F20003DB881AB24B
:10D4580041F69453C2F200031B689B899A4226DA6C
:10D468004FF01000F9F73AFA034683F00103DBB2F4
:10D47800002B0ED041F68453C2F200031B681B88B0
:10D4880099B241F69C53C2F20003BA6823F812100D
:10D498000DE041F68453C2F200031B689B8899B2E1
:10D4A80041F69C53C2F20003BA6823F8121041F601
:10D4B8006C63C2F200035B78002B0DD141F6B453C4
:10D4C800C2F20003BA6833F8121041F69C53C2F254
:10D4D8000003BA6823F81210BB6803F10103BB60AC
:10D4E80040F65643C2F200031B781A46BB689A42BC
:10D4F8003FF603AF07F11007BD46B0BD80B400AFDB
:10D5080040F65843C2F200031B68002B0CBF0023EF
:10D518000123DBB21846BD4680BC704780B582B097
:10D5280000AF0346FB7141F6FC53C2F20003FA79DF
:10D538001A7041F6FC53C2F200034FF000021A6160
:10D54800FCF7F2FD024641F6FC53C2F200035A61B1
:10D5580007F10807BD4680BD80B483B000AF78608E
:10D5680041F61863C2F200037A681A6007F10C07E3
:10D57800BD4680BC704700BF80B586B000AFBA60BA
:10D588007B600346FB730B46BB7340F62B53C2F21A
:10D598000003BA7B1A70B868FFF7DEFF4FF0030389
:10D5A800FB754FF00000FFF7B9FF41F6FC53C2F2DC
:10D5B8000003FA7B5A70FCF7B7FD024641F6FC53AC
:10D5C800C2F200039A6041F6FC53C2F200034FF026
:10D5D80000025A6040F62B53C2F200031B78002B5E
:10D5E80002D14FF00103FB75786800F051FEFA7B19
:10D5F8004DF2F813C0F601034FEA02129B1803F12B
:10D6080004031A68FB7D4FF48840C4F200004FF011
:10D618000001F6F7A1F8024641F60473C2F20003CE
:10D628005A604FF00100FFF779FF07F11807BD4670
:10D6380080BD00BF80B582B000AF40F62B53C2F268
:10D6480000031B78032B00F2E98001A252F823F0B3
:10D6580069D60008A5D6000825D8000825D80008EE
:10D6680041F60473C2F200035A6841F6FC53C2F251
:10D6780000035B7819464DF2F813C0F601034FEA30
:10D6880001115B1803F104031B6810461946FCF7E7
:10D69800EDFB4FF00300FFF741FFBFE041F60473D5
:10D6A800C2F200035B681846FCF7F0FB034683F000
:10D6B8000103DBB2002B40F0B08041F6FC53C2F20C
:10D6C80000031B78012B5CD1FCF72EFD786041F636
:10D6D800FC53C2F200035B697A68D31A632B40F2E9
:10D6E800A58041F6FC53C2F200031B69042B43D802
:10D6F80041F60473C2F200035A6841F6FC53C2F2C1
:10D70800000319694DF2F813C0F601034FEA01113D
:10D718005B1803F104031B6810461946FCF7A6FBC7
:10D7280041F60473C2F200035A6841F6FC53C2F290
:10D7380000035B7819464DF2F813C0F601034FEA6F
:10D7480001115B1803F108031B6810461946FCF722
:10D758003DFB41F6FC53C2F200031B6903F10102D1
:10D7680041F6FC53C2F200031A6141F6FC53C2F2BF
:10D7780000037A685A6151E04FF00200FFF7CEFECD
:10D788004CE041F6FC53C2F200031B69002B18D190
:10D7980041F60473C2F200035A6841F6FC53C2F220
:10D7A80000035B7819464DF2F813C0F601034FEAFF
:10D7B80001115B1803F104031B6810461946FCF7B6
:10D7C80055FB41F6FC53C2F200031B698B2B1FD893
:10D7D80041F60473C2F200035A6841F6FC53C2F2E0
:10D7E800000319694DF24823C0F601035B5C10463B
:10D7F8001946FCF709FB41F6FC53C2F200031B690A
:10D8080003F1010241F6FC53C2F200031A6105E07C
:10D818004FF00300FFF782FE00E000BF41F6FC5323
:10D82800C2F200034FF000025A6000E000BF07F1A7
:10D838000807BD4680BD00BF80B500AF41F6047340
:10D84800C2F200035B68002B17D00BE041F60473AB
:10D85800C2F200035B681846FCF7F8FA034618465C
:10D8680000F0BCF941F60473C2F200035B68184685
:10D87800FCF7DCFA0346002BE8D141F6FC53C2F270
:10D8880000031B78042B72D801A151F823F000BFC4
:10D8980077D90008ADD80008ADD800084BD90008E2
:10D8A800B3D80008FFF7C6FE61E041F6FC53C2F2A8
:10D8B80000035B6803F1010241F6FC53C2F2000366
:10D8C8005A6041F6FC53C2F200035B7803F101038E
:10D8D800DAB241F6FC53C2F200035A7041F6FC5327
:10D8E800C2F200035A784CF6CD43CCF6CC43A3FBE6
:10D8F80002134FEA93010B464FEA83035B18D31ACE
:10D90800DAB241F6FC53C2F200035A70FCF70CFC81
:10D91800024641F6FC53C2F200039A6041F6546392
:10D92800C2F200034FF000021A7041F66C63C2F2B3
:10D9380000034FF00002DA724FF00100FFF7EEFD2E
:10D9480015E0FCF7F1FB024641F6FC53C2F2000376
:10D958009B68D21A40F6C4139A4207D94FF02000A8
:10D9680002F056FD4FF00400FFF7D8FD00BF80BD60
:10D9780080B582B000AF0346FB7140F62B53C2F26C
:10D9880000031B78032B1AD801A252F823F000BF1A
:10D99800A9D90008B5D90008A9D90008C1D9000833
:10D9A800FB79184601F094FC03460AE0FB79184617
:10D9B80001F0CAFE034604E04FF0000301E04FF017
:10D9C8000003184607F10807BD4680BD80B582B040
:10D9D80000AF786039607868F3F7D0F802463B68A2
:10D9E8001B6810461946F3F71DF903461846F3F766
:10D9F800DFFA0346184607F10807BD4680BD00BF99
:10DA0800B0B584B000AFF860B9607A603B607B68FD
:10DA18001C68F868F3F7B2F802463B685B68104682
:10DA28001946F3F7FFF803461A46BB681B68104609
:10DA38001946F3F7F7F8034620461946F2F7EAFFC6
:10DA480003461A467B681A607B681B681846F3F71A
:10DA5800AFFA05463B68DB6883F000431846F3F7E6
:10DA6800A7FA04463B68DB681846F3F7A1FA0346B1
:10DA7800284621461A46F8F7A7FF03461846F3F743
:10DA88007DF802467B681A607B681B681846F3F7C6
:10DA98008FFA0346184607F11007BD46B0BD00BF10
:10DAA800B0B586B000AFF860B9607A603B607B685B
:10DAB8005B68FA68D31A1846F3F760F80246BB6841
:10DAC8001B6810461946F3F761F903461A467B6846
:10DAD8001A6141F61863C2F200031B689B78184666
:10DAE800F3F748F803461846F2F7D8FC02460B4607
:10DAF800104619462CA3D3E90023F2F723FD02466A
:10DB08000B464FF000004FF00001C3F6F071F2F73A
:10DB180043FE02460B4610461946F2F725FF034618
:10DB28007B617B689C68BB681D68BB681B6818467E
:10DB38007969F2F76FFF034628461946F3F726F985
:10DB480003461D467B681A697B689B681046194620
:10DB5800F2F75EFF034628461946F3F763F80346D3
:10DB680020461946F2F756FF03461A467B681A61A3
:10DB78007B68FA685A607B681A697B689A603B68B8
:10DB88009A687B681B6910461946F3F74BF80346F9
:10DB98001846F3F70DFA0346184607F11807BD466D
:10DBA800B0BD00BFAFF30080182D4454FB211940CD
:10DBB80080B483B000AF78607B684FF000021A60D1
:10DBC8007B684FF000025A607B684FF000029A6051
:10DBD80007F10C07BD4680BC704700BF90B589B0FF
:10DBE80002AF0346FB80FB88DBB21846FFF7C0FE96
:10DBF8000346002B00F0A98241F6FC53C2F2000351
:10DC08009A6841F6FC53C2F20003DA60FCF78CFA1A
:10DC1800024641F6FC53C2F200039A604FF020001E
:10DC280002F0E0FB40F62053C2F200031B78012B00
:10DC380007D140F62053C2F200034FF000021A70D9
:10DC480006E040F62053C2F200034FF001021A70BA
:10DC580041F66C63C2F20003DB7A002B00F0758298
:10DC680041F65463C2F200031B78042B40F26D8224
:10DC780041F66C63C2F200035B78002B06D141F6D3
:10DC88006C63C2F200034FF000021A7341F66C6332
:10DC9800C2F200031B7B002B08D141F66C63C2F271
:10DCA80000035B78002B01D000F05AFA40F60263BB
:10DCB800C2F200031B7803F1010146F26763C6F262
:10DCC800666383FB01234FEA63024FEAE173D21ACA
:10DCD80013464FEA83039B18CA1AD2B240F602636E
:10DCE800C2F200031A704FF000037B610CE141F6A9
:10DCF8003C63C2F200037A6953F8221040F6346399
:10DD0800C2F200037A6943F8221040F63463C2F283
:10DD180000037A6953F822204CF66B23C6F65F336A
:10DD280083FB02134FEAA3514FEAE273C91A40F684
:10DD38004463C2F200037A6943F8221040F6346360
:10DD4800C2F200037A6953F8222040F64463C2F213
:10DD58000003796953F821104FF4D343CFF6677362
:10DD680003FB01F3D21848F6AD33C6F6DB0383FB99
:10DD780002134FEA23314FEAE273CB1A99B240F605
:10DD88004C63C2F200037A6923F8121040F62C6340
:10DD9800C2F200037A6953F8220040F60263C2F225
:10DDA80000031B781C4640F60462C2F2000279693F
:10DDB8000B464FEA83035B181B1952F82330C11A2C
:10DDC80040F62C63C2F200037A6943F8221040F649
:10DDD8000263C2F200031B781C4640F63463C2F2A9
:10DDE80000037A6953F8222040F64463C2F2000324
:10DDF800796953F821104FF4D343CFF6677303FBC7
:10DE080001F3D01840F60462C2F2000279690B46A9
:10DE18004FEA83035B181B1942F8230040F62C6372
:10DE2800C2F200037A6953F8220040F60263C2F294
:10DE380000031B781C4640F60462C2F200027969AE
:10DE48000B464FEA83035B181B1952F82330C1189D
:10DE580040F62C63C2F200037A6943F8221040F6B8
:10DE68002C63C2F200037A6953F8222046F26763F2
:10DE7800C6F2666383FB02134FEA63014FEAE2735B
:10DE8800CA1A40F64463C2F20003796953F82110B4
:10DE980049F28063C0F2980303FB01F3D11840F6FE
:10DEA8003C63C2F200037A6943F8221040F62A5311
:10DEB800C2F200031B785BB2012B21D140F64C6300
:10DEC800C2F200037A6933F81230012B18D940F6F0
:10DED8004C63C2F200037A6933F8122040F2E63349
:10DEE8009A420DD840F63C63C2F200037A6953F8AF
:10DEF800221041F63C63C2F200037A6943F822100B
:10DF08007B6903F101037B617B69012B7FF7EFAE2E
:10DF1800FCF70AF9024640F65473C2F200031B6884
:10DF2800D31A1846F2F726FE034618464FF00001AA
:10DF3800C4F27A41F2F72AFF03461A4640F6D45350
:10DF4800C2F200031A60FCF7EFF8024640F6547379
:10DF5800C2F200031A6040F6D453C2F200031B68F1
:10DF680018464FF07E51F2F7FBFF0346002B05D011
:10DF780040F6D453C2F200031A6801E04FF07E5213
:10DF880040F6D453C2F200031A6007F10C03009361
:10DF980007F10803019341F63C60C2F200006D49A5
:10DFA80041F62062C2F200026B4B00F07BFBFA687C
:10DFB80048F21F53C5F2EB13A3FB02134FEA5313A6
:10DFC8009AB241F61C63C2F200031A80BA6848F29A
:10DFD8001F53C5F2EB1383FB02134FEA63114FEA99
:10DFE800E273CB1A9AB241F62863C2F200031A8090
:10DFF80041F66C63C2F200031B7B002B0DD141F686
:10E008001C63C2F200034FF000021A8041F6286335
:10E01800C2F200034FF000021A8000F0B9FB41F68B
:10E028006C63C2F200031B7A002B07D141F66C63C4
:10E03800C2F20003DB79002B00F0878040F6FC5326
:10E04800C2F20003009340F6F053C2F200030193BA
:10E0580041F63C60C2F200003E4940F6E852C2F286
:10E0680000023E4B00F01EFB40F6E850C2F20000F2
:10E078003A4941F63C62C2F20002364B00F048FCD5
:10E0880040F62A53C2F200031B785BB2012B02D080
:10E09800022B03D059E000F06DFC56E041F61863FE
:10E0A800C2F200031B681B899BB21BB218464FF0D3
:10E0B800010100F02BFF03467B82B7F912301846A6
:10E0C80000F05EFD41F61863C2F200031B681B797D
:10E0D800002B15D040F65063C2F200031A6848F2CC
:10E0E8001F53C5F2EB1383FB02134FEA63114FEA88
:10E0F800E273CB1A9AB241F62453C2F200031A8093
:10E1080041F61863C2F200031B681B881A4640F6E2
:10E11800FC53C2F200031B689A4204D200F09EFA34
:10E128000346002B10D040F62A53C2F200034FF0EA
:10E1380001021A7040F65463C2F200031A8841F6CD
:10E148002453C2F200031A8000BF07F11C07BD4622
:10E1580090BD00BF401E0020241E0020EC0D0020B2
:10E1680080B500AF41F66C63C2F20003DB7A002B86
:10E1780033D041F65463C2F200031B78042B2CD928
:10E1880041F63C63C2F200031A6841F62063C2F20A
:10E1980000031A6041F63C63C2F200035A6841F674
:10E1A8002063C2F200035A6041F63C63C2F20003E6
:10E1B8001B68184600F0A6F941F63C53C2F200036A
:10E1C8001A8840F65463C2F200031A8041F66C6361
:10E1D800C2F200034FF001021A7380BD80B582B00D
:10E1E80000AF4FF000037B604BE040F62453C2F2CF
:10E1F80000037A684FF0000123F8121041F6E45347
:10E20800C2F200037A684FF0000123F8121041F6B9
:10E21800EC53C2F200037A684FF0000123F81210A1
:10E228007A6813464FEA83039B184FEA830340F644
:10E238005C52C2F200029B181846FFF7B9FC7A68D4
:10E2480013464FEA83039B184FEA830340F6845230
:10E25800C2F200029B181846FFF7AAFC7A68134618
:10E268004FEA83039B184FEA830340F6AC52C2F28D
:10E2780000029B181846FFF79BFC7B6803F101031B
:10E288007B607B68012BB0DD07F10807BD4680BDC8
:10E2980080B582B000AF78607B681B791846F2F7CA
:10E2A80069FC034618464FF00001C4F2C821F2F792
:10E2B8006DFD03461A4640F62C53C2F200031A605D
:10E2C8007B689B7B1846F2F755FC034618464FF0CF
:10E2D8000001C4F2C821F2F759FD03461A4640F678
:10E2E8002C53C2F200035A6040F62C53C2F20003CA
:10E2F8004FF00002C4F2FA42DA607B685B79184694
:10E30800F2F738FC034618464FF00001C4F220111A
:10E31800F2F73CFD03461A4640F63C53C2F20003AE
:10E328001A607B68DB7B1846F2F724FC0346184624
:10E338004FF00001C4F2C821F2F728FD03461A463F
:10E3480040F63C53C2F200035A607B685B7E184675
:10E35800F2F710FC034618464FF00001C4F27A4168
:10E36800F2F714FD03461A4640F63C53C2F2000386
:10E378009A6040F63C53C2F200034FF00002C4F228
:10E38800FA42DA607B689B791846F2F7F3FB03469A
:10E3980018464FF00001C4F22011F2F7F7FC0346CB
:10E3A8001A4640F64C53C2F200031A607B681B7C85
:10E3B8001846F2F7DFFB034618464FF00001C4F297
:10E3C800C821F2F7E3FC03461A4640F64C53C2F262
:10E3D80000035A607B689B7E1846F2F7CBFB034626
:10E3E80018464FF00001C4F27A41F2F7CFFC034619
:10E3F8001A4640F64C53C2F200039A6040F64C535A
:10E40800C2F200034FF00002C4F2FA42DA6007F1E8
:10E418000807BD4680BD00BF98B500AF41F6FC5364
:10E42800C2F200031B78032B03D04FF0FF035BB24B
:10E4380066E04FF48053C4F600034FF488521A85FF
:10E448004FF48053C4F600034FF488421A8500E065
:10E4580000BF41F60473C2F200035B681846FBF77D
:10E46800E5FC0346002B1FD04FF48053C4F600038D
:10E478004FF488529A6141F60473C2F200031C6893
:10E4880041F60473C2F200035B681846FBF7DEFC32
:10E49800034620461946FBF7B7FC4FF48053C4F6F1
:10E4A80000034FF488521A8541F60473C2F2000340
:10E4B8001B681846FBF7BAFC0346002BC8D04FF47C
:10E4C8008053C4F600034FF488429A6141F60473FE
:10E4D800C2F200035C6841F60473C2F200031B68D1
:10E4E8001846FBF7B3FC034620461946FBF78CFC9D
:10E4F8004FF48053C4F600034FF488421A85A7E707
:10E50800184698BD80B584B000AF78607868F2F797
:10E5180035FB034618464FF00001F2F73FFD03466E
:10E52800002B14D07868F2F729FB0346184649F205
:10E538008061C4F61831F2F729FC034618464FF6F5
:10E548003521C3F68E41F2F76DFB034615E0786876
:10E55800F2F714FB034683F00043184649F2806142
:10E56800C4F61831F2F712FC034618464FF6352167
:10E57800C3F68E41F2F756FB0346FB60F8680AF0D3
:10E588006DF9024640F24403C2F200031A6007F133
:10E598001007BD4680BD00BF80B584B002AF78606B
:10E5A80039607B681A6840F6E853C2F200031A60C3
:10E5B8003B681A6840F6E853C2F200035A607B6869
:10E5C8001B681846FFF79EFF40F6FC53C2F2000393
:10E5D800009340F6F053C2F20003019341F63C6009
:10E5E800C2F200001B4940F6E852C2F200021A4B80
:10E5F80000F058F840F6F053C2F200031A6840F6EB
:10E608005063C2F200031A6040F6E850C2F20000FC
:10E61800114941F63C62C2F200020E4B00F078F953
:10E6280040F6F053C2F200031A6840F6F453C2F2FF
:10E6380000031A6041F61863C2F200031B68DB8806
:10E648009AB240F60063C2F200031A8007F1080785
:10E65800BD4680BD401E0020EC0D002080B582B074
:10E6680000AF40F6F053C2F200031A6840F6F453C4
:10E67800C2F200031B68D31A7B60786800F0AEFC16
:10E6880078607B6883EAE372A2EBE37242F210736C
:10E698009A42D4BF00230123DBB2184607F10807CA
:10E6A800BD4680BD90B587B000AFF860B9607A60AC
:10E6B8003B607B681A68FB681B68D31A1846F2F738
:10E6C8005DFA03467B613B681A68BB681B68D31A0E
:10E6D8001846F2F753FA024640F24403C2F2000326
:10E6E8001B6810461946F2F79DFA03463B617869A4
:10E6F8007969F2F797FA03461C4638693969F2F7DF
:10E7080091FA034620461946F2F784F9034618465B
:10E718000AF0A6F90346184647F62C51C3F68E713F
:10E72800F2F780FA03461846F2F768FC0246BB6A1D
:10E738001A607B6983F00043184639690AF08EF93C
:10E74800034618464FF44A61C4F2B351F2F76AFA25
:10E75800034618464FF42041C4F20C61F2F75AF907
:10E7680003461846F2F724FC0246FB6A1A60FB6A65
:10E778001B68002B07DAFB6A1B6803F50C4303F1DF
:10E78800A003FA6A136007F11C07BD4690BD00BFDD
:10E7980080B582B000AF40F64673C2F200031B7822
:10E7A800002B00F0968040F6D453C2F200031B6899
:10E7B8004FF07E501946F2F7E9FA03467B6041F6BE
:10E7C8003C63C2F200035A6840F64873C2F2000381
:10E7D8005B68D31A1846F2F7D1F9024640F24403AF
:10E7E800C2F200031B6810461946F2F71BFA0346EB
:10E7F80018467968F2F716FA03461846F2F7D8FB76
:10E8080003469AB240F6D853C2F200035A8041F642
:10E818003C63C2F200031A6840F64873C2F2000370
:10E828001B68D31A1846F2F7A9F9034618467968FF
:10E83800F2F7F8F903461846F2F7BAFB03469AB21C
:10E8480040F6D853C2F200031A8040F6D853C2F2F9
:10E8580000035B881AB240F65073C2F200035B886B
:10E868001BB2D3184FEAD372D3184FEA63039AB294
:10E8780040F6D853C2F200035A8040F6D853C2F289
:10E8880000031B881AB240F65073C2F200031B88BB
:10E898001BB2D3184FEAD372D3184FEA63039AB264
:10E8A80040F6D853C2F200031A8040F6D853C2F299
:10E8B80000035A8840F65073C2F200035A8040F6AB
:10E8C800D853C2F200031A8840F65073C2F200030C
:10E8D8001A8040F64673C2F200034FF001021A7024
:10E8E80041F63C63C2F200035A6840F64873C2F22C
:10E8F80000035A6041F63C63C2F200031A6840F60E
:10E908004873C2F200031A6007F10807BD4680BDCC
:10E9180080B584B000AFF860B9607A603B60BB68CE
:10E928001A683B681B68D31A1846F2F727F902469B
:10E9380040F24403C2F200031B6810461946F2F77E
:10E9480071F903461846F2F733FB024640F6E053E6
:10E95800C2F200035A60FB681A687B681B68D21A07
:10E9680040F6E053C2F200031A6007F11007BD46F3
:10E9780080BD00BF90B585B000AF4FF00003BB600D
:10E98800F5E040F6E053C2F20003BA6853F82230CB
:10E99800184640F62C51C2F20001FFF717F87860CC
:10E9A8007B689AB240F6D853C2F20003B96833F8CC
:10E9B80011309BB2D31A9BB299B240F6DC53C2F223
:10E9C8000003BA6823F8121040F6DC53C2F20003C1
:10E9D800BA6833F812301BB2184640F63C51C2F2FE
:10E9E8000001FEF7F3FF03469CB240F6DC53C2F287
:10E9F8000003BA6833F812301AB240F6E053C2F294
:10EA08000003B96853F82130D118BA6813464FEAA1
:10EA180083039B184FEA830340F68452C2F2000234
:10EA28009B18084640F6D451C2F200011A4640F637
:10EA38003C53C2F20003FEF7E3FF03469BB2E31820
:10EA48009BB299B241F6EC53C2F20003BA6823F8BC
:10EA5800121040F6E053C2F20003BA6853F82210CD
:10EA6800BA6813464FEA83039B184FEA830340F6BC
:10EA78008452C2F200029B18084640F6D451C2F2F2
:10EA880000011A4640F63C53C2F20003FFF708F8AB
:10EA9800F860F8684FF63001CFF6FF714FF4FA626C
:10EAA800F7F792FFF86040F6D853C2F20003BA684D
:10EAB80033F812301BB213F1310F0CDB40F6D85388
:10EAC800C2F20003BA6833F812301BB2312B02DCF1
:10EAD8004FF00003FB6041F6EC53C2F20003BA6842
:10EAE80033F812309AB2FB689BB2D3189BB299B232
:10EAF80041F6EC53C2F20003BA6823F8121041F64B
:10EB0800EC53C2F20003BA6833F812301BB218464D
:10EB18004FF24841CFF6FF7140F6B832F7F754FF8D
:10EB2800034699B241F6EC53C2F20003BA6823F8DF
:10EB3800121040F68452C2F20002B9680B464FEA3E
:10EB480083035B184FEA8303D318186840F6AC5266
:10EB5800C2F20002B9680B464FEA83035B184FEA1A
:10EB68008303D3181860BB6803F10103BB60BB685B
:10EB7800012B7FF706AF07F11407BD4690BD00BF14
:10EB880090B587B000AF786000F00EF940F650639A
:10EB9800C2F200031B68C3F50C5303F1280318469F
:10EBA800F1F7ECFF0346184640F2D321C3F63711BC
:10EBB800F2F738F803463B61386909F04FFE03461F
:10EBC800FB60386909F0BEFE0346BB604FF00003E6
:10EBD8007B61E1E07B694FEA830307F11802D318F0
:10EBE80053F8104C7868F1F7C9FF034620461946D8
:10EBF800F2F718F803461C4640F6D853C2F2000351
:10EC08007A6933F812301BB21846F1F7B7FF03469A
:10EC180020461946F1F7FCFE03461846F2F7C8F9F4
:10EC2800034699B240F6DC53C2F200037A6923F82E
:10EC3800121040F6DC53C2F200037A6933F812303E
:10EC48001BB218464FF61841CFF6FF714FF47A728F
:10EC5800F7F7BAFE034699B240F6DC53C2F2000356
:10EC68007A6923F8121040F6DC53C2F200037A697D
:10EC780033F812301BB2184640F64C51C2F200016C
:10EC8800FEF7A4FE03469CB240F6DC53C2F2000332
:10EC98007A6933F8123019B27A6913464FEA830356
:10ECA8009B184FEA830340F6AC52C2F200029B184D
:10ECB800084640F6D451C2F200011A4640F64C53B9
:10ECC800C2F20003FEF79CFE03469BB2E3189CB217
:10ECD80040F6DC53C2F200037A6933F8123019B2F5
:10ECE8007A6913464FEA83039B184FEA830340F679
:10ECF800AC52C2F200029B18084640F6D451C2F248
:10ED080000011A4640F64C53C2F20003FEF7C8FE53
:10ED180003469BB2E3189BB299B241F6EC53C2F298
:10ED280000037A6923F8121041F6EC53C2F200038B
:10ED38007A6933F812301BB218464FF24841CFF6C1
:10ED4800FF7140F6B832F7F73FFE034699B241F635
:10ED5800EC53C2F200037A6923F8121040F6AC5261
:10ED6800C2F2000279690B464FEA83035B184FEA47
:10ED78008303D318186840F68452C2F200027969F6
:10ED88000B464FEA83035B184FEA8303D3181860D6
:10ED98007B6903F101037B617B69012B7FF71AAF64
:10EDA80007F11C07BD4690BD90B583B000AF40F693
:10EDB800F053C2F200031A6840F6F453C2F200039B
:10EDC8001B68D31A184600F009F90346002B16DD14
:10EDD80040F6F053C2F200031A6840F6F453C2F248
:10EDE80000031B68D31A184600F0F8F8024641F2EF
:10EDF80093139A42CCBF00230123DBB217E040F6FD
:10EE0800F053C2F200031A6840F6F453C2F200034A
:10EE18001B68D31A184600F0E1F80346C3F1000254
:10EE280041F293139A42CCBF00230123DBB2002B9B
:10EE38005DD040F6F053C2F200031A6840F6F4536E
:10EE4800C2F200031B68D31A1846F1F797FE03466F
:10EE5800184640F2D321C3F63711F1F7E3FE034613
:10EE68007B60786809F06EFD044640F6FC53C2F2F8
:10EE780000031B681846F1F77DFE03462046194635
:10EE8800F1F7D0FE03461846F2F792F803469AB215
:10EE980040F6F853C2F200031A8040F6F853C2F263
:10EEA80000031B881BB218464FF24841CFF6FF718A
:10EEB80040F6B832F7F788FD024640F6F053C2F242
:10EEC80000031B68D21840F65063C2F200031A60B0
:10EED80040F65063C2F200031B68184600F0A2F81F
:10EEE800024640F65063C2F200031A6009E040F699
:10EEF800F053C2F200031A6840F65063C2F20003EE
:10EF08001A6007F10C07BD4690BD00BF80B582B0FE
:10EF180000AF02460B46FA807B717B79002B0DD03F
:10EF280040F6FC53C2F200031B684FEA5302B7F9DC
:10EF380006309A4238BF1346FB8017E0B7F906201F
:10EF480040F6FC53C2F200031B689A4238BF1346CE
:10EF5800FB8041F61863C2F200031B68DB881A467F
:10EF6800B7F906309A42A8BF1346FB8040F6006303
:10EF7800C2F200031B88B7F906201BB29A4225DDAE
:10EF880040F6D453C2F200031B6818464FF0000144
:10EF9800C4F2C821F1F746FE03461846F2F708F80E
:10EFA80003469AB240F60063C2F200031B889BB284
:10EFB800D3189BB29AB240F60063C2F200031A80DB
:10EFC80040F60063C2F200031B88FB80FB881BB27B
:10EFD800184607F10807BD4680BD00BF80B483B05E
:10EFE80000AF78607A6844F250639A4205DD7B6826
:10EFF800A3F50C43A3F1A0037B607A684BF6B0132A
:10F00800CFF6FF739A4205DA7B6803F50C4303F1E8
:10F01800A0037B607B68184607F10C07BD4680BCDF
:10F02800704700BF80B483B000AF78607A6848F654
:10F03800A0439A4205DD7B68A3F50C43A3F1A00326
:10F048007B607B68002B05DA7B6803F50C4303F1D2
:10F05800A0037B607B68184607F10C07BD4680BC9F
:10F06800704700BF80B489B000AF78604FF00003EC
:10F07800FB754FF00003BB754FF000033B617B68E5
:10F08800FB610CE07B6803F10F02FB699A4202D82E
:10F098004FF00003A0E0FB6903F10103FB6140F2BC
:10F0A8009013C2F200031A68FB691B7803F101038D
:10F0B800D3181B7803F00403002BE3D17B68BB61F2
:10F0C80016E0FB7D002B07D0FB7D1A464FEA820233
:10F0D800D3184FEA4303FB75BB691A78FB7DD31835
:10F0E800DBB2A3F13003FB75BB6903F10103BB611C
:10F0F800FA69BB69D31A022BE3DC16E0BB7D002B4F
:10F1080007D0BB7D1A464FEA8202D3184FEA430361
:10F11800BB75BB691A78BB7DD318DBB2A3F130038A
:10F12800BB75BB6903F10103BB61FA69BB699A420C
:10F13800E4D8FB691B782E2B31D1FB6903F101035D
:10F14800BB614FF00003FB6026E03A6913464FEAC3
:10F1580083039B184FEA43033B6140F29013C2F2CA
:10F1680000031A68BB691B7803F10103D3181B78E5
:10F1780003F00403002B0BD0BB691B781A463B69CC
:10F18800D318A3F130033B61BB6903F10103BB61F1
:10F19800FB6803F10103FB60FB68032BD5DDFA7DF7
:10F1A80049F28063C0F2980303FB02F2B97D44F28E
:10F1B8004023C0F20F0303FB01F13B694FF06400E9
:10F1C80000FB03F3C9184AF6AB23CAF6AA23A3FB2C
:10F1D80001034FEA9303D318184607F12407BD46E5
:10F1E80080BC704780B485B000AF78600B46FB7078
:10F1F8004FF00003BB604FF00003FB603CE07A680F
:10F20800FB68D3181B782E2B0ED1FB6803F1010382
:10F21800FB60FB78002B36D0FA78FB68D3187A6845
:10F22800D3184FF000021A70BA6813464FEA8303E6
:10F238009B184FEA4303BB607A68FB68D3181B78B6
:10F248002F2B0FD97A68FB68D3181B78392B09D86C
:10F258007A68FB68D3181B781A46BB68D318A3F1E1
:10F268003003BB60FB680E2B02D94FF000030CE0A3
:10F27800FB6803F10103FB607A68FB68D3181B780D
:10F28800002BBCD100E000BFBB68184607F114078B
:10F29800BD4680BC704700BF80B483B000AF034652
:10F2A800FB71FB79A3F13003FB71FB79092B03D9BF
:10F2B800FB79A3F10703FB71FB7903F00F03FB71E3
:10F2C800FB79184607F10C07BD4680BC704700BFA4
:10F2D80080B584B000AF0346FB714FF00003FB73A9
:10F2E800FB79242B15D140F63073C2F200034FF09E
:10F2F80000021A7040F63173C2F200034FF00002A8
:10F308001A7040F63273C2F200034FF000021A700E
:10F3180002E2FB792C2B03D0FB792A2B40F0928157
:10F3280040F63173C2F200031B781A4640F6347374
:10F33800C2F200034FF00001995440F63073C2F254
:10F3480000031B78002B60D140F64473C2F200031F
:10F358004FF000021A7040F63473C2F200031B78B3
:10F36800472B22D140F63473C2F200035B78502B4E
:10F378001BD140F63473C2F200039B78472B14D19B
:10F3880040F63473C2F20003DB78472B0DD140F608
:10F398003473C2F200031B79412B06D140F6447343
:10F3A800C2F200034FF001021A7040F63473C2F241
:10F3B80000031B78472B40F0188140F63473C2F2E3
:10F3C80000035B78502B40F0108140F63473C2F292
:10F3D80000039B78522B40F0088140F63473C2F248
:10F3E8000003DB784D2B40F0008140F63473C2F205
:10F3F80000031B79432B40F0F88040F64473C2F2B7
:10F4080000034FF002021A70EFE040F64473C2F2B4
:10F4180000031B78012B40F0A68040F63073C2F23F
:10F4280000031B78022B0DD140F63470C2F20000A5
:10F43800FFF718FE03461A4641F63C63C2F2000382
:10F448001A60D1E040F63073C2F200031B78032B38
:10F4580013D140F63473C2F200031B78532B0CD13E
:10F4680041F63C63C2F200031B68C3F1000241F697
:10F478003C63C2F200031A60B7E040F63073C2F290
:10F4880000031B78042B0DD140F63470C2F2000043
:10F49800FFF7E8FD03461A4641F63C63C2F2000353
:10F4A8005A60A1E040F63073C2F200031B78052BC6
:10F4B80013D140F63473C2F200031B78572B0CD1DA
:10F4C80041F63C63C2F200035B68C3F1000241F6F7
:10F4D8003C63C2F200035A6087E040F63073C2F220
:10F4E80000031B78062B10D140F63473C2F20003D8
:10F4F8001B78302B94BF00230123DBB21A4641F658
:10F508006C63C2F20003DA726EE040F63073C2F246
:10F5180000031B78072B0FD140F63470C2F20000AD
:10F528004FF00001FFF75EFE0346DAB241F654637E
:10F53800C2F200031A7057E040F63073C2F20003BB
:10F548001B78092B50D140F63470C2F200004FF0FE
:10F558000001FFF747FE03469AB241F6E253C2F2B2
:10F5680000031A8040E040F64473C2F200031B789F
:10F57800022B3AD140F63073C2F200031B78072BF6
:10F588001BD140F63470C2F200004FF00101FFF7C2
:10F5980029FE034641F2184202FB03F244F6D35314
:10F5A800C1F26203A3FB02134FEA93139AB241F626
:10F5B800F053C2F200031A8017E040F63073C2F22B
:10F5C80000031B78082B10D140F63470C2F20000FB
:10F5D8004FF00101FFF706FE03469AB240F62853A2
:10F5E800C2F200031A8000E000BF40F63073C2F296
:10F5F80000031B7803F10103DAB240F63073C2F25C
:10F6080000031A7040F63173C2F200034FF0000293
:10F618001A70FB792A2B07D140F64573C2F2000312
:10F628004FF001021A7077E040F63273C2F200031D
:10F638001A78FB795340DAB240F63273C2F200030B
:10F648001A7069E0FB790D2B02D0FB790A2B34D1B3
:10F6580040F64573C2F200031B78002B25D040F614
:10F668003473C2F200031B781846FFF715FE0346F1
:10F67800BB73BB7B4FEA0313BB7340F63473C2F210
:10F6880000035B781846FFF707FE03461A46BB7B64
:10F69800D318BB7340F63273C2F200031B78BA7BEF
:10F6A8009A4202D14FF00103FB7340F64573C2F250
:10F6B80000034FF000021A702EE040F63173C2F2D8
:10F6C80000031B780E2B13D840F63173C2F20003E7
:10F6D8001A78114640F63473C2F20003F879585488
:10F6E80002F10103DAB240F63173C2F200031A7074
:10F6F80040F64573C2F200031B78002B0CD140F68C
:10F708003273C2F200031A78FB795340DAB240F63A
:10F718003273C2F200031A70FB7B002B09D040F64B
:10F728004473C2F200031B78012B02D14FF001038E
:10F7380001E04FF0000303F00103DBB2184607F1C4
:10F748001007BD4680BD00BF80B584B000AF03463A
:10F75800FB714FF00003FB7340F65863C2F20003DD
:10F768001B78082B00F2B78101A252F823F000BFE2
:10F77800CDF700089DF70008F1F7000839F80008F0
:10F788009DF8000803F90008B7F9000867FA0008AF
:10F79800A1FA0008FB79622B0DD140F65863C2F23A
:10F7A80000031B7803F10103DAB240F65863C2F292
:10F7B80000031A708FE140F65863C2F200034FF05D
:10F7C80000021A70FB79B52B40F07E8140F6586331
:10F7D800C2F200031B7803F10103DAB240F6586362
:10F7E800C2F200031A706FE140F65863C2F20003D8
:10F7F8001B7803F10103DAB240F65863C2F2000342
:10F808001A7040F65F63C2F20003FA791A7040F684
:10F818005663C2F20003FA791A7040F65663C2F2D0
:10F8280000031A7840F65763C2F200031A7052E1D7
:10F8380040F65863C2F200031B7803F10103DAB201
:10F8480040F65863C2F200031A7040F65663C2F2DB
:10F8580000031A78FB79D318DAB240F65663C2F27D
:10F8680000031A7040F65663C2F200031A7840F695
:10F878005763C2F200031B78D318DAB240F6576315
:10F88800C2F200031A7040F65963C2F20003FA7913
:10F898001A7020E140F65863C2F200031B7803F1A6
:10F8A8000103DAB240F65863C2F200031A7040F658
:10F8B8005663C2F200031A78FB79D318DAB240F61D
:10F8C8005663C2F200031A7040F65663C2F2000390
:10F8D8001A7840F65763C2F200031B78D318DAB2DD
:10F8E80040F65763C2F200031A70FB799AB240F6E9
:10F8F8005A63C2F200031A80EDE040F65863C2F280
:10F9080000031B7803F10103DAB240F65863C2F230
:10F9180000031A7040F65663C2F200031A78FB79A6
:10F92800D318DAB240F65663C2F200031A7040F6F2
:10F938005663C2F200031A7840F65763C2F2000316
:10F948001B78D318DAB240F65763C2F200031A7074
:10F95800FB799BB24FEA03239AB240F65A63C2F28C
:10F9680000031B88D3189AB240F65A63C2F2000308
:10F978001A8040F65A63C2F200031B88B3F5007F71
:10F988000DD940F65A63C2F200034FF000021A8004
:10F9980040F65863C2F200034FF000021A7040F6B6
:10F9A8005C63C2F200034FF000021A8093E040F655
:10F9B8005663C2F200031A78FB79D318DAB240F61C
:10F9C8005663C2F200031A7040F65663C2F200038F
:10F9D8001A7840F65763C2F200031B78D318DAB2DC
:10F9E80040F65763C2F200031A7040F65C63C2F235
:10F9F80000031B88C72B0BD840F65C63C2F20003D8
:10FA08001B881A4640F66463C2F20003F9799954D8
:10FA180040F65C63C2F200031B8803F101039AB24B
:10FA280040F65C63C2F200031A8040F65C63C2F2DF
:10FA380000031A8840F65A63C2F200031B889A42F0
:10FA480044D140F65863C2F200031B7803F1010366
:10FA5800DAB240F65863C2F200031A7036E040F694
:10FA68005863C2F200031B7803F10103DAB240F6CF
:10FA78005863C2F200031A7040F65663C2F20003DC
:10FA88001B78FA799A4223D040F65863C2F20003F1
:10FA98004FF000021A701BE040F65863C2F20003F0
:10FAA8004FF000021A7040F65763C2F200031B7849
:10FAB800FA799A420ED100F015F80346002B0AD0C5
:10FAC8004FF00103FB7306E000BF04E000BF02E053
:10FAD80000BF00E000BFFB7B184607F11007BD46DA
:10FAE80080BD00BF80B483B000AF40F65963C2F256
:10FAF80000031B78A3F102032E2B00F2B38101A1AE
:10FB080051F823F0C9FB000843FC00086DFE00080B
:10FB18006DFE0008A3FC00086DFE00086DFE0008DD
:10FB28006DFE00086DFE00086DFE00086DFE000801
:10FB38006DFE00086DFE00086DFE00086DFE0008F1
:10FB48006DFE000817FD00086DFE00086DFE000838
:10FB58006DFE00086DFE00086DFE00086DFE0008D1
:10FB68006DFE00086DFE00086DFE00086DFE0008C1
:10FB78006DFE00086DFE00086DFE00086DFE0008B1
:10FB88006DFE00086DFE00086DFE00086DFE0008A1
:10FB98006DFE00086DFE00086DFE00086DFE000891
:10FBA8006DFE00086DFE00086DFE00086DFE000881
:10FBB8006DFE00086DFE00086DFE000869FD000876
:10FBC80040F66463C2F200035A6841F63C63C2F22D
:10FBD80000035A6040F66463C2F200039A6841F673
:10FBE8003C63C2F200031A6040F66463C2F2000389
:10FBF8001A6944F6D353C1F2620383FB02134FEA36
:10FC0800A3114FEAE273CB1A9AB241F6E253C2F259
:10FC180000031A8040F65E63C2F200031B781A469E
:10FC280041F66C63C2F20003DA7240F66063C2F216
:10FC380000034FF001021A7018E140F66463C2F243
:10FC480000035B7903F00103002B09D040F66463DD
:10FC5800C2F200031B79032B02D14FF0010301E02C
:10FC68004FF0000303F00103DAB240F65E63C2F21C
:10FC780000031A7040F65E63C2F200031B7883F03B
:10FC88000103DBB2002B00F0F08041F66C63C2F296
:10FC980000034FF00002DA72E7E040F66463C2F254
:10FCA8000003DB7A03F00103002B09D040F66463FC
:10FCB800C2F200039B7A032B02D14FF0010301E04B
:10FCC8004FF0000303F00103DAB240F65E63C2F2BC
:10FCD80000031A7040F65E63C2F200031B7883F0DB
:10FCE8000103DBB2002B06D041F66C63C2F20003BD
:10FCF8004FF00002DA7240F66463C2F2000393F830
:10FD08002F2041F65463C2F200031A70AEE040F6A9
:10FD18006463C2F200035B699AB241F6F053C2F21F
:10FD280000031A8040F66463C2F200039A6948F639
:10FD3800AD33C6F6DB0383FB02134FEA23314FEAE8
:10FD4800E273CB1A9AB240F62853C2F200031A8023
:10FD580040F66163C2F200034FF001021A7085E0B9
:10FD680040F66463C2F200031A7941F65563C2F2A1
:10FD780000031A7041F65563C2F200031B78102B7A
:10FD880006D941F65563C2F200034FF010021A700B
:10FD98004FF000037B605BE040F66462C2F2000251
:10FDA80079680B464FEA43035B184FEA8303D3187D
:10FDB80003F108031A7841F6D053C2F200037968B8
:10FDC8005B181A7040F66462C2F2000279680B464A
:10FDD8004FEA43035B184FEA8303D31803F1080380
:10FDE8005A7841F62C63C2F2000379685B181A70DE
:10FDF80040F66462C2F2000279680B464FEA430398
:10FE08005B184FEA8303D31803F10803DA7841F645
:10FE18004463C2F2000379685B181A7040F66462A2
:10FE2800C2F2000279680B464FEA43035B184FEAB7
:10FE38008303D31803F108031A7941F65863C2F211
:10FE4800000379685B181A707B6803F101037B6013
:10FE580041F65563C2F200031B781A467B689A4242
:10FE68009ADC03E04FF0000324E000BF40F6606333
:10FE7800C2F200031B78002B1AD040F66163C2F26D
:10FE880000031B78002B13D040F66063C2F2000316
:10FE98004FF000021A7040F66063C2F200031A784D
:10FEA80040F66163C2F200031A704FF0010301E0EB
:10FEB8004FF00003184607F10C07BD4680BC704799
:10FEC80090B583B000AF41F63C53C2F200031B88E3
:10FED8001BB21846F0F752FE034618464FF6352176
:10FEE800C3F68E41F0F79EFE0346184608F02AFD39
:10FEF800786041F63C53C2F200031B881BB21846D7
:10FF0800F0F73CFE034618464FF63521C3F68E41FE
:10FF1800F0F788FE0346184608F0A0FC386041F662
:10FF28001863C2F200031B68DB78002B00F0D58051
:10FF380041F6E453C2F200035B889CB241F6EC53ED
:10FF4800C2F200035B881AB241F6E453C2F200031E
:10FF58005B881BB2D31A1846FFF740F8014641F6F2
:10FF68001863C2F200031B68DB78C3F1000241F694
:10FF78001863C2F200031B68DB78084611461A466C
:10FF8800F6F722FD03469BB2E3189BB29AB241F6FC
:10FF9800E453C2F200035A8041F6E453C2F200036C
:10FFA8001B889CB241F6EC53C2F200031B881AB2BC
:10FFB80041F6E453C2F200031B881BB2D31A184659
:10FFC800FFF70CF8014641F61863C2F200031B68FC
:10FFD800DB78C3F1000241F61863C2F200031B6824
:10FFE800DB78084611461A46F6F7EEFC03469BB244
:08FFF800E3189BB29AB241F636
:020000040801F1
:10000000E453C2F200031A8041F6E453C2F2000343
:100010005B881BB21846F0F7B5FD034618463968F1
:10002000F0F704FE03461C4641F6E453C2F2000317
:100030001B881BB21846F0F7A5FD034618467968E1
:10004000F0F7F4FD034620461946F0F7E5FC0346B9
:1000500018464FF00001C4F22011F0F79BFE034652
:100060001846F0F7A9FF03469AB240F62453C2F2AD
:1000700000031A8041F6E453C2F200035B881BB20E
:100080001846F0F77FFD034618467968F0F7CEFD75
:1000900003461C4641F6E453C2F200031B881BB220
:1000A0001846F0F76FFD034618463968F0F7BEFDB5
:1000B000034620461946F0F7B1FC034618464FF0B8
:1000C0000001C4F22011F0F765FE03461846F0F770
:1000D00073FF03469AB240F62453C2F200035A80DB
:1000E0006BE041F6EC53C2F200035B881BB218468A
:1000F000F0F748FD034618463968F0F797FD0346C8
:100100001C4641F6EC53C2F200031B881BB2184692
:10011000F0F738FD034618467968F0F787FD034687
:1001200020461946F0F778FC034618464FF00001C8
:10013000C4F22011F0F72EFE03461846F0F73CFFFC
:1001400003469AB240F62453C2F200031A8041F6E5
:10015000EC53C2F200035B881BB21846F0F712FDA5
:10016000034618467968F0F761FD03461C4641F6E0
:10017000EC53C2F200031B881BB21846F0F702FDD5
:10018000034618463968F0F751FD034620461946E4
:10019000F0F744FC034618464FF00001C4F220116A
:1001A000F0F7F8FD03461846F0F706FF03469AB24B
:1001B00040F62453C2F200035A8007F10C07BD46F3
:1001C00090BD00BF80B500AF41F66C63C2F2000382
:1001D000DB7A002B00F0A68041F65463C2F20003E4
:1001E0001B78042B40F29E8041F68063C2F200032C
:1001F0009B7A002B2BD041F66C63C2F20003DB79B3
:10020000002B40F0A58041F66C63C2F200034FF072
:100210000102DA7141F66C63C2F200034FF0000292
:100220001A7240F24803C2F200034FF000021A7043
:1002300041F62060C2F200004649FEF7B1F940F6EF
:100240002A53C2F200034FF002021A7080E041F616
:100250006C63C2F200034FF00002DA7141F6806372
:10026000C2F20003DB7A002B43D041F61863C2F2DE
:1002700000031B685B89184600F0F2F80346002B68
:1002800037D041F66C63C2F200031B7A002B48D1D1
:1002900041F66C63C2F200034FF001021A7240F2A1
:1002A0004803C2F200034FF000021A7041F63C63AB
:1002B000C2F200031A6841F6F453C2F200031A6056
:1002C00041F63C63C2F200035A6841F6F453C2F2AD
:1002D00000035A6041F6F450C2F200001E49FEF7D6
:1002E0005FF940F62A53C2F200034FF001021A7080
:1002F00017E041F66C63C2F200034FF000021A727D
:1003000040F24803C2F200031B78002B20D140F2D8
:100310004803C2F200034FF001021A70FDF762FFBA
:1003200016E015E041F66C63C2F200034FF00002E4
:10033000DA7141F66C63C2F200034FF000021A72E8
:1003400040F62A53C2F200034FF000021A7000E098
:1003500000BF80BD241E0020F81D002080B483B0A3
:1003600000AF786040F62C73C2F200031B687A6815
:10037000D31A002B1EDB41F65463C2F200031B7834
:10038000042B17D97B6803F5123202F5F87240F698
:100390002C73C2F200031A604FF48053C4F60003BA
:1003A0004FF48052C4F60002928A92B282F48842DC
:1003B00092B29A8207F10C07BD4680BC704700BF1D
:1003C00080B483B000AF786040F65873C2F2000387
:1003D0001A687B681340002B0CBF00230123DBB29B
:1003E000184607F10C07BD4680BC704780B483B047
:1003F00000AF786040F65873C2F200031A687B6859
:100400001A4340F65873C2F200031A6007F10C0752
:10041000BD4680BC704700BF80B483B000AF786039
:100420007B686FEA030240F65873C2F200031B6850
:100430001A4040F65873C2F200031A6007F10C0725
:10044000BD4680BC704700BF80B400AF40F6587313
:10045000C2F200031B681846BD4680BC704700BF4F
:1004600080B483B000AF0346FB8041F69863C2F2CC
:1004700000031B881BB283EAE372A2EBE372FB88E2
:100480009A420FDA41F69863C2F200035B881BB20E
:1004900083EAE372A2EBE372FB889A4202DA4FF03E
:1004A000010301E04FF0000303F00103DBB2184643
:1004B00007F10C07BD4680BC704700BF80B485B013
:1004C00000AF78604FF00003FB7329E0F97B7B6895
:1004D0005B78FA7BF87B00FB02F2A2F1190202FBC7
:1004E00003F303F6C413FA7B02FB03F37A68127872
:1004F00002FB03F248F6AD33C6F6DB0383FB0203CF
:100500004FEAA3204FEAE273C31A9AB241F6B863E6
:10051000C2F2000323F81120FB7B03F10103FB73FC
:10052000FB7B062BD2D907F11407BD4680BC704770
:10053000F0B484B000AF786039604FF00003FB7313
:1005400084E0FB7B9BB21A464FEA8202D3184FEA43
:1005500043039AB27B689B78D31A9BB2BB814FF05E
:100560000103BB73B7F90C30002B04DD7B689B786B
:10057000C3F16403BB73B7F90C30002B02DA7B685C
:100580009B78BB73F97B7B689B781A464FEA8202A3
:10059000D3184FEA430398B2B7F90C307A68D2788F
:1005A000C2F164047A68D278B7F90C50B7F90C60DC
:1005B00006FB05F505FB02F5BA7BBE7B06FB02F2E6
:1005C00095FBF2F2A21802FB03F246F26763C6F251
:1005D000666383FB02C34FEAA3044FEAE273E31AA4
:1005E0009BB2C3189BB29AB241F6A063C2F2000359
:1005F00023F81120F97B3B6818883B685B881A4612
:100600003B681B88D21AFC7B41F6A063C2F2000350
:1006100033F814301BB203FB02F244F6D353C1F299
:10062000620383FB02C34FEAA3144FEAE273E31AA7
:100630009BB2C3189BB29AB241F6A063C2F2000308
:1006400023F81120FB7B03F10103FB73FB7B0B2BD6
:100650007FF677AF07F11007BD46F0BC704700BFCB
:1006600080B584B000AF786039604FF00003FB7351
:100670000DE0FA7B7B685B8999B241F6CC63C2F2EC
:10068000000323F81210FB7B03F10103FB73FB7BD8
:10069000112BEED94FF00800F6F724F90346002B92
:1006A00004D07868396800F011F80AE041F6C860B3
:1006B000C2F20000396840F65C72C2F2000200F03B
:1006C0001FFA07F11007BD4680BD00BF80B582B09C
:1006D00000AF786039607B681B7A042B40D801A298
:1006E00052F823F0F9060108F9060108130701087A
:1006F0002D07010847070108786841F6C861C2F272
:1007000000013A6840F65C73C2F2000300F0D4FCCA
:1007100026E0786841F6C861C2F200013A6840F606
:100720005C73C2F2000300F001FA19E0786841F648
:10073000C861C2F200013A6840F65C73C2F200037D
:1007400000F082FB0CE0786841F6C861C2F200015B
:100750003A6840F65C73C2F2000300F0A1F900BFF2
:1007600007F10807BD4680BD80B582B000AF786054
:100770007B681B7A042B1DD801A252F823F000BF1E
:1007800095070108950701089D070108A5070108BD
:10079000AD07010800F05EFD03460DE000F084FAAD
:1007A000034609E000F006FC034605E000F058F9B6
:1007B000034601E04FF00003184607F10807BD4665
:1007C00080BD00BFB0B584B000AF786039604FF035
:1007D0000800F6F787F80346002B1DD04FF0000302
:1007E000FB7315E0FC7B40F65C73C2F200031B68F0
:1007F000FA7B78683968984703469AB241F6CC6329
:10080000C2F2000323F81420FB7B03F10103FB7306
:10081000FB7B072BE6D9CEE040F66073C2F2000303
:100820001B7803F10103DAB240F66073C2F20003F1
:100830001A7040F66073C2F200031B7803F00303E2
:100840007B734FF00003FB73B1E0FD7B7C7B40F6D4
:100850005C73C2F200031B68FA7B786839689847BA
:10086000034699B240F66473C2F200034FEA850270
:10087000121923F81210FA7B40F6A473C2F2000397
:100880004FF0000123F812104FF00003BB7321E07A
:10089000FA7BF97B40F6A473C2F2000333F81130FF
:1008A00099B2FC7BB87B40F66473C2F200034FEA56
:1008B0008404201833F810309BB2CB189BB299B245
:1008C00040F6A473C2F2000323F81210BB7B03F1BD
:1008D0000103BB73BB7B032BDAD9FA7BF97B40F6B0
:1008E000A473C2F2000333F811301BB203F1020308
:1008F000002B01DA03F103034FEAA30399B240F698
:10090000A473C2F2000323F81210FA7B40F6A4731A
:10091000C2F2000333F812301AB2F97B41F6CC630D
:10092000C2F2000333F811301BB2A3F103039A4261
:1009300012DAFA7BF97B40F6A473C2F2000333F8B3
:1009400011309BB203F102039BB299B241F6CC6322
:10095000C2F2000323F81210FA7B40F6A473C2F22D
:10096000000333F812301AB2F97B41F6CC63C2F2BD
:10097000000333F811301BB203F103039A4212DD76
:10098000FA7BF97B40F6A473C2F2000333F811300E
:100990009BB2A3F102039BB299B241F6CC63C2F2BF
:1009A000000323F81210FB7B03F10103FB73FB7BB5
:1009B000072B7FF64AAF07F11007BD46B0BD00BF59
:1009C00080B584B000AF786039607B68FB601CE064
:1009D000FB681B784DF2D420C0F6010019460AF0DE
:1009E00053F8B860BB68002B0BD0BA684DF2D42323
:1009F000C0F60103D31AF9687A688A1AD1B23A6844
:100A0000D154FB6803F10103FB60FB681B78002BEA
:100A1000DED107F11007BD4680BD00BF80B485B0B0
:100A200000AFF860B9601346FB71FA7941F6CC6308
:100A3000C2F2000333F812309BB2184607F11407D4
:100A4000BD4680BC704700BF80B400AF40F6B473B1
:100A5000C2F200034FF001021A70BD4680BC70471D
:100A600080B500AF40F6B473C2F200031B78002BD0
:100A700011D041F21823C2F200031B681B681B68E7
:100A8000984740F6B473C2F200034FF000021A70A8
:100A90004FF0010301E04FF00003184680BD00BF96
:100AA00080B485B000AFF860B9607A603B6041F215
:100AB0001823C2F200037A681A603B68002B05D045
:100AC0003A6840F61D23C0F60103136007F11407CE
:100AD000BD4680BC704700BF80B584B000AFF860F1
:100AE000B9601346FB71FB79FA68D35C1846F2F7DC
:100AF0000FFE0346184607F11007BD4680BD00BF34
:100B000080B485B000AFF860B9607A607A6840F66A
:100B1000D923C0F601031360FB684FF008021A7076
:100B200007F11407BD4680BC704700BF80B586B092
:100B300000AFF860B9607A603B6041F21823C2F2FE
:100B400000037A681A604FF000037B6111E0FB68D4
:100B50005B89A3F577734FEA4303194640F6B873F0
:100B6000C2F200037A6943F822107B6903F10103A2
:100B70007B617B69072BEADD4FF48840C4F20000FB
:100B800040F6C931C0F6010148F2A062C0F201028C
:100B90004FF00503F2F7E4FD024641F60473C2F29A
:100BA0000003DA603B68002B05D03A6840F60D631D
:100BB000C0F601031360BB684FF008021A7007F11A
:100BC0001807BD4680BD00BF80B584B000AF0346A6
:100BD000FB80F9F77FFAF86040F6F473C2F2000385
:100BE0001B68FA68D21A40F6C4139A4206D940F636
:100BF000F873C2F200034FF000021A7040F6F4736B
:100C0000C2F20003FA681A6040F6F873C2F20003F9
:100C10001B78002B02D1FB880F2B3FD140F6B57318
:100C2000C2F200034FF000021A7040F6F873C2F2ED
:100C300000031B78002B0DD040F6F873C2F20003BE
:100C40001B7803F1FF32FB88D9B240F6D873C2F2A9
:100C50000003995440F6F873C2F200031B78182B76
:100C60000ED140F6B573C2F200034FF001021A70C4
:100C700040F6F873C2F200034FF000021A700EE063
:100C800040F6F873C2F200031B7803F10103DAB2F5
:100C900040F6F873C2F200031A7000E000BF07F1DB
:100CA0001007BD4680BD00BF80B500AF40F6B573EC
:100CB000C2F200031B78002B00F0A48040F6D8732A
:100CC000C2F200039B7D4FEAD303DBB203F00103C2
:100CD000002B40F0908041F21823C2F200031B6801
:100CE0001B681B68984740F6D873C2F200031B8844
:100CF000C3F30A039BB21A4640F6B873C2F200036C
:100D00001A6040F6D873C2F200031B68C3F3CA230B
:100D10009BB21A4640F6B873C2F200035A6040F61E
:100D2000D873C2F200035A884FEA921292B21B792A
:100D300003F001034FEA832313439BB21A4640F6A4
:100D4000B873C2F200039A6040F6D873C2F200038F
:100D50009B88C3F34A039BB21A4640F6B873C2F2AB
:100D60000003DA6040F6D873C2F200035B68C3F395
:100D70000A339BB21A4640F6B873C2F200031A61F6
:100D800040F6D873C2F20003DA884FEAD21292B268
:100D90001B7A03F003034FEA432313439BB21A4623
:100DA00040F6B873C2F200035A6140F6D873C2F23B
:100DB00000031B89C3F38A039BB21A4640F6B8733B
:100DC000C2F200039A6140F6D873C2F200039B6836
:100DD000C3F34A339BB21A4640F6B873C2F200031B
:100DE000DA6140F6B573C2F200034FF000021A70E8
:100DF0004FF0010308E040F6B573C2F200034FF074
:100E000000021A704FF00003184680BD80B485B010
:100E100000AFF860B9601346FB71FB79FA68D35CE8
:100E20001A4640F6B873C2F2000353F822304FEA74
:100E300053039BB203F577739BB2184607F114076F
:100E4000BD4680BC704700BF80B584B000AFF8607D
:100E5000B9607A603B6041F21823C2F200037A68FD
:100E60001A604FF48840C4F2000040F6AD61C0F64D
:100E700001014FF4E1324FF00103F2F771FC024639
:100E800041F60473C2F20003DA603B68002B05D020
:100E90003A6841F28503C0F601031360BB684FF066
:100EA00008021A7007F11007BD4680BD80B584B0F6
:100EB00000AF0346FB80F9F70DF9F86041F2380303
:100EC000C2F200031B68FA68D31AB3F57A6F06D929
:100ED00041F23C03C2F200034FF000021A7041F2EB
:100EE0003803C2F20003FA681A6041F23C03C2F20E
:100EF00000031B78002B09D1FB88A82B55D140F6A5
:100F0000F973C2F200034FF000021A7041F23C0381
:100F1000C2F200031B78022B06D1FB88DAB241F241
:100F20003403C2F200031A7041F23C03C2F2000320
:100F30001B78142B0CD841F23C03C2F200031B783F
:100F40001A46FB88D9B241F21C03C2F2000399543D
:100F500041F23C03C2F200031B7803F10103DAB251
:100F600041F23C03C2F200031A7041F23C03C2F2A8
:100F700000031B781A4641F23403C2F200031B78C7
:100F80004FEA430303F105039A420FD141F23C03B8
:100F9000C2F200034FF000021A7040F6F973C2F279
:100FA00000034FF001021A7000E000BF07F11007C4
:100FB000BD4680BD80B582B000AF40F6F973C2F285
:100FC00000031B78002B55D040F6F973C2F20003E2
:100FD0004FF000021A7041F21C03C2F200035B786A
:100FE000012B47D141F21823C2F200031B681B6892
:100FF0001B68984741F23403C2F200031B78082BA8
:1010000006D941F23403C2F200034FF008021A700D
:101010004FF00003FB7122E0FA79FB794FEA4303BA
:1010200003F1030141F21C03C2F200035B5C4FEACF
:101030000321FB7903F102034FEA430041F21C0351
:10104000C2F200031B5C0B43194640F6FC73C2F26C
:10105000000343F82210FB7903F10103FB7141F215
:101060003403C2F200031B78FA799A42D4D34FF0CA
:10107000010301E04FF00003184607F10807BD46E1
:1010800080BD00BF80B485B000AFF860B960134682
:10109000FB71FB79FA68D35C1A4640F6FC73C2F226
:1010A000000353F822304FEAD3039BB2184607F1EE
:1010B0001407BD4680BC704780B584B000AFF860AF
:1010C000B9607A603B6041F21823C2F200037A688B
:1010D0001A60FB681B7A002B1BD0012B33D141F225
:1010E0003D03C2F200034FF003021A7041F23E03C7
:1010F000C2F200034FF007021A7041F24003C2F23D
:1011000000034FF001021A70BB684FF00C021A7016
:1011100019E041F23D03C2F200034FF002021A70DF
:1011200041F23E03C2F200034FF003021A7041F293
:101130004003C2F200034FF000021A70BB684FF088
:1011400007021A7000BF4FF48840C4F2000041F259
:101150008911C0F601014FF4E1324FF00103F2F7BB
:10116000FFFA024641F60473C2F20003DA603B68FC
:10117000002B05D03A6841F26D23C0F601031360DD
:1011800007F11007BD4680BD80B584B000AF0346AF
:10119000FB8041F24103C2F200034FF001021A70DA
:1011A000F8F798FFF86041F27403C2F200031B687D
:1011B000FA68D21A41F27803C2F200031A6041F2CF
:1011C0007403C2F20003FA681A6041F27803C2F2B3
:1011D00000031A6841F288339A4206D941F27C032F
:1011E000C2F200034FF000021A7041F27C03C2F217
:1011F00000031B781A46FB88D9B241F6F063C2F2AD
:101200000003995441F27C03C2F200031B780F2BB8
:101210000FD141F23F03C2F200034FF001021A70F6
:1012200041F21823C2F200031B681B681B68984731
:101230000CE041F27C03C2F200031B7803F10103CE
:10124000DAB241F27C03C2F200031A7007F1100710
:10125000BD4680BD80B400AF41F23F03C2F200033F
:101260001B781846BD4680BC704700BF80B487B06D
:1012700000AFF860B9601346FB7141F23F03C2F260
:1012800000031B78002B4FD04FF003037B7541E028
:101290007B7D03F1FF3241F6F063C2F200039B5CF9
:1012A000DBB21A4641F23D03C2F200031B7842FA58
:1012B00003F3DBB203F00F033B75BB681B783A7D89
:1012C0009A4223D23B7D0B2B20D83A7D7B7D03F1C4
:1012D000FF3141F6F063C2F200035B5CD9B241F228
:1012E0003E03C2F200031B780B40DBB24FEA03213E
:1012F000787D41F6F063C2F200031B5CDBB2C918D3
:1013000041F24403C2F2000343F822107B7D03F153
:1013100002037B757B7D0F2BBAD941F23F03C2F2EA
:1013200000034FF000021A70BB681B78FA799A42EA
:1013300009D241F24103C2F200031B7883F001039A
:10134000DBB2002B03D0FB685B89FB8225E041F216
:101350004003C2F200031B78002B10D0FB79FA681F
:10136000D35C1A4641F24403C2F2000353F8223020
:101370004FEA53039BB203F57773FB820DE0FB79D1
:10138000FA68D35C1A4641F24403C2F2000353F8F0
:1013900022309BB203F57773FB82FB8A184607F174
:1013A0001C07BD4680BC704780B483B000AF786036
:1013B00041F60073C2F200037A681A6007F10C0765
:1013C000BD4680BC704700BF80B400AF41F60073DB
:1013D000C2F200031B681B78002B14BF00230123FB
:1013E000DBB21846BD4680BC704700BF80B400AF7A
:1013F00041F60073C2F200031B681B78012B14BF77
:1014000000230123DBB21846BD4680BC704700BFF5
:1014100080B500AF4FF40060F5F764FA034683F03F
:101420000103DBB2002B02D04FF000032EE04FF09F
:101430004000F5F757FA034683F00103DBB2002BB7
:1014400012D041F60073C2F200031B685B78012BD7
:1014500007D041F60073C2F200031B685B78022BD1
:1014600002D14FF0000311E0FFF7C0FF0346002B4D
:101470000AD041F60073C2F200031B685B78002BB0
:1014800002D14FF0000301E04FF00103184680BD88
:1014900080B582B000AF7860F5F780FA034683F03C
:1014A0000103DBB2002B07D041F60073C2F2000348
:1014B0001B684FF000025A70FFF7AAFF03461A4656
:1014C00041F27D03C2F200031A7041F60073C2F2CA
:1014D00000031B685B78012B06D17A6841F21C235C
:1014E000C2F2000393600FE041F60073C2F2000302
:1014F0001B685B78022B03D17B68064A9A6003E085
:101500007B681A687B689A6000F072F807F1080738
:10151000BD4680BD6414002080B483B000AF4FF09E
:101520000103FB7141F60073C2F200031B685B7894
:10153000002B1CD141F60073C2F200031B689B789C
:10154000002B0AD141F66C63C2F200035B78002BDA
:101550000CBF00230123FB7109E041F68063C2F256
:1015600000031B7D002B0CBF00230123FB71FB79C3
:10157000184607F10C07BD4680BC704780B483B0A5
:1015800000AF0346FB7141F27E03C2F200031B78F9
:10159000FA799A420CBF00230123DBB2184607F107
:1015A0000C07BD4680BC704780B500AFFFF70CFF4D
:1015B0000346002B01D000F0B5FBFFF717FF0346F1
:1015C000002B01D000F03CFF80BD00BF80B500AF14
:1015D000FFF7FAFE0346002B01D000F095FBFFF762
:1015E00005FF0346002B01D000F038FF80BD00BF8F
:1015F00080B582B000AF41F27D03C2F200031B78D8
:1016000083F00103DBB2002B1CD1FFF785FF0346FB
:10161000FB71FB791846FFF7B1FF034683F0010326
:10162000DBB2002B10D1FB79002B02D0FFF7BCFFFF
:1016300001E0FFF7CBFF41F27E03C2F20003FA792B
:101640001A7002E000BF00E000BF07F10807BD46C6
:1016500080BD00BF80B500AF41F27D03C2F2000340
:101660001B7883F00103DBB2002B16D1FFF754FF88
:10167000034683F00103DBB2002B0ED1FFF7A4FE7B
:101680000346002B01D000F085FBFFF7AFFE0346B9
:10169000002B03D000F0F0FE00E000BF80BD00BFD3
:1016A00080B582B000AF0346FB7141F60473C2F20D
:1016B00000039B6818464FF05E01F8F7A9FB41F65E
:1016C0000473C2F200039A68FB7910461946F8F7D2
:1016D0009FFB07F10807BD4680BD00BF80B500AF86
:1016E00041F60473C2F200039B6818464FF05E0196
:1016F000F8F78EFB80BD00BF80B582B000AF034617
:10170000FB71FB795E2B14D141F60473C2F2000326
:101710009B6818464FF05D01F8F77AFB41F60473B9
:10172000C2F200039B6818464FF03E01F8F770FBC9
:1017300021E0FB795D2B14D141F60473C2F2000362
:101740009B6818464FF05D01F8F762FB41F60473A1
:10175000C2F200039B6818464FF03D01F8F758FBB2
:1017600009E041F60473C2F200039A68FB7910465F
:101770001946F8F74DFB07F10807BD4680BD00BFCD
:1017800080B584B000AF0346FB80FB88FB73FB7B16
:101790001846FFF7B1FFB7F906304FEA23239BB293
:1017A000FB73FB7B1846FFF7A7FF07F11007BD4649
:1017B00080BD00BF90B583B000AF4FF000037B60E9
:1017C00036E07B68DBB203F12403DBB21846FFF797
:1017D00067FF41F66853C2F200037A6833F81230AB
:1017E0001BB21846EFF7CEF9044640F22203C2F2CC
:1017F00000031B881846EFF7C5F903462046194633
:10180000EFF7C8FA034618464FF00001C4F27A41D8
:10181000EFF70CFA03461846EFF7CEFB03469BB2F0
:101820001BB21846FFF7ACFF7B6803F101037B6036
:101830007B68022BC5DD07F10C07BD4690BD00BFDC
:1018400080B500AF4FF01000FFF72AFF40F640339D
:10185000C2F200031A6848F21F53C5F2EB1383FB70
:1018600002134FEA63114FEAE273CB1A9BB21BB229
:101870001846FFF785FF4FF02100FFF711FF40F6F4
:101880004033C2F200031A6848F21F53C5F2EB134B
:1018900083FB02134FEA63114FEAE273CB1A4FF056
:1018A000640101FB03F3D31A002BB8BF5B429BB268
:1018B0001BB21846FFF764FF80BD00BF80B500AFC4
:1018C0004FF00200FFF7ECFE41F6EC43C2F20003DA
:1018D0001B881AB246F26763C6F2666383FB021383
:1018E0004FEAA3014FEAE273CB1A9BB21BB2184630
:1018F000FFF746FF80BD00BF80B582B000AFF8F7AC
:1019000017FC024644F6D353C1F26203A3FB021351
:101910004FEA93137B607A6848F68903C8F6880318
:10192000A3FB02134FEA531148F68903C8F6880354
:10193000A3FB01234FEA531213464FEA03139B1AEA
:101940004FEA8303CA1A1346FB704FF01700FFF7E4
:10195000A7FEFB784FEA03239BB21BB21846FFF7A2
:101960000FFF4FF01800FFF79BFE796848F68903D8
:10197000C8F68803A3FB01234FEA531213464FEA2C
:1019800003139B1A4FEA8303CA1A93B21BB2184679
:10199000FFF7F6FE07F10807BD4680BD80B500AF32
:1019A0004FF01300FFF77CFE41F63C63C2F20003E8
:1019B0001B6883EAE372A2EBE3724BF28953C1F234
:1019C000F84383FB02134FEA63314FEAE273CB1A09
:1019D0009BB21BB21846FFF7D3FE4FF01B00FFF778
:1019E0005FFE41F63C63C2F200031B6883EAE372C8
:1019F000A2EBE37246F26763C6F2666383FB0213EF
:101A00004FEAA3014FEAE273CA1A48F6AD33C6F6AD
:101A1000DB0383FB02134FEA23314FEAE273CB1A55
:101A200042F2107101FB03F3D31A9BB21BB21846AA
:101A3000FFF7A6FE4FF02300FFF732FE41F63C63AE
:101A4000C2F200031B68002B02DA4FF0530301E0DF
:101A50004FF04E031BB21846FFF792FE4FF01200F4
:101A6000FFF71EFE41F63C63C2F200035B6883EAA7
:101A7000E372A2EBE3724BF28953C1F2F84383FBAA
:101A800002134FEA63314FEAE273CB1A9BB21BB2E7
:101A90001846FFF775FE4FF01A00FFF701FE41F6FA
:101AA0003C63C2F200035B6883EAE372A2EBE37279
:101AB00046F26763C6F2666383FB02134FEAA30133
:101AC0004FEAE273CA1A48F6AD33C6F6DB0383FB6E
:101AD00002134FEA23314FEAE273CB1A42F210713C
:101AE00001FB03F3D31A9BB21BB21846FFF748FE63
:101AF0004FF02200FFF7D4FD41F63C63C2F2000331
:101B00005B68002B02DA4FF0570301E04FF045030A
:101B10001BB21846FFF734FE80BD00BF80B500AF92
:101B20004FF03000FFF7BCFD40F60843C2F200035F
:101B30001B689BB21BB21846FFF722FE80BD00BF98
:101B400080B582B000AF41F66C03C2F200031A7890
:101B500040F22003C2F200031B78B2FBF3F3DBB2C6
:101B60007B607B6840F6340202FB03F34FEA5302CA
:101B700040F63143C3F2C303A3FB02134FEA9303BE
:101B80007B6041F28603C2F200031B881A4640F2D2
:101B90002003C2F200031B7892FBF3F103FB01F375
:101BA000D31A7B807B884FEA03133B807B689BB210
:101BB0004FEA03239AB23B8813433B807B6803F4CC
:101BC00070634FEA13239AB23B8813433B804FF074
:101BD0000600FFF765FD3B881BB21846FFF7D0FDF6
:101BE00041F28603C2F200031B8803F101039AB29B
:101BF00041F28603C2F200031A8041F28603C2F268
